:020000040800F2
:1000000000200010C98E02084538020845F6000895
:10001000413802083D380208393802080000000063
:100020000000000000000000000000003538020859
:1000300031380208000000002D38020885E1000870
:10004000318F0208318F0208318F0208318F020888
:10005000318F0208318F02088DF00008B9F10008D5
:100060007DF1000841F1000805F1000871BB0008AE
:1000700061BB000851BB000841BB000831BB000850
:100080001DBB000809BB0008318F0208318F020830
:100090006D3B0208318F0208318F0208C9F0000859
:1000A000DDFF00081D000108CDFF00084500010824
:1000B0000D000108FDFF0008EDFF0008318F020868
:1000C000318F0208318F0208318F0208318F020808
:1000D000318F0208B1E2000835E20008B9E10008FA
:1000E00051F00008318F02081D380208318F0208D4
:1000F000318F0208318F0208318F0208318F0208D8
:10010000000000000000000000000000318F020825
:10011000318F0208318F0208318F0208318F0208B7
:10012000F5BA0008E1BA0008CDBA0008B9BA00086B
:10013000A5BA0008318F020800000000000000008E
:10014000318F0208318F0208318F02080000000051
:10015000000000000000000000000000000000009F
:100160000000000000000000318F0208318F0208FB
:10017000318F0208000000000000000000000000B5
:0801800000000000318F0208AD
:100188002DE9F04FB0F908502DED048B0D81EDB23B
:10019800382D8FB00C4600F061848046914634D9E2
:1001A800802D00F0EF8078D8522D00F09F8040F22B
:1001B8004382542D00F08E846E2D40F00B817A4BD3
:1001C8000A681B88794DFF2BA8BFFF23511C2160AB
:1001D8001370A96881F3100189B220460AF0A4FDC2
:1001E800734B204619880AF09FFD296801F30F0117
:1001F80089B2204601250AF097FD2B4628466381DF
:100208000FB0BDEC048BBDE8F08F042D00F04D84D9
:1002180040F2E581202D71D040F2F981242D00F0C3
:100228005084282D40F0D6800B68DFF8A481614EF9
:10023800591C022221601A70236806275A1C226062
:100248001F7023680A22591C21601A70236801252F
:100258005A1922601D70B8F8001020460AF064FD93
:10026800B8F8021020460AF05FFD23685A19226088
:100278001F7023685022591921601A7023680022C0
:10028800591921601A70318820460AF04DFD71888D
:1002980020460AF049FD2B46B0E7822D4AD0C0F02F
:1002A8003284A02D00F02384FE2D40F09380424D2F
:1002B80005F1080635F8021B20460AF035FDB5425F
:1002C800F8D101252B4699E7531C1146C8F8003090
:1002D8003A4811F8023B0372C8F80010527842728B
:1002E800042B42F2D080FF2B01F0B0872268002156
:1002F800531C012523602B4611707FE70B68304D96
:10030800591C6A7821601A7023682A78591C216060
:100318001A702368AA78591C21601A70E988204647
:100328000AF002FD23682A79591C21601A70226894
:100338006979DDE70B68234A1C4D1178204A581C5F
:1003480020601970D18820460AF0EEFC164B22680E
:100358001B88FF2B02F10101A8BFFF232160137046
:10036800A96881F3100189B220460AF0DDFC2968EA
:1003780001F30F0189B220460AF0D6FC124B22681D
:100388001978B5E70B68114A581C0A2112882060B1
:1003980019702168FF2A01F10103A8BFFF22012576
:1003A80023602B460A7029E75C4200206042002047
:1003B80050290020A8310020D2420020801B0020B4
:1003C800C84400209E42002030300020B831002070
:1003D800342B0020A5F10A03E72B00F2EA80DFE8BE
:1003E80013F05C04E800E800E800E800E800E80032
:1003F800E800E800E800E800E800E800E800E800B5
:10040800E800E800E800E800E800E800E800E800A4
:10041800E8009B08E800E800E8008A08E800E8002F
:10042800E8008508E8004408E800E800E800E8007B
:10043800E800A704E8008104E8006E04E800E8008A
:10044800E8005404FE04E800F404E800E800EB04C3
:10045800E800E800E800E800E800CD04E800E8006B
:10046800E800E8006A07E8004807E80043043007A6
:10047800E800E800E800E800E800E800E800D10744
:10048800E8008607E8001508E800E606E800A20686
:10049800E800E800E800E8007906B3063906110626
:1004A800FF05E800E800E605D805E8009E05810597
:1004B800E800E800E800E8007505E800E8005305F2
:1004C800E800E800E800420529051805E800E8000A
:1004D800E800E8000705E800E800E800E800E800B0
:1004E800E800E800E800E800E800E800E800E800C4
:1004F800E800E800E800E800E8007906E800E8001D
:10050800E800E800E800E800E800E800E800E800A3
:10051800E800E800E800E800E800E800E800E80093
:10052800E800E800E800E800E800E800E800E80083
:10053800E800E800E800E800E800E800E800E80073
:10054800E800E800E800E800E800E800E800E80063
:10055800E800E800E800E800E800E800E800E80053
:10056800E800E800E800E800E800E800E800E80043
:10057800E800E800E800E800E800E800E800E80033
:10058800E800E800E800E800E800E800E800E80023
:10059800E800E800E800E800E800E800E800E80013
:1005A800E800E800E800E800E800E800E800F708EC
:1005B800CC08742D00F0FE82772D53D1D8F8003086
:1005C800D8F804209A421EBF5A1CC8F8002019788F
:1005D8001F4A08BF002120460EF0C2FF71E6022D17
:1005E80000F0DF8200F2CB82012D7FF4F3AE0B68BE
:1005F8000022591C21601A7023685A1C22601D7041
:1006080022682421531C23602B461170F6E5052D22
:100618007FF4E0AE0B220F4920460AF055FB082272
:100628000D4920460AF050FB012507220B492046B8
:100638000AF04AFB2B46E1E5442D7FF4CBAE002AB5
:100648003FF43FAE064B136001252B46D6E500BFAD
:10065800A5F200084CDE020858DE020864DE020833
:1006680065F30008F52D01F0E985472D00F0B48207
:10067800292DD8F8003001F00785392D01F0EC84D8
:10068800212D01F0C284D8F804600B3DF61AEF2D35
:1006980001F2298401A252F825F000BF7F1F00084B
:1006A800EF1E0008EF1E0008EF1E0008EF1E0008EE
:1006B800EF1E0008EF1E0008EF1E0008EF1E0008DE
:1006C800EF1E0008EF1E0008EF1E0008EF1E0008CE
:1006D800EF1E0008EF1E0008EF1E0008EF1E0008BE
:1006E800EF1E0008EF1E0008EF1E0008EF1E0008AE
:1006F800EF1E0008EF1E0008EF1E0008151F000877
:10070800EF1E0008B71F0008EF1E0008FB1C0008BA
:10071800EF1E0008EF1E0008EF1E0008451E000827
:10072800EF1E00088F1D0008EF1E0008EF1E0008CE
:10073800EF1E0008EF1E0008EF1E00087F1D0008CE
:10074800EF1E00081D1D0008EF1E0008AD1E000862
:10075800EF1E0008EF1E0008EF1E0008EF1E00083D
:10076800CB020008EF1E0008591E0008EF1E000803
:10077800EF1E0008F91E0008EF1E0008EF1E000813
:10078800EF1E0008EF1E0008EF1E0008EF1E00080D
:10079800C51A0008EF1E0008EF1E0008EF1E00082B
:1007A800291C0008EF1E0008DB1B0008EF1E0008CC
:1007B800EF1E0008A71B0008EF1E0008EF1E000828
:1007C800EF1E0008EF1E0008EF1E0008EF1E0008CD
:1007D800EF1E0008D11A0008EF1E0008751C00085B
:1007E800EF1E0008391A0008EF1E0008D919000882
:1007F800EF1E0008AB190008EF1E0008EF1E0008E6
:10080800EF1E0008EF1E0008EF1E0008EF1E00088C
:10081800EF1E0008EF1E0008EF1E0008EF1E00087C
:10082800EF1E0008EF1E0008EF1E0008EF1E00086C
:10083800EF1E0008EF1E0008EF1E0008EF1E00085C
:10084800EF1E0008EF1E0008EF1E0008EF1E00084C
:10085800EF1E0008EF1E0008EF1E0008EF1E00083C
:10086800EF1E0008EF1E0008EF1E0008EF1E00082C
:10087800EF1E0008EF1E0008EF1E0008EF1E00081C
:10088800EF1E0008EF1E0008EF1E0008EF1E00080C
:10089800EF1E0008EF1E0008EF1E0008EF1E0008FC
:1008A800EF1E0008EF1E0008EF1E0008EF1E0008EC
:1008B800EF1E0008EF1E0008EF1E0008EF1E0008DC
:1008C800EF1E0008EF1E0008EF1E0008EF1E0008CC
:1008D800EF1E0008EF1E0008EF1E0008EF1E0008BC
:1008E800EF1E0008EF1E0008EF1E0008EF1E0008AC
:1008F800EF1E0008EF1E0008EF1E0008EF1E00089C
:10090800EF1E0008EF1E0008EF1E0008EF1E00088B
:10091800EF1E0008EF1E0008EF1E0008EF1E00087B
:10092800EF1E0008EF1E0008EF1E0008EF1E00086B
:10093800EF1E0008EF1E0008EF1E0008EF1E00085B
:10094800EF1E0008EF1E0008EF1E0008EF1E00084B
:10095800EF1E0008EF1E0008EF1E0008EF1E00083B
:10096800EF1E0008EF1E0008EF1E0008EF1E00082B
:10097800EF1E0008EF1E0008EF1E0008EF1E00081B
:10098800EF1E0008EF1E0008EF1E0008EF1E00080B
:1009980051190008EF1E000813190008EF1E00087F
:1009A800851800086B1800084F180008EF1E00088B
:1009B80035180008EF1E00080B180008EF1E000885
:1009C800AB170008EF1E000883170008EF1E000889
:1009D800EF1E0008611700082D170008E11600082F
:1009E800B3160008EF1E000891160008EF1E000855
:1009F800EF1E0008EF1E0008EF1E0008EF1E00089B
:100A0800EF1E0008EF1E0008EF1E0008EF1E00088A
:100A1800EF1E0008EF1E0008EF1E0008EF1E00087A
:100A2800EF1E0008EF1E0008EF1E000877160008EA
:100A3800EF1E0008EF1E00080D160008EF1E000844
:100A4800EF1E0008EF1E0008EF1E0008EF1E00084A
:100A5800EF1E0008EF1E0008F31500080A68B74BE0
:100A68000125511C2160157022680521501920604C
:100A7800117022680A215019206011702268002123
:100A8800501920601170226819785019206011706F
:100A98002268597850192060117022689978531982
:100AA80023602B461170FFF7A9BB2A46A4492046AC
:100AB8000AF00AF9002120460AF036F922680021D6
:100AC80016E4A04B1968204601250AF015F92B46B3
:100AD800FFF794BB0B6800215A1C2260197022682A
:100AE8000125531923602B461170FFF787BB964BDE
:100AF800084619680AF000F9944B204619680AF06C
:100B0800FBF8934BDEE7934A934E9368116803EB27
:100B180083034FF6FF725B009342A8BF13469142CE
:100B2800A8BF114623EAE37321EAE1719DB289B2B5
:100B38000A22002713E0B368316803EB83034FF6FA
:100B4800FF725B009342A8BF13469142A8BF1146AB
:100B580023EAE37321EAE1719DB289B25022236846
:100B6800581C206020461A700AF0DEF80137294622
:100B780020460AF0D9F8022FDDD1FFF7A2BB0B6897
:100B88000222591C21601A70236801255A19226013
:100B98001D7022680021531923602B461170FFF73E
:100BA8002DBB04226D49204601250AF08DF82B46FD
:100BB800FFF724BBD8F80030D8F804209A421EBFAB
:100BC8005A1CC8F800201978654A08BF0021204639
:100BD8000EF0C6FCFFF775BBD8F80430D8F8005003
:100BE80040465D1B0AF04CF8052D064601F2D483F9
:100BF80080252F464FF0010894E80C009B1A103B03
:100C0800DFF87491AB42B8BF9FB2D9F80C309B1B88
:100C18009F423146204688BF9FB20AF06DF8B8F16E
:100C2800000F01F0CF83D9F80C30D4F80080F21906
:100C3800934200D29F1B0AF071FC41463A46304667
:100C48000AF0ECFC2368A84203442360B8BF0021E3
:100C580002DBFFF736BB236801305A1CA84222602A
:100C68001970F8D1FFF72DBB236800255A1C2260A4
:100C78001D7023685A1C22601D7023685A1C22604C
:100C880029461D7020460AF037F800212046012524
:100C98000AF032F82B46FFF7B1BA324827F052FC77
:100CA80000287FF70EAB2F4B1D18226813F8011B85
:100CB800501CAB4220601170F7D1FFF702BB2A4DE0
:100CC8002A4E05F1280795F902100023F2568A42A8
:100CD80001F07D810C333C2BF8D10835BD42F2D1AF
:100CE800FFF7EFBA224B03F15A0522685979501CD5
:100CF8002060117022681978501C206011702268D9
:100D08005978501C2060117022689978501C206016
:100D180011702268D978501C2060117022681979E6
:100D28000633501C9D4220601170DED1FFF7C9BA0E
:100D3800104B2268597DFFF7DBBA00BF4B26002015
:100D480044DE02086C2B0020ACF7FF1FB0F7FF1F32
:100D5800B4F7FF1F6C310020AC3100203CDE0208E4
:100D68003DF30008F8420020486A0020C0490020EE
:100D780044300020204A0020880000200AF0D6FADB
:100D88002368B94D002803F101010CBF0222032298
:100D980021601A702988204609F0AEFFE9682046CC
:100DA80009F0AAFF0AF012FA01250146204609F0C7
:100DB800A3FF2B46FFF722BA0822AC49204601259B
:100DC80009F082FF2B46FFF719BA2268A84B501C7E
:100DD80099782060117022685978FFF789BA2268DB
:100DE8000121531823600D460B461170FFF706BA10
:100DF800A04D2046A98A09F097FFE98A204609F004
:100E080093FF298B2046012509F08EFF2B46FFF71B
:100E1800F5B92368984A99491078994A5D1C256064
:100E2800187023689278581C20601A702268897894
:100E3800FFF75EBA2268934B93491878551C2560D2
:100E4800107022685878551C2560107022689B78AD
:100E5800501C20601370C9882046012509F064FFE2
:100E68002B46FFF7CBB9884D2046298809F05CFF4F
:100E78006988204609F058FFA9882046012509F00D
:100E880053FF2B46FFF7BAB9804D05F16006A988D4
:100E9800204609F049FFE988204609F045FF2989DD
:100EA800204609F041FF2368AA7A591C21601A706C
:100EB8002368EA7A591C21601A7055F80C1B2046E1
:100EC80009F01AFFAE42E2D1FFF7FBB9704952238D
:100ED8002268501C2060137011F8013F002BF7D1D5
:100EE800FFF7EFB96B4D00232268286803EB430135
:100EF800561C405C266010702A6820680A44461C0C
:100F08005278266002702A6820680A440133927871
:100F1800411C0A2B21600270E6D1FFF7D2B95E4D61
:100F280023682A68591C127821601A702B68226875
:100F38009978531C2360002311702A6821681A4489
:100F480001335279481C032B20600A70F5D12368BD
:100F58002A68591C127A21601A7023682A68591C59
:100F6800D27821601A7023682A68591C1279216086
:100F78001A702B682046598909F0D6FE23682A681A
:100F8800591C527A21601A702B6822685978FFF729
:100F9800AFB9424B2046196809F0AEFE404B2046D7
:100FA8001988012509F0C0FE2B46FFF727B93D4DEA
:100FB8002046298809F0B8FE6988204609F0B4FE61
:100FC800B5F904303849DA1781FB0313C2EBA303E0
:100FD80099B22046012509F0A7FE2B46FFF70EB966
:100FE800324E3378002B3FF46CA9314F002537F887
:100FF800021F204609F098FE337801359D42F6DB42
:10100800FFF75FB92B4D2C4EDFF8C080DFF8C0909A
:10101800DFED2A8ADFED2A9A9FED2A9A05F120074B
:1010280008E02046043509F07FFEAF4206F11806B5
:101038003FF447A9717C0029F3D095ED008AB0EE02
:10104800480A28F0DFFA98F80030002B41F05F8159
:1010580081B2E6E710221C492046012509F034FE3A
:101068002B46FFF7CBB800BF88000020204A00209D
:10107800682B00202C450020746A00205C2B00207F
:10108800442B00203C2B0020C4400020F42D0020DD
:10109800A0B902080C43002000690020B01C002001
:1010A800201F002078430020676666668043002082
:1010B8001063002064290020F04F00200000404207
:1010C8000040744400E08244542900205445002024
:1010D800504A00200DF1140900220592DFF8A0A261
:1010E800984B03920492C9F80420904601214FF6C8
:1010F800FF7B07E008F10108B8F10B0F00F0DC876F
:101108001AF9011F4E1CF5D04BFA08F2D007F1D599
:101118001A8842FA08F2D207ECD5484601930AF039
:1011280037F8019BE6E72368874A8849D078884AD8
:101138005D1C2560187023681278581C20601A708E
:101148002268C978FFF7D4B8824E338AB3F5007F96
:1011580006F1340594BF01270427403655F8041BCF
:1011680091FBF7F1204689B209F0DEFDB542F5D1D1
:10117800794D7A4F05F10C06B5EC010AD7ED087ADE
:1011880080EE270A28F03EFA81B2204609F0CCFD0D
:10119800B542F1D1724D05F10C0655F8041B2046F5
:1011A80089B209F0C1FDB542F7D1FFF78AB800212D
:1011B800204609F0B9FD0021204609F0B5FD0021BF
:1011C800204609F0B1FD2268664D0023511C2160BC
:1011D800137022682968501C91F82F102060117034
:1011E80022682968501C91F83A1020601170226812
:1011F8002968501C91F83B10206011702268511C1E
:10120800216013702268511C216013702268511CE0
:10121800216013702B682046D98F09F085FD2B6853
:101228002046998F09F080FD23682A68591C92F896
:10123800312021601A702B68226893F83210FFF76A
:1012480057B82268484B0125511C21601570226847
:101258009978501920601170226819785019206007
:10126800117022685978531923602B461170FEF7C4
:10127800C5BF3E4E3378002B3FF423A83C4F0025D2
:10128800B846236817F81520591C21601A7098F879
:10129800011001EB810101EB810101F2EE2189B21C
:1012A800204609F041FD337801359D4208F10208D6
:1012B800E7DBFFF706B823682E4D591C2A78216012
:1012C8001A7023686A78591C21601A706988204648
:1012D80009F02AFD23682A79591C21601A70E988C7
:1012E800204609F021FD2268297AFFF701B8224E2D
:1012F800F378002B00F0FE8723680822591C216030
:101308001A7023680122991821601A7023681B4DEE
:10131800591C2A7921601A702368AA78591C2160FF
:101328001A702988204609F0FFFC698A204609F0CE
:10133800FBFC2368F279591C21601A702268E9784D
:10134800FEF7D6BFEE2D0020442B00205C2B00209A
:10135800542B002034430020B0720020886A0020FB
:10136800FC4000200C430020CF27002080430020B1
:1013780024260020DC400020746A00202C45002030
:10138800D0B9020812F0BAFAFF28064601F00D801B
:101398000EA9002501F82E5D0DF109008DF8095000
:1013A80023F06EF90EA800F82D5D23F05DF90EA864
:1013B80000F82C5D23F04CF90EA820F8245D12F0FB
:1013C8007DFA23685A1C22601E7023689DF8092044
:1013D800591C21601A7023689DF80A20591C216045
:1013E8001A7023689DF80B20591C21601A70236815
:1013F8009DF80C20591C21601A70BDF81410204665
:10140800012509F091FC2B46FEF7F8BEB74D23687D
:101418006A79B74E591C21601A7033682046198CB6
:1014280009F082FC33682046598C09F07DFC6989F3
:10143800204609F079FCA989204609F075FC336833
:101448002046998C09F070FC33682046D98C09F045
:101458006BFCE989204609F067FC298A20460125AA
:1014680009F062FC2B46FEF7C9BEA24D23682A7A12
:10147800591C21601A70A98B204609F055FC298B4C
:10148800204609F051FC698B204609F04DFC236881
:10149800EA7C591C21601A70E98C204609F044FC4A
:1014A800298D204609F040FC2368AA7F591C216039
:1014B8001A70236895F82020591C21601A70A98C8D
:1014C800204609F031FC2368EA7A591C21601A7019
:1014D800E968204609F010FC23682A7C591C216021
:1014E8001A70226895F82110FEF702BF824B226815
:1014F8001978FEF7FDBE814D2046298809F014FCB5
:10150800A988204609F010FC29892046012509F000
:101518000BFC2B46FEF772BE794D7A4F05F150064B
:1015280000212878784A0B4607E00133242B02F182
:101538000C0200F0498512F80C1C8842F5D103EB27
:101548004303226807EB8303511C93F8443021605E
:10155800137023686A78591C21601A702368AA7866
:10156800591C21601A702368EA780435591CAE4268
:1015780021601A70D4D1FEF7A4BE644B03F1700544
:1015880022681978501C2060117022685978501C04
:101598002060117022689978501C206011702268B0
:1015A800D978501C2060117022681979501C20606D
:1015B800117022685979501C20601170226899793D
:1015C8000733501CAB4220601170D9D1FEF779BEA9
:1015D8004F4D2046A98909F0A7FB698920460125B6
:1015E80009F0A2FB2B46FEF709BE4A4B1B78DB0726
:1015F80000F1798401250EF053F80EF0F1F82B462E
:10160800FEF7FCBD5A1CC8F800201A780F2A00F211
:101618006A84991CC8F80010C2EBC2023B4958788A
:101628008854D81CC8F800000A4499785170191DCC
:10163800C8F80010D9789170591DC8F800101979A8
:10164800D170991DC8F8001059791171D91DC8F8C1
:1016580000109979517103F10801C8F80010DB797D
:101668009371012517F08AFC2B46FEF7C7BD40464B
:1016780009F01EFB264EB081404609F019FB0125F2
:1016880070812B46FEF7BABD404609F011FB224E89
:10169800B082404609F00CFBF082404609F008FB96
:1016A800012530832B46FEF7A9BD1A46591CC8F8F8
:1016B80000100E4912F8020B0870C8F800201449EF
:1016C8005A788A70DA1CC8F80020144A9B789370FC
:1016D80001252B46FEF792BD054B114918684A2291
:1016E80001252AF080F82B46FEF788BD746A002091
:1016F8000C430020204A0020942B00209839002019
:10170800982B0020A0B90208E8B90208E82E0020AA
:10171800442B0020D15600202C4500205C2B0020B3
:101728002CD5020819465A1CC8F80020D24A11F8CC
:10173800020B1070C8F8001059785170D91CC8F8FD
:1017480000109B789370404609F0B2FACB4B012504
:10175800D8802B46FEF752BD404609F0A9FAC74E7D
:101768003080404609F0A4FA7080404609F0A0FA9B
:101778000125B0802B46FEF741BDC14F3B78002BB9
:101788003EF49FADBF4E0025404609F091FA18F08F
:1017980065F83B78A6EC010A01359D42F4DBFEF7BB
:1017A80090BD0F2E40F09F835A1CC8F800201D786A
:1017B800072D00F29883B44F40460C2609F078FABA
:1017C80006FB05F6BD19A880404609F071FAE880C5
:1017D800404609F06DFAD8F8003028811A46591C9D
:1017E800C8F8001012F8021BA972C8F800205B782C
:1017F800EB72404609F044FA0125B8512B46FEF732
:10180800FDBC5A1CC8F800201878060600F1598655
:101818009E4B1B78DD073EF554AD032828BF0020FA
:1018280001250DF025FF2B46FEF7E8BC974B1B78EA
:10183800D8073EF546AD01250EF0A4F90DF0D0FF0E
:101848002B46FEF7DBBC914B1B78DA073EF539AD2A
:101858008F4A1378012543F0040313702B46FEF7D3
:10186800CDBC8A4B1B78D9073EF52BAD894B4FF47D
:10187800C87201251A802B46FEF7C0BC092E40F21B
:101888003283854F1A46591C3D68C8F8001012F873
:10189800021B2970C8F800205A78AA70DA1CC8F808
:1018A80000209A78642A03F10401A8BF64226A71AF
:1018B800C8F80010DA78642A03F10501A8BF642289
:1018C800AA71C8F800101A79EA719A1DC8F80020A0
:1018D8005A79642A28BF6422D91D2A72C8F80010D0
:1018E8009A79EA7003F10802C8F80020DB792B71B5
:1018F800404609F0DDF90A2E688140F06986012525
:1019080024F076FB2B46FEF779BC644A1068DA1C93
:1019180001462133951EC8F8005012F8035C0D707B
:10192800551EC8F8005012F8025C4D70C8F8002027
:1019380012F8015C8D700332934201F10301E9D181
:1019480017F068FBFEF7BDBCC6F34706122E00F27F
:10195800CA82B6B10EAB0DF1120903EB46054F462C
:10196800263D404609F0A4F927F8020FBD42F8D1F8
:101978004B4B39F8022F23F8022F4F45F9D1112E7E
:1019880009D8484A7300023B13440021223223F845
:10199800021F9A42FBD1444A01231D461370FEF7E9
:1019A8002DBC1A46591CC8F80010404912F8020B01
:1019B800C870C8F800203E495A780A70DA1CC8F87E
:1019C80000203C4A9B78D37001252B46FEF716BCB5
:1019D800404609F06DF9404609F06AF9404609F0B9
:1019E80067F9D8F800302D4D9A1C2F68C8F80020E8
:1019F8005A7887F82F20DA1CC8F800209A7887F8D8
:101A08003A201A1DC8F80020DA7887F83B200733F7
:101A1800C8F80030404609F04BF9F88740462F686F
:101A280009F046F9112EB88700F29085286887E7F3
:101A38005A1CC8F80020194D1F4F1B78D5F8009084
:101A48007B71404609F034F9A9F820004046D5F8E2
:101A5800009009F02DF9052EA9F8220000F23C8526
:101A68000DF028FE24F0EEFF2868012517F0E6FBAC
:101A78002B46FEF7C3BB00BF3C2B0020C440002010
:101A88002C290020CC3F0020F42D0020D156002026
:101A9800245600201E690020006900200C43002005
:101AA8004A2400204C24002070240020442B0020CD
:101AB800542B00205C2B0020746A0020012509F0BB
:101AC8008FFD2B46FEF79ABB404609F0F1F8054614
:101AD80011F014FFFF283EF4F4ABB5F57A7F80F0DF
:101AE80047850DF13809002309F8243DEE084946D9
:101AF80003A88DF80C30013622F0C2FD9DF80C3099
:101B0800F6B205F00705B34205F1010503D19DF8CA
:101B18001430AB4203D02946304611F0DBFED8F82A
:101B28000030D8F80420D21A012A7EF7CAAB5A1C12
:101B38000EA8C8F8002000221D7800F82C2D22F0ED
:101B480093FD9DF80C30AB420AD0C94B1B683BB1E2
:101B58009A79AA4204D31B681B690BB12846984797
:101B6800D8F800305A1CC8F80020484600221D78D2
:101B78008DF8142022F06CFD9DF81430AB423EF431
:101B8800A0ABBB4B1B68002B3EF49BAB1B685B698F
:101B9800002B3EF496AB28469847FEF792BBB54A11
:101BA8001278012A3EF68DAB19465A1CC8F8002057
:101BB800B14A11F8020B9070C8F8001059781170EA
:101BC800D91CC8F800109B78537001252B46FEF7E6
:101BD80015BB5A1CC8F800201E78112E00F283810C
:101BE8009A1CC8F80020A54D5B7805F816304046C9
:101BF80009F05EF840F6CA039842A8BF184640F2BA
:101C0800EE23984205EB4601B8BF18460125A0F21D
:101C1800EE222B46192092FBF0F24A70FEF7EEBA3C
:101C28001A46591C964DC8F8001012F8021B297064
:101C3800C8F800205B786B70404609F039F8D8F88E
:101C4800003068805A1CC8F800201B782B71404669
:101C580009F02EF8D8F80030E8805A1CC8F800209F
:101C68001B782B7201252B46FEF7C8BA1A46591C59
:101C7800C8F80010834E12F8021BB170C8F8002093
:101C880081495A780A70DA1CC8F800207F4D9A7882
:101C98002A711A1DC8F80020DB78092BA8BF092370
:101CA8004046AB7009F004F8D8F80030D8F80420A2
:101CB8002880D11A012907DD404608F0F9FFD8F835
:101CC8000030D8F8042068829A4240F035840DF03C
:101CD800F1FCD8F80030D8F804209A423EF4F1AA72
:101CE8005A1CC8F800201B78EB7001252B46FEF71C
:101CF80085BA404608F0DCFF654E3060404608F083
:101D0800D7FF7060404608F0D3FF0125B0602B462E
:101D1800FEF774BA5A1CC8F800201A780E2A00F286
:101D2800E280991CC8F800105D78032D00F2DB8072
:101D38005848062101FB02F14218DE1C5571C8F80B
:101D480000609D784554191DC8F80010D978517065
:101D5800591DC8F8001019799170991DC8F800101C
:101D68005979D170D91DC8F800109B7913710125D4
:101D78002B46FEF743BA5A1CC8F80020464A1B787F
:101D88005375FEF79EBA5A1CC8F80020424D1B78BE
:101D98002B72404608F08CFFA883404608F088FF65
:101DA8002883404608F084FFD8F8003068835A1C1E
:101DB800C8F800201B78EB74082E7EF682AA4046ED
:101DC80008F076FFE884404608F072FF0C2E28855C
:101DD8007EF677AAD8F800301A46591CC8F80010C1
:101DE80012F8021BA977C8F800205B7885F8203024
:101DF800404608F05DFF102EA8847EF662AAD8F847
:101E080000305A1CC8F800201B78EB72404608F0D6
:101E180037FFD8F80030E8605A1CC8F800201A7854
:101E28002A74162E7EF64DAA9A1CC8F800205B78F4
:101E380085F8213001252B46FEF7E0B95A1CC8F871
:101E48000020164A1B78137001252B46FEF7D6B9D9
:101E5800591C1A46C8F80010114912F8020B88706C
:101E6800C8F800205B784B7001252B46FEF7C6B9F1
:101E7800D05F0020CE270020CF2700202426002076
:101E8800DC400020746A0020382B00202C450020FC
:101E98009839002044300020204A0020942B00204C
:101EA800682B00200722B6FBF2F2C2EBC201761AB9
:101EB80019D1D2B2571EFFB2002A3EF402AADFF8A7
:101EC80030A301375A1CC8F8002093F90010C84BFA
:101ED800002593F902208A4200F093820135052DEE
:101EE80003F10803F5D14FF0FF352B46FEF786B90D
:101EF800C04A03F108010133C8F8003013F8010C97
:101F080002F8010F9942F6D1FEF7DBB95A1CC8F85E
:101F1800002018781328E6D89A1CC8F800205D78A5
:101F2800B54A002104E00131242902F10C02DAD07B
:101F3800167AAE42F7D1B14DB14A0C2606FB0151D3
:101F4800DD1C91F83C1002F82010C8F8005002EB94
:101F5800800299785170191DC8F80010D8789070CF
:101F6800581DC8F80000A7491B790868D37023F0EA
:101F7800CDFFFEF7A6B9A44B102E4FF0000228BFE4
:101F880010261A605A609A60DA601A74002E3EF4BD
:101F980098A9D8F8002016440132C8F8002012F891
:101FA800011C03F8011B9642F6D1FEF78AB9974E39
:101FB80000233360404608F063FE3368012503437D
:101FC80033602B46FEF71AB900231B7AFFDE23681D
:101FD8005A1C226019702988204608F0A5FE23683B
:101FE800EA78591C21601A7023682A79591C2160E3
:101FF8001A702368AA79591C21601A7023686A79B3
:10200800591C21601A70FEF768BE1A46591CC8F898
:1020180000107F4D12F8021B6970C8F800205A782A
:102028002A70DA1CC8F800209B78AB70404608F08C
:102038003FFED8F80030E880591C1A46C8F800104E
:1020480012F8021B2971C8F800205B786B714FF0F9
:10205800FF352B46FEF7D2B85A1CC8F800201A786C
:102068000A2A7FF440AF9A1CC8F80020694A5978B8
:102078001170D91CC8F8001099785170191DC8F84A
:102088000010DB7893702EE75A1CC8F800201B78E4
:102098000A2B00F09281502B7FF425AF404608F0C0
:1020A80007FE5D4E3080404608F002FE4FF0FF35D7
:1020B80070802B46FEF7A2B8DFF87CB14FF000081D
:1020C8004FF0080A08F10108B8F1240F1BD0C8F135
:1020D80020020AFA02F22BFA08F6A8F120031643A6
:1020E8002AFA03F31E4306F0010200231343E9D042
:1020F8005FFA88F023F004FF0028E3D04146484601
:1021080009F046F8DEE7454B1B78DF0700F1A381AD
:102118000026434FB04602E00136242E0ED0314649
:10212800384609F045F80028F6D03146484609F007
:102138003FF8002856D108F10108EDE7394B3A4E2F
:10214800B3F85010204608F0EFFD384B19882046A8
:1021580089B208F0E9FD364B1A68530103F02001F3
:10216800C2F340030B43C2F3800143EA4103C2F3C5
:10217800C00143EA8103C2F3401143EAC10102F0FE
:1021880010021143204608F0CFFD03A9042220467F
:1021980008F09AFD23683178264A581C2060197087
:1021A80011886429A8BF6421204608F0BDFD962D3A
:1021B80000F056810021204608F0B6FD2168B8F1EC
:1021C800190348BFA8F11203A3F3C4034A1C2260F1
:1021D80020460B701A4604A9012508F075FD2B4608
:1021E800FEF70CB8414603A808F0D2FFA3E700BFEA
:1021F800486A00201F4A0020DCB90208A0B902087A
:10220800982B00200C430020F84200206C2B002063
:10221800C84400204B260020A8310020D1560020B9
:10222800801B0020280E0020F4420020C8730020E4
:10223800684B00203430002090E33FF498E80C000D
:1022480093427EF441A8D64BFF221A724FF0000841
:10225800D44D21F0C7F941463022D34885F8008093
:1022680029F0E6FA8DF814809DF814300B2B00F253
:102278002681CE4FCC4E42469DF8143003EB4303E3
:1022880007EBC3035B7CE3B19DF8143003EB430316
:1022980007EBC3035B69A3B19DF8143003EB430359
:1022A80007EBC3032021586946F822000CF0D6FC3E
:1022B8002B7856F823000CF093FE2A780132D2B21C
:1022C8002A709DF814300133DBB28DF814309DF874
:1022D80014300B2BD0D92368591C21601A70B9F11E
:1022E800000F3DF4EEAFB24BC9F8003001252B4684
:1022F800FDF784BF2368B178AE4A581C2060197076
:1023080023681278591C21601A70FEF7FFBFD9F8AC
:10231800003013F48053B4EEE88A00F0AC80F1EE9C
:1023280010FAC0F2C980B4EEC98AF1EE10FA0DD8DD
:10233800DFEDA17A9FEDA17A77EEC87AB4EEC78A6D
:10234800F1EE10FAB0EE678A00F2B680F7EE007A86
:1023580078EE677AB6EE007AF0EE696AE7EE876A99
:1023680040F2E932FDEEE67A17EE901AB1F5FA6F0F
:10237800A8BF4FF4FA619142B8BF114689B2002B49
:102388003EF44FAEB5EE408AF1EE10FA40F2DC535F
:1023980008BF1946FEF745BE404608F089FC4FF0D5
:1023A800000807460546FEF727BC22680125531991
:1023B80023602B461070FDF721BF404608F078FCDB
:1023C8007F4E6FE63946204608F0AEFC23685A1C5B
:1023D800226083F80080D9F80C50D4F80080F219F4
:1023E800AA4200F29C8009F099F83A4641463046E4
:1023F80009F014F923680125034423602B46FDF7EF
:10240800FDBE0AEBC509404689F8021008F050FCE9
:10241800D8F800202AF835001346511CC8F80010D7
:1024280013F8021B89F80310C8F80030537889F8AC
:102438000430D31CC8F80030937889F80630131D8F
:10244800C8F800300136D27889F80520B7427FF401
:1024580039ADFDF736BF059B43F00103059357E6F9
:1024680023680322591C21601A7023687278591C4A
:1024780021601A70A2E6F1EE10FABFF667AF4FF4CA
:102488007A71FEF7CEBD4F490978914205D8022BE3
:102498007DF42CAFFF2A7DF429AF236801255A1952
:1024A80022601D70B9F1000F3DF40BAF464BC9F81F
:1024B80000302B46FDF7A2BE4FF47A7162E7424620
:1024C80009E700F07F00032828BF0020012521F03C
:1024D800C9F82B46FDF792BE404608F0E9FB788123
:1024E800404608F0E5FBB8814046D5F8009008F072
:1024F800DFFBA9F824004046D5F8009008F0D8FB87
:102508000D2EA9F826007FF6ABAA404608F0D0FBAE
:10251800F881404608F0CCFB3882FFF7A1BAAD1B22
:1025280008F0FCFF2A464146304609F077F8236850
:1025380003442360FDF7C5BE5A1CC8F800201B7869
:10254800003318BF0123F371FFF7C1BBD8F800307F
:102558002968581C1A46C8F8000012F8020B81F8BE
:102568003100C8F800205B7881F83230FFF75EBA96
:102578000DF11409484611F0A1F9BDF81430AB4229
:102588003FF4CDAA114B1B68002B3FF4C8AA1B6867
:102598009B69002B3FF4C3AA28469847FFF7BFBAA8
:1025A800801B00208B2C002048250020F04F0020A5
:1025B80095540108382B002000C0884400C082448C
:1025C800342B00202C2900207DF30008D05F002048
:1025D800D8F800303A68591CC8F8001019785172B8
:1025E8000B2E3FF48CA9991CC8F800105B78537027
:1025F800FFF785B92DE9F04FDFF804912DED0C8B2D
:1026080099F800309BB0012B099002F02084DFF884
:10261800F4A09AF80021002A41F03C83072B354C9E
:1026280002F06783002305936368324898470028BF
:102638006ED0B4F8A860002284F84920002E40F03B
:102648008A82B4F92600226BB4F92450E16AB4F9FD
:102658002830DFF8B4B0821A606BE263691A1B1A7B
:10266800A163254894F84A1023641EF0F3FFDBF8B1
:10267800003013F0005302F06383D4ED0F5AD4ED09
:102688000E7A1E4A9AED706ADAED716A9AED727ADC
:10269800DAF8CC311268B8EEE58AD4ED105AF8EEC3
:1026A800E77AF8EEE58A013377EE867A38EE268AFD
:1026B80078EE878A9342CAED707A8AED718ACAEDFC
:1026C800728ACAF8CC3101F0F58699F80060142EA8
:1026D80003F010840023DAF8D4510693062D02F291
:1026E8004084DFE815F0431B121BDE13121A7B1A15
:1026F800A1191B19886A0020C06A00206C4B0020B1
:10270800902B00208C1B0020504A0020DDF818A0D8
:1027180099F80080B8F1070F00F0D2829AF8DC31FE
:10272800002B40F0D882D04B5B79002B40F00E8212
:10273800012399F800208AF8DC31072A02F0BB85CA
:1027480000230C93C94B9AED789A93ED007AC84A06
:10275800C84B12680692F7EE007A37EEC9CAC64A25
:1027680007922CEE07CAC54A9AED418ADFF888839A
:102778009FEDC3AADFEDC38ADFEDC3AADFEDC3CAAD
:10278800DFEDC39A9FEDC3BAC34FDFF870B3C34EF2
:102798000B93B4EEE7CA0024F1EE10FA089288BF52
:1027A800B0EE67CA05932546BD4B2344D3ED007AA6
:1027B800BC4BF5EE407A2344F1EE10FAD3ED00BAA3
:1027C80017D0B94B234493ED007A7BEEC76AB0EE7D
:1027D800E66AF4EEC67AF1EE10FA08D5F5EEC06AAC
:1027E800F1EE10FACCBF77EE87BA77EE67BAC3ED91
:1027F80000BA079B1888810700F07582022D05F042
:1028080064810699A94A91F8323007EE103A91F896
:1028180031302244D2ED006A5A42B8EEC77A07EE48
:10282800902A27EE267AF8EEE77AB4EEE77AF1EE08
:1028380010FA0AD407EE903AF8EE677AF4EEC77AFF
:10284800F1EE10FA88BFF0EE477ADFF8B4E2984A62
:102858000A920EEB450332F91510B3F90A30CA1A79
:1028680007EE102AB8EEC77AC207E7EE687A40F199
:10287800E9829048D0ED00BA67EEABBA9AF8F00159
:10288800E0B18C48DAF8F421D0ED00BA8A485B1A36
:1028980007EE903A099B01686BEEA8BAF8EEE77A62
:1028A800981A88426BEEA7BA00F36382F7EE007AB3
:1028B800B4EEE79AF1EE10FA00F127827F4B234439
:1028C800D3ED007A059BD3ED01DA68EE277A3BEE6B
:1028D800EDDA67EE8D7ACBED007A089BD8ED006AC9
:1028E80093ED007A764BD6ED007A26EE877A23446C
:1028F80067EE0C6A93ED007A26EE877AF0EE676A47
:10290800E7EE0D6AB0EE667A9AED786AF7EE006A3D
:10291800B4EEE66AF1EE10FAACBF0123002343B12E
:10292800F0EEE77AF0EEC76AF4EEE76AF1EE10FA35
:1029380001D586ED007A022D05F02A80614A624BA6
:1029480052F825001B68B0EE6D0A98475F4A604B45
:1029580052F825001B689847069B93F83A30632B7A
:1029680004D8079B1B88002B01F06781F0EE6C7A76
:10297800584B98ED007A37EEC00A2344D3ED007A1D
:1029880083ED000A069B30EE670A93F84830C0EEE4
:10299800077ADBB1B7EE007AB4EEC79AF1EE10FA17
:1029A80014DB4D4B93ED007AF0EEE76AF4EEC76A5C
:1029B800F1EE10FA0ADD494B93ED007AB0EECDDA6C
:1029C800B4EEC7DAF1EE10FA01F36483444B9AF8D7
:1029D8000022234493ED007A28EE077A67EE277ADF
:1029E800C7ED007A2AB9CBED00CAC6ED00CAC7ED1B
:1029F80000CA059B043404330C2C05F1010507F1CA
:102A080004070BF1040B06F1040605937FF4CCAE22
:102A180099F80030072B02F03182012B02F03B8439
:102A2800002305932F4B124A1B68126892F82F1047
:102A380013F48052069200F083822B482B4E0278C2
:102A48002B4C2C4DE48895ED037A12F0010F328B54
:102A580008BFAAF80822151B07EE905AF8EEE77A85
:102A6800B4EEE77A4EE000BF746A0020C83A00204E
:102A78000C430020AC720020EE2D00200000002046
:102A880000009642CDCCCC3DAE47813F000000000F
:102A98000000C842000034432029002014290020E7
:102AA800BC3A0020BC1C0020701D0020241D002002
:102AB80078430020A03A0020CC3A0020743A002045
:102AC800803A0020E43A0020E03A0020483B002009
:102AD800443B0020841D0020DC3A0020D83A002026
:102AE8008C3A0020504A0020D1560020204A00206D
:102AF800C4400020A0420020B83A00200829002045
:102B0800442B0020F1EE10FA42F2DB82171906EE90
:102B1800907AF8EEE66AB4EEE67AF1EE10FA81F20F
:102B28009C84BAF80822954283F2C787B34AB44C0A
:102B3800D2ED004AD4ED003AB24ACAED833ACAED62
:102B4800844AD2ED006ADFEDB07A12E2AF4B1B780F
:102B5800013BDBB2EDE5AE4BAE490B9391F801B00A
:102B68001B68AD4F99F80080B7F906004FF47A71E9
:102B7800B1FBF3F3C3EB431503EB8503DD00ADB203
:102B8800AE4203F03B82E16FB4F924E0236E4A1CA5
:102B980007EE90EA7344012AE2672366F8EEE77AC3
:102BA80003F03682D4ED1B5AD4ED1D6A07EE102AC5
:102BB80037EEE56AB8EEC75A012E86EE057A37EE8B
:102BC800257A77EEC77A84ED1C7AE7EE866A84ED7B
:102BD8001B7AF0EE667AC4ED1E6AC4ED1D6A03F036
:102BE800FF87D4F89010B4F926E0636E4A1C07EE0C
:102BF80090EA7344012AC4F890206366F8EEE77AF5
:102C080003F01E82D4ED205AD4ED226A07EE102A72
:102C180037EEE56AB8EEC75A012E86EE057A37EE2A
:102C2800257A77EEC77A84ED217AE6EE276A84ED75
:102C3800207AF0EE667AC4ED236AC4ED226A03F0C6
:102C4800A687D4F8A410B4F928E0A36E4A1C07EEAE
:102C580090EA7344012AC4F8A420A366F8EEE77A40
:102C680003F00782D4ED255AD4ED276A07EE102A1F
:102C780037EEE56AB8EEC75A012E86EE057A37EECA
:102C8800257A77EEC77A84ED267AE6EE276A84ED10
:102C9800257AF0EE667AC4ED286AC4ED276A03F057
:102CA8006987F880013E99F80080A4F8A8600B991C
:102CB8000023B8F1070F4B608B60CB607FF42EAD1B
:102CC8000BF018F9059B544FC01A9AF8DC3138807C
:102CD800002B3FF428AD013B8AF8DC311BB0BDEC7A
:102CE8000C8BBDE8F08F9AF8F031002B45D0022DFF
:102CF80004F0DA86DFF848E1484A0A920EEB450309
:102D080032F91510B3F90A30BBE50A9B4449B3F907
:102D18000000BEF90A300968C21A82EAE273A3EB1E
:102D2800E2738B42BFF6CAAD0A9BBEF90C20B3F919
:102D380002309A1A82EAE273A3EBE27399427FF7B0
:102D4800BDAD0B99374BD1ED017A93ED007AF0EEDA
:102D5800E77AF4EEC77AF1EE10FA7FF5AFADD1ED70
:102D6800027AF0EEE77AB4EEE77AF1EE10FA7FF73E
:102D7800A5AD00238AF8F031A0E52B4B234493ED51
:102D8800000A059BD3ED01DA28EE000A3BEEEDDAE6
:102D9800022D20EE0D0A8BED000A7FF49EAD234A2A
:102DA800234B10681B689847089BD8ED006A93ED81
:102DB800007A204BD6ED007A1A781F4B83ED020A71
:102DC8001E4B26EE877A234427EE0C7A93ED006A91
:102DD80027EE067AF0EE676AE7EE0D6A012AB0EE92
:102DE800667A02D0192A7FF48FADB4EECADAF1EE12
:102DF80010FACCBF0123002391E500BFBC4000209E
:102E0800282B0020D440002000000000382B002090
:102E1800AC720020746A0020D2420020784300205F
:102E2800D03A0020D43A0020743A0020A83F00206D
:102E3800BC3F0020EC2D002008290020803A00200B
:102E4800442B0020DAED696A9AED6A7A0A9AB4EEA0
:102E5800E67AF1EE10FAB2F90200B2F900C00D906C
:102E68004BBFB7EE007AF7EE006A77EE665A76EE59
:102E7800C75A8CEAEC720028A2EBEC72B8BF404249
:102E8800824201F3C7800D9A2948002AD8BF5242CE
:102E980007EE102A0078B8EEC77A27EE287A0028BD
:102EA80001F0CA80234890ED005AB5EEC05AF1EE01
:102EB80010FA41F3DF872048D0ED004AF5EEC04A0A
:102EC800F1EE10FA41F3D68734EEC77AB7EE006A0E
:102ED800C7EE246A75EEC65AF4EEC66A65EEA95ABC
:102EE800F1EE10FA85EE857A88BFF0EE466AF5EEC7
:102EF800C06AF1EE10FA37EE067AB8BFF0EE6C6AE7
:102F080066EE876AF4EEC66AF1EE10FA88BFF0EE54
:102F1800466AF5EEC06AF1EE10FAB8BFF0EE6C6AD8
:102F2800064890ED007A67EE877AE7EEA6BAA5E440
:102F3800AC3A0020A83A0020B03A0020A43A002079
:102F4800E14EE24A708B92ED037AE14A07EE900A6D
:102F5800E048D2ED003AE04AD0ED004AD2ED006AEE
:102F6800DE48CAED844AF8EEE77ACAED833A77EE8E
:102F7800677AC7EEA65ADA4CDA4A94ED005ADA4C68
:102F88009FEDDA7A94ED003AD94C9FEDDA6A94ED28
:102F9800004AD2ED006AF7EE007AF4EEE75A35EE11
:102FA800035AF1EE10FA88BFF0EE675A35EE045A6C
:102FB800F4EEC75AF1EE10FA25EE065AB8BFF0EE55
:102FC800475AB1EE667A33EEE43AB4EEC75AF1EEF8
:102FD80010FACAED855A8AED873A00F17184B4EE89
:102FE800E65AF1EE10FA88BFB0EE665ABC4A9FED79
:102FF800C16AD2ED017ABC4AD2ED012ABC4A77EE09
:10300800A27A92ED014A77EE847A67EE867AB4EE78
:10301800E77AF1EE10FA08DCF4EEE76AF1EE10FA5E
:103028008CBFB0EE677AB0EE667AAD4A9FEDB16AB2
:10303800D2ED027AAC4A92ED024AAF4A77EE847A30
:10304800D2ED006A67EE867AB1EE664AF4EEC47A8B
:10305800F1EE10FA08D4F4EEE67AF1EE10FA8CBF2D
:10306800B0EE664AB0EE674A002941F0AE82B7EE8C
:10307800002AA24AA24D52789AF82012002AFFEE9E
:10308800002AB7EE006A2A7814BFF0EE467AF0EE0E
:10309800627A002914BFF0EE626AF0EE466A002AEE
:1030A80003F05080B4EEC62AF1EE10FA24EE274A57
:1030B800944941F3D18291ED026A91ED011AD1ED63
:1030C800037ADFED8A1A27EE066A62EE262AA5EE53
:1030D800016AA7EE846A26EE226AB4EEE16AF1EE8E
:1030E80010FAB4BFF0EE617AF0EE467A8DED0E6A12
:1030F80088BFB0EE616A012A00F0BE81D1ED066A90
:10310800D1ED051A91ED072A67EE266AE5EE216AE8
:10311800E2EE046A66EEA26AF4EEC66AF1EE10FA0E
:10312800F4EEE76A8CBFB0EE462AB0EE662AF1EEFE
:1031380010FA98BFB0EE426AA8BFF0EE667A022A8B
:10314800CDED0F6A00F09881D1ED0A6AD1ED091A28
:1031580091ED0B2A67EE266AE5EE216AE2EE046A33
:1031680066EEA26AF4EEC66AF1EE10FAF4EEE76AC9
:103178008CBFB0EE462AB0EE662AF1EE10FA98BF80
:10318800B0EE426AA8BFF0EE667A032ACDED106A67
:1031980000F07281D1ED0E6AD1ED0D1A91ED0F2A72
:1031A80067EE266AE1EE856AE2EE046A66EEA26AD6
:1031B800F4EEC66AF1EE10FAF4EEE76A8CBFB0EEF0
:1031C800462AB0EE662AF1EE10FA98BFB0EE426ACF
:1031D800A8BFF0EE667A042ACDED116A00F04C81A2
:1031E800D1ED126AD1ED111A91ED132A67EE266A14
:1031F800E1EE856AE2EE046A66EEA26AF4EEC66A59
:10320800F1EE10FAF4EEE76A8CBFB0EE462AB0EEA3
:10321800662AF1EE10FA98BFB0EE426AA8BFF0EE47
:10322800667A052ACDED126A00F02681D1ED166A7C
:10323800D1ED151A91ED172A67EE266AE1EE856A37
:10324800E2EE046A66EEA26AF4EEC66AF1EE10FADD
:10325800F4EEE76A8CBFB0EE462AB0EE662AF1EECD
:1032680010FA98BFB0EE426AA8BFF0EE667A062A56
:10327800CDED136A00F00081D1ED1A6AD1ED191A6B
:1032880091ED1B2A67EE266AE1EE856AE2EE046A92
:1032980066EEA26AF4EEC66AF1EE10FAF4EEE76A98
:1032A8008CBFB0EE462AB0EE662AF1EE10FA98BF4F
:1032B800B0EE426AA8BFF0EE667A072ACDED146A2E
:1032C80000F0DA8020E000BF204A0020A042002061
:1032D800282B0020A4290020CC400020D156002013
:1032E80008290020C03F0020142900200000000009
:1032F800202900206F12833AC43F0020942B00201D
:103308002C290020FC3F0020D1ED1E6AD1ED1D1AAA
:1033180091ED1F2A67EE266AE1EE856AE2EE046AFD
:1033280066EEA26AF4EEC66AF1EE10FAF4EEE76A07
:103338008CBFB0EE462AB0EE662AF1EE10FA98BFBE
:10334800B0EE426AA8BFF0EE667A082ACDED156A9B
:1033580000F09280D1ED226AD1ED211A91ED232A55
:1033680067EE266AE1EE856AE2EE046A66EEA26A14
:10337800F4EEC66AF1EE10FAF4EEE76A8CBFB0EE2E
:10338800462AB0EE662AF1EE10FA98BFB0EE426A0D
:10339800A8BFF0EE667A092ACDED166A6CD0D1ED99
:1033A800266AD1ED251A91ED272A67EE266AE1EE05
:1033B800856AE2EE046A66EEA26AF4EEC66AF1EE87
:1033C80010FAF4EEE76A8CBFB0EE462AB0EE662A31
:1033D800F1EE10FA98BFB0EE426AA8BFF0EE667A36
:1033E8000A2ACDED176A47D0D1ED2A6AD1ED291AFC
:1033F80091ED2B2A67EE266AE1EE856AE2EE046A11
:1034080066EEA26AF4EEC66AF1EE10FAF4EEE76A26
:103418008CBFB0EE462AB0EE662AF1EE10FA98BFDD
:10342800B0EE426AA8BFF0EE667A0B2ACDED186AB4
:1034380022D0D1ED2E1A91ED2D2AD1ED2F6A27EE4B
:10344800217AA2EE057AA6EE847A27EE227AB4EEE5
:10345800C76AF1EE10FAF4EEC77A8CBFF0EE476A4D
:10346800F0EE466AF1EE10FA8DED197A58BFB0EE1B
:10347800666AB8BFF0EE477A77EEC67AF7EE006A6A
:10348800F4EEE67AF1EE10FACAED787A43F3FE82AA
:1034980086EEA77A012ADDED0E7A67EE877ACDED02
:1034A8000E7A55D0DDED0F7A67EE877A022ACDEDD8
:1034B8000F7A4DD0DDED107A67EE877A032ACDEDCD
:1034C800107A45D0DDED117A67EE877A042ACDEDC2
:1034D800117A3DD0DDED127A67EE877A052ACDEDB7
:1034E800127A35D0DDED137A67EE877A062ACDEDAC
:1034F800137A2DD0DDED147A67EE877A072ACDEDA1
:10350800147A25D0DDED157A67EE877A082ACDED95
:10351800157A1DD0DDED167A67EE877A092ACDED8A
:10352800167A15D0DDED177A67EE877A0A2ACDED7F
:10353800177A0DD0DDED187A67EE877A0B2ACDED74
:10354800187A05D0DDED197A27EE877A8DED197A8C
:10355800DD49096811F0805100F03685F6EE005A11
:10356800CAED855A0078002A02F0D685DFF8708304
:10357800D64CDFF870B3DFF870E39AF818C2768B90
:103588000796FDEEE37AD8ED006A9BF803B0B4F92C
:1035980006809EF800E003F0100600F0010003F436
:1035A800800317EE904ABCF1000F40F09F81002E77
:1035B80000F0E885002843F09A80BBF1000F43F043
:1035C800A382C349DDED0E7A91ED007AC14BE7EE97
:1035D800257ABDEEE47A17EE100AB0EE647AA3EE0F
:1035E800277AFDEEC77A17EE907A17EE906AA7420F
:1035F800A8BF2646B842C8BF064607EE906AF8EE4E
:10360800E77A012AC3ED007A00F04D8191ED047A42
:10361800DDED0F7AE7EE257AB0EE647AA3EE277A2D
:10362800FDEEC77A17EE907A17EE906AA742A8BF08
:1036380026468742B8BF064607EE906AF8EEE77A54
:10364800022AC3ED017A00F02E8191ED087ADDEDB2
:10365800107AE7EE257AB0EE647AA3EE277AFDEECB
:10366800C77A17EE907A17EE906AA742A8BF264647
:103678008742B8BF064607EE906AF8EEE77A032A53
:10368800C3ED027A00F00F8191ED0C7ADDED117A2D
:10369800E7EE257AB0EE647AA3EE277AFDEEC77AD4
:1036A80017EE907A17EE906AA742A8BF264687427F
:1036B800B8BF064607EE906AF8EEE77A042AC3ED2B
:1036C800037A00F0F08091ED107ADDED127AE7EEE2
:1036D800257AB0EE647AA3EE277AFDEEC77A17EE64
:1036E800907A17EE906AA742A8BF26468742B8BFCD
:1036F800064607EE906AF8EEE77A052AC3ED047AE3
:1037080000F0D18091ED147ADDED137AE7EE257A99
:10371800B0EE647AA3EE277AFDEEC77A17EE907AB8
:1037280017EE906AA742A8BF26468742B8BF06464A
:1037380007EE906AF8EEE77A062AC3ED057A00F0FC
:10374800B28091ED187ADDED147AE7EE257AB0EEC5
:10375800647AA3EE277AFDEEC77A17EE907A17EE11
:10376800906AA742A8BF26468742B8BF064607EE1A
:10377800906AF8EEE77A072AC3ED067A00F093809C
:1037880091ED1C7ADDED157AE7EE257AB0EE647AD4
:10379800A3EE277AFDEEC77A17EE907A17EE906AB5
:1037A800A742A8BF26468742B8BF064607EE906ADA
:1037B800F8EEE77A082AC3ED077A74D091ED207AFB
:1037C800DDED167AE7EE257AB0EE647AA3EE277A75
:1037D800FDEEC77A17EE907A17EE906AA742A8BF57
:1037E80026468742B8BF064607EE906AF8EEE77AA3
:1037F800092AC3ED087A56D091ED247ADDED177ABF
:10380800E7EE257AB0EE647AA3EE277AFDEEC77A62
:1038180017EE907A17EE906AA742A8BF264687420D
:10382800B8BF064607EE906AF8EEE77A0A2AC3EDB3
:10383800097A38D091ED287ADDED187AE7EE257A05
:10384800B0EE647AA3EE277AFDEEC77A17EE907A87
:1038580017EE906AA742A8BF26468742B8BF064619
:1038680007EE906AF8EEE77A0B2AC3ED0A7A1AD0C7
:1038780091ED2C7ADDED197AE7EE257AE3EE274A09
:10388800FDEEE47A17EE901A8C42A8BF0C468842E7
:10389800D8BF204607EE900AF8EEE77AC3ED0B7A18
:1038A800002A00F0A48192000B490A4827F09BFFE8
:1038B8000A4B1B68002B00F09F8112F027F99BE14F
:1038C800B0EE475AFFF792BB1C2B00201263002072
:1038D800FC3F002064290020CC3F0020582F002006
:1038E800C83F0020A044002054450020002E40F08E
:1038F800DE83DF49DDED0E7A91ED007ADD4BE7EEF0
:10390800257AB1EE433AB0EE637AA3EE277AF0EE69
:10391800477ABEF1000F41F00985BBF1000F43F073
:103928006A83FDEEE77ABDEEE47A17EE90EA17EEC9
:10393800907AA64517EE106AA8BF27467645C8BFF5
:10394800374607EE907AF8EEE77A012AC3ED007A57
:1039580000F04A8191ED047ADDED0F7AE7EE257AE1
:10396800B0EE637AA3EE277AFDEEC77A17EE90EAF7
:1039780017EE907AA645A8BF2746B645B8BF374682
:1039880007EE907AF8EEE77A022AC3ED017A00F0A2
:103998002B8191ED087ADDED107AE7EE257AB0EE0D
:1039A800637AA3EE277AFDEEC77A17EE90EA17EE50
:1039B800907AA645A8BF2746B645B8BF374607EE52
:1039C800907AF8EEE77A032AC3ED027A00F00C81C8
:1039D80091ED0C7ADDED117AE7EE257AB0EE637A97
:1039E800A3EE277AFDEEC77A17EE90EA17EE907AE3
:1039F800A645A8BF2746B645B8BF374607EE907A12
:103A0800F8EEE77A042AC3ED037A00F0ED8091ED31
:103A1800107ADDED127AE7EE257AB0EE637AA3EE3E
:103A2800277AFDEEC77A17EE90EA17EE907AA64548
:103A3800A8BF2746B645B8BF374607EE907AF8EED6
:103A4800E77A052AC3ED047A00F0CE8091ED147A66
:103A5800DDED137AE7EE257AB0EE637AA3EE277AE6
:103A6800FDEEC77A17EE90EA17EE907AA645A8BF42
:103A78002746B645B8BF374607EE907AF8EEE77A9C
:103A8800062AC3ED057A00F0AF8091ED187ADDEDD6
:103A9800147AE7EE257AB0EE637AA3EE277AFDEE84
:103AA800C77A17EE90EA17EE907AA645A8BF274680
:103AB800B645B8BF374607EE907AF8EEE77A072A98
:103AC800C3ED067A00F0908091ED1C7ADDED157A51
:103AD800E7EE257AB0EE637AA3EE277AFDEEC77A91
:103AE80017EE90EA17EE907AA645A8BF2746B64586
:103AF800B8BF374607EE907AF8EEE77A082AC3EDA2
:103B0800077A71D091ED207ADDED167AE7EE257A05
:103B1800B0EE637AA3EE277AFDEEC77A17EE90EA45
:103B280017EE907AA645A8BF2746B645B8BF3746D0
:103B380007EE907AF8EEE77A092AC3ED087A53D0AF
:103B480091ED247ADDED177AE7EE257AB0EE637A07
:103B5800A3EE277AFDEEC77A17EE90EA17EE907A71
:103B6800A645A8BF2746B645B8BF374607EE907AA0
:103B7800F8EEE77A0A2AC3ED097A35D091ED287A6A
:103B8800DDED187AE7EE257AB0EE637AA3EE277AB0
:103B9800FDEEC77A17EE90EA17EE907AA645A8BF11
:103BA8002746B645B8BF374607EE907AF8EEE77A6B
:103BB8000B2AC3ED0A7A17D091ED2C7ADDED197A2C
:103BC800E7EE257AE3EE273AFDEEE37A17EE901A50
:103BD8008C42A8BF0C468E42D8BF264607EE906A94
:103BE800F8EEE77AC3ED0B7A00283FF459AE224B82
:103BF8001B68002B7FF461AE204B1B7883B12878BB
:103C080058B11C4E1E4F0024E0B23B68B6EC010AC6
:103C18009847287801348442F6DB1A4B1B6898478A
:103C280099F80030072B01F0B08101238AF80031A0
:103C38001BB0BDEC0C8BBDE8F08F134B134A23442B
:103C4800D3ED006A92ED007A114B26EE877AF7EEF3
:103C5800006AB4EEE67AD3ED007AF1EE10FA88BF86
:103C6800B0EE667A27EE277A67EE2B7AFEF780BEEB
:103C7800FC3F002064290020582F0020BC49002068
:103C88004845002050450020301D00209C3A002067
:103C9800983A0020072B02F0F48600230893DFF8F7
:103CA8006CB3CC4CDBF8003007935A0501F1208245
:103CB800C94BCA49D3F80080B1F90630B8F80A20D0
:103CC80005939342C0F2EE81B3F5FA6F81F2FA825E
:103CD80098F808009B1A03FB00F3C2F5FA6293FBFD
:103CE800F2F3C3F1640307EE903AF8EEE77A9FED3A
:103CF800BC7A67EE877ACAED417ABA4BBA4E93F925
:103D08000420B848378BB1F9003090F800E090F8FB
:103D180001C0002AA3EB070014BF01224FF0FF32B5
:103D2800002841F30180B0F5FA7FC1F202804FF418
:103D3800FA70A0EB0E0007EE900AF8EEE77AAB4DAA
:103D48009F42C5ED007A03DDF1EE677AC5ED007A92
:103D5800B1F90200C31B002B41F36D80B3F5FA7F64
:103D6800C1F26E804FF4FA73A3EB0E0307EE903A9C
:103D7800F8EEE77A8742C5ED017A03DDF1EE677A5E
:103D8800C5ED017AB1F90430D91B0029D8BFF91A59
:103D9800B1F5FA7F80F222866145D8BF4FF0000C5A
:103DA80000F31E8602FB0CF207EE902AF8EEE77A83
:103DB800BB42079BC5ED027ABCBFF1EE677AC5ED41
:103DC800027A13F48053069300F09887059BB3F5A5
:103DD800FA6FA8BF4FF4FA63B3F57A7F1A46B8BFF3
:103DE8004FF47A72A2F57A728149DFF824E281FBF6
:103DF8000230D317C3EB6013581C6FF0630C3EF905
:103E080010003EF913E00CFB0323A0EB0E0003FBAC
:103E180000F381FB0321DB17C3EB61139E440FFA08
:103E28008EFE07EE90EA069BB8EEE78A85ED038AD8
:103E3800002B41F003826F4B1B8813F040020A925B
:103E480041F0AB806C4A126812F0140F03D013F4DF
:103E5800027F41F03F82694A12789AB1728B0599C4
:103E68008A420FDB664A1278012A02F02D81192A4C
:103E780002F02A810E2A05D0082A03D00022AA605F
:103E8800CAF838219AF83E7117B19B0742F09F8310
:103E98009AF84431F27F002B41F03781B17F002935
:103EA80000F0A285022902F03081032901F01E8565
:103EB800544949880232D2B2002B02F01A810029F3
:103EC80002F0178150480068B1FBF0F109B2059182
:103ED800AAF87411AAB3DDED057AF8EEE77AF7EEE1
:103EE800006A86EEA77A012AD5ED007ADAED626AD1
:103EF80077EEE67A67EE877ACAED5E7A21D0D5ED5D
:103F0800017ADAED636A77EEE67A022A67EE877A53
:103F1800CAED5F7A15D0D5ED027ADAED646A77EEEC
:103F2800E67A032A67EE877ACAED607A09D0D5ED7A
:103F3800037ADAED656A77EEE67A67EE877ACAED94
:103F4800617A99F80010092903F0B58305990029C9
:103F580040F3508592B3DAED627A9AED5E7A77EEA5
:103F6800877A012ACAED627AC5ED007A21D0DAEDA6
:103F7800637A9AED5F7A77EE877A022ACAED637AD6
:103F8800C5ED017A15D0DAED647A9AED607A77EEAC
:103F9800877A032ACAED647AC5ED027A09D0DAED88
:103FA800657A9AED617A77EE877ACAED657AC5ED1A
:103FB800037A013A022AB8BF0222D2B2002B0CBF00
:103FC8001146022100F017BD5C023FF5C7AAFFF7B2
:103FD800C9BA00BF886A0020006900201263002067
:103FE8000AD7233C3C2B0020204A0020A042002076
:103FF8001F85EB51EE2D0020684B0020561800203D
:10400800942B002080430020742B0020504A00206D
:1040180004690020BCF1000FD6BFCCF1000207EE06
:1040280010CA07EE102A5148B8EEC77A007827EE72
:10403800287A00287EF436AF4D48D0ED006AF4EEB9
:10404800EA6AF1EE10FA41F13780B7EE005A35EE20
:10405800665A9FED486A48483BEE477A25EE065A6D
:1040680090ED006AE7EE056A26EE867AB5EEC07A2C
:10407800F1EE10FA40F2FE86C9EE876AB7EE006AE2
:1040880035EEC67AF0EE465AE7EE265AF0EE656A45
:10409800FEF738BF0123099ACAF8F4218AF8F031EB
:1040A800FEF794BC4FF07E53CAF8043125E6002889
:1040B80042F0C782BEF1000F41F0AF83FDEEE47A13
:1040C8000DF1380E17EE907AFDEEE67A2B4B2C4860
:1040D800CDF820A00EEB820117EE906AB1EE433ABC
:1040E80006918BF001084FFA8BFC07929A465346CB
:1040F80093ED007AFEEC017AE7EE257A0AF1100AD0
:10410800B0EE637AA3EE277AFDEEC77A17EE903AFF
:1041180017EE902AA342A8BF22469E42CCBF002198
:104128000BF00101002914BF114631469F42CCBF54
:10413800002308F0010307EE901A002B14BF134662
:104148003B46B8EEE77A07EE903A069BF8EEE77A38
:10415800BCF1000F18BFF0EE477A9E45E0EC017AFB
:10416800C5D1079ADDF820A0FFF79ABBAC3A00202A
:10417800B43A0020610BB63BA83A0020FC3F00206F
:1041880064290020C649DDED0E7A91ED007AC54B11
:10419800E7EE257ABBF1000F42F00E83BDEEE47A1C
:1041A80017EE106AB0EE647AA3EE277AFDEEC77AAE
:1041B80017EE90EA17EE907AA645A8BF27467645EF
:1041C800C8BF374607EE907AF8EEE77A012AC3EDC2
:1041D800007A3FF409AD91ED047ADDED0F7AE7EE50
:1041E800257AB0EE647AA3EE277AFDEEC77A17EE49
:1041F80090EA17EE907AA645A8BF27467645C8BF2D
:10420800374607EE907AF8EEE77A022AC3ED017A8C
:104218003FF4EAAC91ED087ADDED107AE7EE257A05
:10422800B0EE647AA3EE277AFDEEC77A17EE90EA2D
:1042380017EE907AA645A8BF27467645C8BF3746E9
:1042480007EE907AF8EEE77A032AC3ED027A3FF494
:10425800CBAC91ED0C7ADDED117AE7EE257AB0EE74
:10426800647AA3EE277AFDEEC77A17EE90EA17EE86
:10427800907AA645A8BF2746B645B8BF374607EE89
:10428800907AF8EEE77A042AC3ED037A3FF4ACACEF
:1042980091ED107ADDED127AE7EE257AB0EE647AC8
:1042A800A3EE277AFDEEC77A17EE90EA17EE907A1A
:1042B800A645A8BF2746B645B8BF374607EE907A49
:1042C800F8EEE77A052AC3ED047A3FF48DAC91ED58
:1042D800147ADDED137AE7EE257AB0EE647AA3EE70
:1042E800277AFDEEC77A17EE90EA17EE907AA64580
:1042F800A8BF2746B645B8BF374607EE907AF8EE0E
:10430800E77A062AC3ED057A3FF46EAC91ED187A88
:10431800DDED147AE7EE257AB0EE647AA3EE277A1B
:10432800FDEEC77A17EE90EA17EE907AA645A8BF79
:104338002746B645B8BF374607EE907AF8EEE77AD3
:10434800072AC3ED067A3FF44FAC91ED1C7ADDEDF8
:10435800157AE7EE257AB0EE647AA3EE277AFDEEB9
:10436800C77A17EE90EA17EE907AA645A8BF2746B7
:10437800B645B8BF374607EE907AF8EEE77A082ACE
:10438800C3ED077A3FF430AC91ED207ADDED167A73
:10439800E7EE257AB0EE647AA3EE277AFDEEC77AC7
:1043A80017EE90EA17EE907AA645A8BF2746B645BD
:1043B800B8BF374607EE907AF8EEE77A092AC3EDD8
:1043C800087A3FF411AC91ED247ADDED177AE7EE27
:1043D800257AB0EE647AA3EE277AFDEEC77A17EE57
:1043E80090EA17EE907AA645A8BF2746B645B8BF0B
:1043F800374607EE907AF8EEE77A0A2AC3ED097A8B
:104408003FF4F2AB91ED287ADDED187AE7EE257AE4
:10441800B0EE647AA3EE277AFDEEC77A17EE90EA3B
:1044280017EE907AA645A8BF2746B645B8BF3746C7
:1044380007EE907AF8EEE77A0B2AC3ED0A7A3FF492
:10444800D3AB91ED2C7ADDED197AE7EE257AE3EE20
:10445800274AFDEEE47AFFF7B9BB07EE902AF8EE9B
:10446800E77A114DDFF848E0D5ED004ADEED003A75
:104478000E4DCAED833A77EE677A06EE904ABCEEA7
:10448800C77AF8EEE66A17EE102A77EEE67ACAEDF2
:10449800844AAAF80822D5ED006AFEF76ABD00BF73
:1044A800FC3F002064290020BC400020D4400020AC
:1044B800282B002007EE103A99F800305B4FCAF815
:1044C800CC61B8EEC77AF7EE006A132B86EE879AAE
:1044D800B7F90400BAF8D05194ED080A01F019852B
:1044E800534B544A93ED001AD3ED093A93ED162A2B
:1044F80093ED1F3AD3ED0B1AD3ED144A93ED016AED
:1045080093ED0A4A93ED0C7AD3ED155AD3ED172A99
:10451800D3ED206A93ED045AD3ED030A69EE277AA6
:1045280069EE288A29EE088AE1EE273A02EB850629
:104538000021A2EE283ACAF8C011CAF8C411E1EE67
:10454800884AA6EE274AE7EE085A93ED1A7A93EDC1
:104558000F6A93ED021AD3ED0E1AC6ED003AE2EE99
:10456800A86A25EE635A27EE437A93ED0D2AD3ED18
:10457800192AC6ED204AA0EEE34A26EE646AD3ED76
:10458800183A83ED094AA7EE815AF0EE477AE1EE30
:10459800E45AA2EE086AE2EEC36AE3EEA87A83ED73
:1045A8000A5AC3ED145A83ED156A86ED403AC3EDF5
:1045B8001F6AC3ED207ACAF8C8116B1C03F01F03E9
:1045C800AAF8D031B880FEF780B81B4A11790029C3
:1045D8003EF44DAD1949097800293EF448AD1278EA
:1045E800DFED172A07EE902A164AF8EE676A128856
:1045F80007EE901A06EE102AF8EEE77AB8EE466A49
:1046080066EEA77AF7EE006A87EE862AB4EEE22A0B
:10461800F1EE10FA88BFB0EE622AB4EEE62AF1EEA7
:1046280010FAB8BFB0EE662AFEF723BDD2420020CA
:104638002C4E0020904B0020C84400209E420020B1
:10464800713DAA3F5C420020000000000AD7233CCD
:10465800D7A368416F12033B91ED026A91ED012ADD
:10466800D1ED037A5FED082A27EE066AA5EE026A05
:10467800A7EE846A26EE266AB4EEE26AF1EE10FA34
:10468800B4BFF0EE627AF0EE467A8DED0E6A88BF1E
:10469800B0EE626A012A3EF4EFAED1ED062AD1ED02
:1046A800051A91ED072A67EE222AE5EE212AE2EEA5
:1046B800042A62EEA62AF4EEC62AF1EE10FAF4EE07
:1046C800E72A8CBFB0EE462AB0EE622AF1EE10FA65
:1046D80098BFB0EE426AA8BFF0EE627A022ACDED2A
:1046E8000F2A3EF4C9AED1ED0A2AD1ED091A91ED8F
:1046F8000B2A67EE222AE5EE212AE2EE042A62EE70
:10470800A62AF4EEC62AF1EE10FAF4EEE72A8CBFD8
:10471800B0EE462AB0EE622AF1EE10FA98BFB0EE7B
:10472800426AA8BFF0EE627A032ACDED102A3EF461
:10473800A3AED1ED0E2AD1ED0D1A91ED0F2A67EE39
:10474800222AE5EE212AE2EE042A62EEA62AF4EEF7
:10475800C62AF1EE10FAF4EEE72A8CBFB0EE462A2C
:10476800B0EE622AF1EE10FA98BFB0EE426AA8BF26
:10477800F0EE627A042ACDED112A3EF47DAED1ED39
:10478800122AD1ED111A91ED132A67EE222AE5EECD
:10479800212AE2EE042A62EEA62AF4EEC62AF1EEF7
:1047A80010FAF4EEE72A8CBFB0EE462AB0EE622A81
:1047B800F1EE10FA98BFB0EE426AA8BFF0EE627A46
:1047C800052ACDED122A3EF457AED1ED162AD1EDC9
:1047D800151A91ED172A67EE222AE5EE212AE2EE54
:1047E800042A62EEA62AF4EEC62AF1EE10FAF4EED6
:1047F800E72A8CBFB0EE462AB0EE622AF1EE10FA34
:1048080098BFB0EE426AA8BFF0EE627A062ACDEDF4
:10481800132A3EF431AED1ED1A2AD1ED191A91EDD1
:104828001B2A67EE222AE5EE212AE2EE042A62EE2E
:10483800A62AF4EEC62AF1EE10FAF4EEE72A8CBFA7
:10484800B0EE462AB0EE622AF1EE10FA98BFB0EE4A
:10485800426AA8BFF0EE627A072ACDED142A3EF428
:104868000BAED1ED1E2AD1ED1D1A91ED1F2A67EE70
:10487800222AE5EE212AE2EE042A62EEA62AF4EEC6
:10488800C62AF1EE10FAF4EEE72A8CBFB0EE462AFB
:10489800B0EE622AF1EE10FA98BFB0EE426AA8BFF5
:1048A800F0EE627A082ACDED152A3EF4E5ADD1ED99
:1048B800222AD1ED211A91ED232A67EE222AE5EE6C
:1048C800212AE2EE042A62EEA62AF4EEC62AF1EEC6
:1048D80010FAF4EEE72A8CBFB0EE462AB0EE622A50
:1048E800F1EE10FA98BFB0EE426AA8BFF0EE627A15
:1048F800092ACDED162A3EF4BFADD1ED262AD1ED19
:10490800251A91ED272A67EE222AE5EE212AE2EE02
:10491800042A62EEA62AF4EEC62AF1EE10FAF4EEA4
:10492800E72A8CBFB0EE462AB0EE622AF1EE10FA02
:10493800CDED172A98BFB0EE426AB8BFF0EE672AED
:104948000A2A02F0C485D1ED2A7AD1ED291A91ED0F
:104958002B2A67EE277AE5EE217AE2EE047A67EEF3
:10496800A67AF4EEC67AF1EE10FAF4EEE27A8CBF8B
:10497800B0EE462AB0EE672AF1EE10FACDED187ABD
:1049880098BFB0EE426AB8BFF0EE627A0B2A3EF4E6
:1049980073ADD1ED2E2AD1ED2D1A91ED2F2A67EEA8
:1049A800222AE5EE212AE4EE022A62EEA62AB4EED5
:1049B800E26AF1EE10FAF4EEE27A8CBFB0EE627AB7
:1049C800B0EE467AF1EE10FACDED192A58BFB0EEE6
:1049D800476AB8BFF0EE627AFEF74EBD4FF4FA713F
:1049E800A1EB0C0CFFF7DEB9AAF874110591002BA6
:1049F80000F06C81022198F800305FEDEC6A99F8BC
:104A0800000098F8022007EE903AF8EEE77AB0EE48
:104A1800007A67EEA67AF4EEC77AF1EE10FA40F360
:104A2800488337EEC77A5FEDF66AB0EE676AA7EE9D
:104A3800266AB0EE467A1FEDF96AD5ED006A66EE91
:104A4800866AB0EEE66ACAED666A8AED696A9AB164
:104A580005EE902AB8EEE55ADFEDE55A66EEA64A6D
:104A680025EE255AF7EE005A75EEC55A64EE864AC9
:104A7800E5EE245A66EEA56ADFEDDE5A98F80530B1
:104A880027EE257A27EE267ACBB1DFEDD96ADFED5E
:104A9800DA5A26EE266A06EE903AF8EEE66A66EEEE
:104AA800866AF4EEE56AF1EE10FA00F3A486F7EEF2
:104AB800005A75EEE66A85EEA66A27EE067A0C2895
:104AC8009FEDCE8ADFEDCE6A00F07086B4EEC87A2C
:104AD800F1EE10FA98BFB0EE478AB4EEE68AF1EE2E
:104AE80010FAB8BFB0EE668A8AED4C8A002900F049
:104AF800E280B0EE007AF4EEC77AF1EE10FA05DD46
:104B080037EEC77ADFEDBF6AE7EE267A95ED017AD0
:104B1800DFEDBD6A27EE267AB0EEC76A8AED677ABE
:104B28008AED6A6A9AB106EE902ADFEDB15AF8EE7C
:104B3800E66A27EE075A66EEA56AF7EE005A75EEA2
:104B4800E65A25EE065AE6EE855A27EE257ADFED77
:104B5800A96A98F8063067EEA67A67EE877AABB14D
:104B680007EE103AB8EEC77ADFEDA15ADFEDA26A78
:104B780027EE067A27EE257AB4EEE67AF1EE10FAF9
:104B880040F33D86DFEDA16A67EEA67A0C2800F0B7
:104B9800E685DFED9A6A9FED9A7AF4EEE67AF1EE11
:104BA80010FA88BFF0EE667AF4EEC77AF1EE10FAE2
:104BB800B8BFF0EE477A0129CAED4D7A7BDD98F847
:104BC8000130DFED8B6A07EE903AF8EEE77AB0EE47
:104BD800007A67EEA67A98F80930F4EEC77AF1EE13
:104BE80010FA05DD37EEC77ADFED866AE7EE267A3A
:104BF80095ED027ADFED846A27EE267AB0EEC76A71
:104C08008AED687A8AED6B6A9BB106EE903ADFED21
:104C1800785AF8EEE66A27EE075A66EEA56AF7EEC6
:104C2800005A75EEE65A25EE065AE6EE855A27EE44
:104C3800257ADFED706A98F8073067EEA67A67EE96
:104C4800877A0BB307EE103AB8EEC77ADFED685AE9
:104C5800DFED696A27EE067A27EE257AB4EEE67A62
:104C6800F1EE10FA0CDCB5EEC07AF1EE10FA01F1B3
:104C78003682B7EE006A36EE477AC6EE076A01E07A
:104C8800DFED626A67EEA67A0C2800F08785DFED13
:104C98005B6A9FED5B7AF4EEE67AF1EE10FA88BF74
:104CA800F0EE667AF4EEC77AF1EE10FAB8BFF0EEDD
:104CB800477ACAED4E7A092800F0468596F82150C1
:104CC800002D40F0FC8400238AF84431504B1B78B7
:104CD80023B9504DAF78002F41F09B8299F80030EE
:104CE800072B00F07E850022072B8AF800217DF42F
:104CF80099AC09F0FFF80590FDF796BC718B059A01
:104D08008A42C0F2DD82B2F5FA6FD4BFC1EB02036A
:104D1800C1F5FA634FF47A7202FB03F2C1F5FA6146
:104D2800B2FBF1F2FFF760B8F81AB0F5FA7FBEF6F9
:104D3800FEAF8645FEF6FDAFDFED3A7AFEF7FFBF20
:104D4800354A0B920025354E354FDDF82C80CDF8CD
:104D580018A0AA46B6EC018AD4ED087AB8EEC88A3B
:104D680028EE278ABAF1000F02F064867BBB99F817
:104D78000030082B58D005F5D260B0EE480A204420
:104D8800D4F88C36984705F5E360D4F814372044F6
:104D9800984799F80030032BB0EE408A22D0D4F817
:104DA800AC30D6F84406B0EE480A984708EB8A03B8
:104DB8000AF1010ABAF1030F05F12C0583ED010A86
:104DC8003DF4A4ACDBF8003003F00053C2E705F56E
:104DD800F460B0EE480A2044D4F89C379847B0EE07
:104DE800408AC4E724F00EFC27F81A00D7E700BF72
:104DF8000AD7233C00004843A4707D3F00C0F94413
:104E080000C0F9C4D7A368416F12033B0000C84231
:104E1800D1420020CF270020AC720020C06A0020B9
:104E2800D242002000000000B0EE480A24F0EAFB5D
:104E380027F81A009FE73B1AB3F5FA7FBEF692AF40
:104E48009E45FEF691AF5FED097AFEF793BFDB4B07
:104E5800DFF8E0A31A68DA4BDA4F9AF80001D26952
:104E68001B883A807B8000287EF417AF0590D64CCB
:104E7800FDF7DABBDFEDD56AFEF752B809F03AF86C
:104E880099F800300C9ACF4F801A012B788000F0E7
:104E98000382072B7DF4C4AD09F02CF80590FDF7CB
:104EA800C1BDDFF89483DAED017A9AED006AB8F8AB
:104EB8000000D8F8143077EEA77AF0EE006AB0EE6A
:104EC800677AA6EE267A01380AEBC002D6EE267A71
:104ED800083A1033F6EE003A27EE237A67EEA37A03
:104EE8008AED207ACAED217ADFF848A357460AF1FD
:104EF800800192ED027A92ED036AD7ED036AD7ED4D
:104F0800027A53ED014A13ED025A37EE674A76EEFC
:104F1800C65A77EE277AE4EE845A0138A2F10802DD
:104F2800E5EE047A07F1080703F1080336EE267A5E
:104F380001F10801E4EE877AE5EE475A67EEA37AB5
:104F480025EEA37AC1ED007A81ED017AD1D1142E34
:104F580007D108F0CFFF069B9A4FC01A7880DAF87D
:104F6800D4519B4B0B939B4ADBF80030013582FBF5
:104F780005125119EA17C2EBA102C2EBC202AD1A1F
:104F8800CAF8D45103F00053DCE608F0B3FF059AE1
:104F98008C4B801AD880FEF748BE8F4A8F48B2F9EA
:104FA8000420BAF80811DFED8E6A9FED8E7A80FB37
:104FB8000270D217C2EBA002521A12B207EE902A60
:104FC800F8EEE77A67EEA67A77EE876ABDEEE66ACC
:104FD80016EE102A2032402A41F2D380DFED7B6A98
:104FE800BDEEE77A17EE102A2032402A01F2C5807A
:104FF8009FED7D7AF4EEC77AF1EE10FA42F304835E
:10500800DFED7A5A9FED7A6A01E0F0EE477AF4EE26
:10501800C67AF1EE10FA37EEE57AF6DCDFED757A4E
:10502800B4EEE77AF1EE10FA42F1EA82DFED6F5A58
:105038009FED716A01E0B0EE677AB4EEC67AF1EEE0
:1050480010FA77EE257AF6D49FED667AF4EEC77AF1
:10505800F1EE10FA00F35C849FED687AF4EEC77AFB
:10506800F1EE10FA44BF9FED637A77EE677A67EE48
:10507800A75A9FED635A9FED636A9FED637AA5EE89
:10508800856A27EEA55AA5EE867AE5EE077A95EDAC
:10509800016AD5ED005A27EEC67A65EEA77AA5EE25
:1050A800A67AE6EE267A85ED007AC5ED017AFEF756
:1050B800C9BEB0EE677ABEE4544890ED007AFEF7B8
:1050C800D5BF534C534D544AD4ED004AD5ED003A60
:1050D800524C1278CAED833ACAED844AD4ED006A7C
:1050E80012B101228AF81822DAED857AFDF741BF5C
:1050F800A368002B3EF4DCAD04F144012046984738
:10510800DBF800300793FEF7D3BD45494548D1F891
:10511800EC10006844F62067B942A8BF3946B1F5DB
:105128007A7FB8BF4FF47A7189B2C706AAF84611D8
:1051380041F1BD840698002840F0E2833A480068AF
:105148000690B0F936C0394FDAF84801A7FB01716B
:105158008F09642191FBF7F11429FDEEC87A0AEB57
:10516800400EA8BF142101308142CAF8480117EE49
:10517800907ADCBF0020CAF848010AEB4000AEF87C
:105188004C71B0F94C1107EE901AF8EEE77A38EE48
:10519800678AFDEEC87ACDED057ABDF9140080EA7C
:1051A800E071A1EBE071614502F31B8220490846DA
:1051B8004FF07E510160FEF771BE00BF2845002008
:1051C80034300020D2420020886A0020000000000D
:1051D800AC72002093244992784300206766666683
:1051E80035FA8E3CDB0FC93FDB0F4940DB0FC94066
:1051F800E4CB1641DB0F49C0E4CB16C1DB0FC9BFB6
:1052080092E741B99730083C15A82ABEA83A002071
:10521800A4290020C040002054450020D040002090
:10522800280E00201C2B00200C430020D34D6210B8
:10523800000000208C1B0020784B00201D213448E2
:1052480005F0B6FF00283EF4F6AD324BDB78002BB4
:105258007EF4F1ADDFED307A304938EE678AC7F574
:10526800FA62FDEEC87A12B2CDED0A7ABDF928309D
:105278001B0381FB0301DB17C3EBA11302FB03F341
:1052880043F30F333B4407EE903AB8EEE78A85EDD7
:10529800038AFEF7D0BD224F08F02CFE214ADAF827
:1052A800043212680590C31A9A1ACAF80402BB801D
:1052B800FA80FDF7B7BB08F01DFE0C90FDF742BA67
:1052C800069A2BE598F80830C3F1640307EE903A84
:1052D800FEF70BBD144A127812F0100201F0E687AF
:1052E8009AF80C11DAF8102195ED017A00290CBF13
:1052F80001214FF0FF3102FB01F207EE902AF8EE90
:10530800E77A77EE877AC5ED017AFEF7A4BD00BF8C
:105318001C2B0020A044002000007A44D34D6210CA
:10532800D2420020742B002024560020BBF1000F2D
:105338003EF4F7AAF4EEE47AF1EE10FAB8BFF0EE14
:10534800667AFDEEE77ABDEEE67A17EE907A17EE0A
:1053580090EAA74217EE106AA8BFA646BE42C8BF89
:10536800B64607EE90EAF8EEE77A012AC3ED007A2E
:105378003EF43AAC91ED047ADDED0F7AE7EE257A4A
:10538800B0EE637AA3EE277AB4EEE47AF1EE10FA7F
:10539800F0EE477AB8BFF0EE667AFDEEE77A17EEE0
:1053A800907A17EE90EAA742A8BFA646B742B8BFC0
:1053B800B64607EE90EAF8EEE77A022AC3ED017ADC
:1053C8003EF412AC91ED087ADDED107AE7EE257A1D
:1053D800B0EE637AA3EE277AB4EEE47AF1EE10FA2F
:1053E800F0EE477AB8BFF0EE667AFDEEE77A17EE90
:1053F800907A17EE90EAA742A8BFA646B742B8BF70
:10540800B64607EE90EAF8EEE77A032AC3ED027A89
:105418003EF4EAAB91ED0C7ADDED117AE7EE257AF0
:10542800B0EE637AA3EE277AB4EEE47AF1EE10FADE
:10543800F0EE477AB8BFF0EE667AFDEEE77A17EE3F
:10544800907A17EE90EAA742A8BFA646B742B8BF1F
:10545800B64607EE90EAF8EEE77A042AC3ED037A37
:105468003EF4C2AB91ED107ADDED127AE7EE257AC3
:10547800B0EE637AA3EE277AB4EEE47AF1EE10FA8E
:10548800F0EE477AB8BFF0EE667AFDEEE77A17EEEF
:10549800907A17EE90EAA742A8BFA646B742B8BFCF
:1054A800B64607EE90EAF8EEE77A052AC3ED047AE5
:1054B8003EF49AAB91ED147ADDED137AE7EE257A96
:1054C800B0EE637AA3EE277AB4EEE47AF1EE10FA3E
:1054D800F0EE477AB8BFF0EE667AFDEEE77A17EE9F
:1054E800907A17EE90EAA742A8BFA646B742B8BF7F
:1054F800B64607EE90EAF8EEE77A062AC3ED057A93
:105508003EF472AB91ED187ADDED147AE7EE257A68
:10551800B0EE637AA3EE277AB4EEE47AF1EE10FAED
:10552800F0EE477AB8BFF0EE667AFDEEE77A17EE4E
:10553800907A17EE90EAA742A8BFA646B742B8BF2E
:10554800B64607EE90EAF8EEE77A072AC3ED067A40
:105558003EF44AAB91ED1C7ADDED157AE7EE257A3B
:10556800B0EE637AA3EE277AB4EEE47AF1EE10FA9D
:10557800F0EE477AB8BFF0EE667AFDEEE77A17EEFE
:10558800907A17EE90EAA742A8BFA646B742B8BFDE
:10559800B64607EE90EAF8EEE77A082AC3ED077AEE
:1055A8003EF422AB91ED207ADDED167AE7EE257A0E
:1055B800B0EE637AA3EE277AB4EEE47AF1EE10FA4D
:1055C800F0EE477AB8BFF0EE667AFDEEE77A17EEAE
:1055D800907A17EE90EAA742A8BFA646B742B8BF8E
:1055E800B64607EE90EAF8EEE77A092AC3ED087A9C
:1055F8003EF4FAAA91ED247ADDED177AE7EE257AE2
:10560800B0EE637AA3EE277AB4EEE47AF1EE10FAFC
:10561800F0EE477AB8BFF0EE667AFDEEE77A17EE5D
:10562800907A17EE90EAA742A8BFA646B742B8BF3D
:10563800B64607EE90EAF8EEE77A0A2AC3ED097A49
:105648003EF4D2AA91ED287ADDED187AE7EE257AB4
:10565800B0EE637AA3EE277AB4EEE47AF1EE10FAAC
:10566800F0EE477AB8BFF0EE667AFDEEE77A17EE0D
:10567800907A17EE90EAA742A8BFA646B742B8BFED
:10568800B64607EE90EAF8EEE77A0B2AC3ED0A7AF7
:105698003EF4AAAA91ED2C7ADDED197AE7EE257A87
:1056A800E3EE273AF4EEE34AF1EE10FAD4BFF0EE57
:1056B800637AF0EE667AFDEEE77AFEF787BA1E2186
:1056C800CA4805F075FD00283FF4FDAA0A9B002B87
:1056D8007FF4F9AA9AF8B031AB4242F00B80C44B80
:1056E800DAED6D7A93ED010ADAED4E5A9FEDC16A53
:1056F800DFEDC16A27EEE57A68EE277AA8EE007A30
:10570800E5EE807AB4EEC67AF1EE10FA88BFB0EE14
:10571800467AB4EEE67AF1EE10FAF4EEC67AB8BF3D
:10572800B0EE667AF1EE10FA88BFF0EE467AF4EE43
:10573800E67AF1EE10FAB8BFF0EE667A8AED4C7AA6
:10574800CAED4E7AFFF7BFBAAC4FBDF81430BB8034
:10575800FDEEC87A17EE903AFB80FFF7AFBA9FEDDF
:10576800A57ADFEDA56AA54FF4EEC77AF1EE10FA37
:1057780098BFB0EE677AFDEEE77AB4EEE67AF1EE1E
:1057880010FA17EE903AB8BFB0EE667A01298AEDA2
:105798004D7A7B803FF713AAFFF790BABDEEE77A00
:1057A800964F17EE103ABB80FFF771BAB4EEC87A7D
:1057B800F1EE10FA98BFB0EE478ABDEEC77AB4EEA4
:1057C800E68A8E4FF1EE10FA17EE103AB8BFB0EE37
:1057D800668A8AED4C8A3B8000297FF48AA9FFF704
:1057E8006DBA08F087FB089A844F99F80030801A40
:1057F800B880FFF778BA9FED826AFFF75EB9B5EE19
:10580800C07AF1EE10FA00F16684B7EE006A36EE5F
:10581800477AC6EE076AFFF7B7B9FDEEE47A0EA835
:1058280017EE907AFDEEE67A764BDFF8F8E107920C
:1058380000EB820117EE906A0691B1EE433A8BF0C5
:1058480001084FFA8BFC1946CDF820A00B4693EDC2
:10585800007AF0EC017AE7EE257A0BF001031031BB
:10586800B0EE637AA3EE277AF4EEC74AF1EE10FAA7
:10587800D8BF0023002BF0EE477A18BFB0EE667A47
:10588800BDEEC77AFDEEE77A17EE102A17EE90AA5A
:10589800A24217EE103AA8BF23469642CCBF002278
:1058A8000BF00102002A08BF3346A24517EE902AE2
:1058B80007EE103AA8BF22465745CCBF002308F090
:1058C8000103002B08BF3A4607EE902AB8EEC77AC4
:1058D800F8EEE77A069BBCF1000F18BFF0EE477AA6
:1058E8008342EEEC017AB1D1FEF73BBC96F820106A
:1058F800C1EB411001EB8001C90089B2FEF7DABAA9
:10590800414800680690B0F836C04FEA5C0C1AE4CB
:105918009FED3E7A77EE677AFFF7A9BB3C4BDAF842
:10592800D8C10B93BAF8D081C8F12003D8B2394B4B
:1059380008EB4C1703EB8707830801F0B7860133A0
:105948001B013549354A079307EB030E07F110038E
:1059580013ED024A13ED035A13ED016A13ED047AAD
:1059680051ED024A51ED035A51ED016A51ED047AA5
:1059780064EE244A65EE255A66EE266A67EE277AB3
:105988001033734542ED024A42ED035A42ED016A73
:1059980042ED047A01F1100102F11002D8D1079BFF
:1059A8001F49A3F11002174401EB020E524410F0F4
:1059B800030309D0B7EC017AFEEC017A67EE277A87
:1059C800013BE2EC017AF5D1B8F1000F41F09B847C
:1059D800142E7FF4C8AA08F08DFA069B074FDAF850
:1059E800D451C01A7880FFF7BEBA00BF1C2B002024
:1059F8000000002000C0F94400C0F9C4D2420020D1
:105A08000000C842FC3F00200C430020DB0F494047
:105A1800AC720020904B0020204D00209C1B0020E1
:105A2800104D002064290020DAF8D881C14AC24B01
:105A38000B9203EBC803126807929DED077A9B88C7
:105A4800DFEDBE7ABE4AF8EE478A09EE103A643BAB
:105A5800C82BA8BFC82368EEA78AF8EE497A782B26
:105A6800B8BF782368EEA78A07EE903A2C27B0EEE5
:105A7800680A07FB0827B8EEE78A23F00FFEB8EE9E
:105A8800C99AF0EE409AB0EE680A23F069FD38EE44
:105A9800097A79EE487A28EE098A67EE877AB7EEAE
:105AA800006A88EE277A142EF8EE007A77EE076AF5
:105AB80060EE277A89EEA67A77EE065A36EE477AAE
:105AC800C6EE256A67EEA67A27EE267AC7ED006A43
:105AD80087ED047AC7ED026AC7ED017AC7ED037A4C
:105AE80001F08F86974B99F8006008F1010883FB55
:105AF800083CACEBE87C0CEB4C0C0135A8EB0C0C2F
:105B0800CAF8D451CAF8D8C10CE7DFF83C8298F833
:105B180000205FEA920C01F00F87DFF848E20CF1F1
:105B2800010040010EEB00070EF12003AEF17001F9
:105B380013ED076A53ED056A13ED037A53ED017A05
:105B480053ED025A13ED084A53ED064A13ED045A71
:105B580026EE066A66EEA66A27EE077A67EEA77A49
:105B6800A4EE046A2033BB42E4EEA46A01F11001FA
:105B7800A5EE057AE5EEA57AF1EEC65AB1EEE66A2B
:105B8800F1EEC76AB1EEE77A41ED085A01ED076A0E
:105B980041ED066A01ED057ACAD1203886440AEB40
:105BA8000C1112F0030318BF0EF1080E0FD05EEDB2
:105BB800017A1EED027A67EEA77A013BE7EE077AD3
:105BC8000EF1080EB1EEE77AA1EC017AEFD1142EAE
:105BD80001F0FF850135CAF8D45101E05A4B1A7813
:105BE800DAF8D8E154489FED597A4FEACE07C3193D
:105BF80083ED007A002A7AD05549B0EE476AF0EE74
:105C0800476A0023F1EC017A013367EEA77A05EEC3
:105C1800903AB4EEE77AF1EE10FAF8EEE55AB8BF2A
:105C2800B0EE677A934276EEA76AA7EEA56AE9D145
:105C3800F5EEC06AC319F1EE10FA83ED007A56DD6D
:105C4800C6EE265A434B444A1288F7EE007A75EEA0
:105C5800E75AD3ED007A65EEA77AFDEEE77A17EEFC
:105C6800903A812B41F34B839342A8BF134607EE2A
:105C7800903AF8EEE77A394B2C2101FB0E3393ED7D
:105C8800097AD3ED003A93ED0A6A93ED014AD3ED10
:105C9800046AD3ED034A93ED025AA3EEA77AA4EE61
:105CA800276A66EEC76AA7EE646ABDEEC77AE5EEB4
:105CB800276A17EE101A812983ED096AC3ED0A6A6B
:105CC80041F31A838A42A8BF0A4607EE902AF8EEE3
:105CD800E77AFCEEE77ACDED077ABDF81C30C219F9
:105CE8009380BEF1000F02D1132E01F0C484152E4B
:105CF8007FF42DA938441A4F838827F81E300D4B9E
:105D0800DAF8D4510B93FFF72EB9DFF85C8010480E
:105D1800D8F80820B8F80C1022F0B4FB99F8006005
:105D2800142E01F06485DAF8D4510135CAF8D4513B
:105D3800FFF7B9B8AC720020904D002027D4D236B6
:105D48002872002056555555724B0020000000005F
:105D58008C1B0020744B0020704B0020A84D0020A5
:105D6800D24200200C1C0020784B0020DFF8CC83A6
:105D7800B8F80060D8F804E04FEA560C4FEA8C02F5
:105D88000AEB8607F6080AEB020300F09F80103240
:105D98000136E34803EB06163A4410330EF11005BA
:105DA80007F1100151ED032A51ED043A10ED043AC0
:105DB80010ED032A51ED026A11ED016A10ED020A95
:105DC80010ED018A12ED044A12ED035A53ED044A0C
:105DD80053ED035A13ED027A53ED017A52ED020A9C
:105DE80012ED011A73EE238A72EE221A40ED048A2C
:105DF80040ED031A70EE268A78EE061A40ED028A04
:105E080040ED011A74EE848A75EE851A43ED048A12
:105E180043ED031A77EE208A77EE811A43ED028A62
:105E280043ED011A73EE633A75EE655A15ED035AA0
:105E380032EE623A74EE644A65EE631A15ED044A6E
:105E480023EE052A64EE652AE3EE041A1033B34202
:105E580024EE843AA3EE842A00F1100005F110051F
:105E6800A5EE853A01F1100102F11002E4EE852A4F
:105E780041ED071A01ED082A02ED073A42ED082A1A
:105E880055ED055A15ED065A70EE666A38EE466A03
:105E980030EEC77A71EE677A26EE253A65EEE63A75
:105EA80025EE674A67EE054AE6EE053AA6EE853A1C
:105EB800A7EE254AE7EEA54A01ED063A41ED053A77
:105EC80002ED064A42ED054A7FF46CAF1FFA8CF5E5
:105ED80072462946934818F00FFF2946D8F804203F
:105EE800384618F009FF99F80030142B7FF437A8CA
:105EF800FFF72FB807F0FEFF99F800600690142E00
:105F080005BF894FDAF8D451DAF8D4513D80FCF74F
:105F1800E5BB864EDFF8288296ED004A96ED097AB1
:105F2800D6ED014A96ED0A6AD6ED046A96ED035A53
:105F3800D6ED025A69EE277A08EB8503A4EE277A94
:105F4800A4EEA76A66EEC76AA7EE456AE5EEA76AF9
:105F580027EE000A86ED096AC6ED0A6A83ED007A23
:105F680029EE088A23F04EFB69EE288AD6ED145AEA
:105F7800D6ED1F6A96ED0B1AD6ED161A96ED155A40
:105F880096ED207A96ED0C2AD6ED172A96ED0F6A33
:105F9800D6ED1A7A96ED0E3AD6ED0D3A96ED194AE7
:105FA800D6ED184AE8EE015A002208EB8503E8EE20
:105FB800A16A00B2CAF8C021A2EE085ACAF8C421E0
:105FC800CAF8C821A8EEA27A26EE656A67EEE67AD4
:105FD800A3EE655AA8EE236AA6EEC47AE8EEA47A80
:105FE80086ED145AC3ED205A86ED156AC3ED406A52
:105FF80086ED1F7AC6ED207AFEF7DFBAB4F92430B1
:10600800E26207EE903A0122F8EEE77A2366E26749
:106018000023012EC4ED1C7AC4ED1B7A636701F0DE
:10602800FB82AE427CF4DDADB4F92630636607EE40
:10603800903A00220123F8EEE77A2263C4F8903000
:106048000023012EC4ED217AC4ED207AC4F88830EB
:1060580001F0DE82AE427CF4F4ADB4F92830A366D8
:1060680007EE903A00220123F8EEE77A6263C4F85B
:10607800A4300023012EC4ED267AC4ED257AC4F895
:106088009C307CF40EAE9FED2A8AB8F1030F2AD01B
:10609800BBF1000F09D007EE90BAF8EEE77AF4EEFC
:1060A800C87AF1EE10FA01F14C84224AA36E126804
:1060B800F880002103EB550393FBF5F565639162C6
:1060C8001163D162FCF7EEBD1B4A927B002A3DF4B6
:1060D800D5AEFDF7D7BEF7EE006AFEF755BDF7EE71
:1060E800006AFEF7CFBDB0EE480A23F08BFA00B283
:1060F800CEE7BAF87411013909B200290591AAF856
:1061080074113DF727AFFEF772BCBAF8461101F5D6
:106118007A7189B2FDF7CEBE00F00100FDF764BDCB
:106128009C1B00208C1B0020D24200202C4E0020FB
:10613800000000002845002010510020784B002066
:10614800904B0020CD49DFEDCE7A0968CAED787A08
:1061580011F0805100F0CA84B7EE007A77EE677AC2
:10616800F4EEE57AF1EE10FA88BFF0EE657AF0EE1B
:10617800675ACAED857AFDF7F5B9DFEDC27AFEF701
:1061880086BFF4EEC77AF1EE10FA41F34683DFEDED
:10619800BE5A9FEDBE6A01E0F0EE476AF4EEC66AA9
:1061A800F1EE10FA36EEE57AF6DCDFEDB96AB4EE18
:1061B800E67AF1EE10FA41F14E83DFEDB35A9FED26
:1061C800B56A01E0B0EE667AB4EEC67AF1EE10FA7E
:1061D80077EE256AF6D49FEDB07AF4EEC76AF1EE51
:1061E80010FA40F326859FEDAD7A77EE666A66EE83
:1061F800A65A9FEDAB5A9FEDAB6A9FEDAB7AA5EE21
:10620800856A26EEA55AA5EE867AE5EE076AFEF7B8
:10621800E7BEA64E3378013B0D2B15D8DFE813F007
:106228007C01CC01A40189011400140067015E01FE
:10623800EE00D8001001D000CA000E001F201FF089
:106248005FFE08B901233370012F01F0B080EB78AD
:10625800002B3EF443ADDBF80030D80441F148830D
:10626800934B9B8807EE903AF8EEE77A914A92EDC5
:10627800012AD2ED022A92ED033AD2ED043A92EDC8
:10628800054AD2ED064A92ED075AD2ED085A92ED28
:10629800096AD2ED0A6A92ED0B7AB4EE672AF1EE3A
:1062A80010FAF4EE672A14BF01230023F1EE10FA66
:1062B800B4EE673A18BF43F00103F1EE10FAF4EEBA
:1062C800673A18BF43F00103F1EE10FAB4EE674ADB
:1062D80018BF43F00103F1EE10FAF4EE674A18BF55
:1062E80043F00103F1EE10FAB4EE675A18BF43F019
:1062F8000103F1EE10FAF4EE675A18BF43F00103F8
:10630800F1EE10FAB4EE676A18BF43F00103F1EE3C
:1063180010FAF4EE676A18BF43F00103F1EE10FAC1
:10632800B4EE677A18BF43F00103F1EE10FA18BF14
:1063380043F00103002B41F0748292ED007AB4EE31
:10634800677AF1EE10FA41F06C825B4DDAF8BC2105
:106358002B689A4201F26C823378012B3EF4BEAC72
:106368009AF8B821002A3EF4B9AC0B2B18D80122B0
:106378009A4040F6030112EA010716D112F4C06FE1
:106388000ED0093B012B0BD8452014F077FEFF20D7
:1063980014F074FE494814F0E3FD384614F06EFE1C
:1063A800474B2A685A600B23337000238AF8B831A8
:1063B800FEF794BC012F01F0D9820E23337043E716
:1063C800012F02D105F00CF9AF780D2333703BE7AC
:1063D8003C4B1B78002B01F086821A201FF090FDA1
:1063E800002841F080829AF8B831002B41F07B8276
:1063F800092333700EF044F9AF7825E71A201FF00F
:106408007FFD0028F6D0304B1B88002BF2D12F4B94
:1064180045201F6814F032FE0E2014F02FFE384677
:106428000DF04EFE099F38460DF04AFE284A4FF4FB
:1064380080510A233846118033700DF053FED9E796
:106448001F4B1D4A5B681268C833934205D322F07C
:10645800ADFEAF7800283FF4F7AE032F7FF4F2AE1D
:106468001C4F38681EF00CFC1B4B1B780022022BBB
:106478003A6001D111F0F6FDAF78E3E61C2B00205D
:106488000000008000000000DB0FC940E4CB16418B
:10649800DB0F49C0E4CB16C1DB0FC93FDB0F494016
:1064A80092E741B99730083C15A82ABECE270020AC
:1064B800C4400020CC3F0020E84A002008E0020841
:1064C8002C2B0020E82B002094290020982900205C
:1064D800242B002098410020712B002014F01AFD75
:1064E8000EF0EEF8002841F09782AF78ACE614F091
:1064F80011FDA44B002105208DE80300A3F108023B
:10650800029153200EF090FD0028EED19E4BAF78FB
:1065180018600823337097E69C480378DF0701F179
:10652800A4821F201FF0ECFC0028DED00C2333705F
:10653800DBE714F0EFFC964A0292A2F10C03262145
:1065480001930091A2F10A035021163A49200EF056
:106558006BFD0028C9D18C4BAF7818604FF0FF3223
:106568005A60072333706FE6874F14F0D3FC894ACB
:106578007B68126864339342B7D2402014F0A0FCC1
:106588000028B2D13B6884494FF040080DE00591DE
:1065980014F074FD05993B680A680133013AB8F1B3
:1065A80001080A603B6001F0FA817C4AD35C184616
:1065B800002BECD101F0F8B9764B734A1B68536095
:1065C80075490023136003220B6032703CE6744B5C
:1065D800DFED747A93ED080AB4EEE70AF1EE10FAEB
:1065E80040F2F98623F0A4F8DAED507A20EE270A73
:1065F80023F008F8B0F5617F00F3F18607EE900A02
:10660800F8EEE76ADFED687A66EEA76A07EE907A39
:10661800B8EEE77AFDEEE67A17EE903A2033402B93
:1066280041F21D819FED610A22F0ECFF00B207EEF6
:10663800900AF8EEE77A38EE278A85ED038AFDF7A7
:1066480027BC0698002800F0E486FDEEE47A0EA93F
:1066580001EB820217EE907AFDEEE67A1346544873
:10666800544E5A4617EE90CAB1EE433A9B4614E090
:10667800FDEEC77A17EE903ABB4203DBA342A8BFF0
:106688002346984607EE908AF8EEE77A5945E6ECF5
:10669800017A00F110003DF4AAAA90ED007AF1EC1D
:1066A800017AE7EE257AB846B0EE637AA3EE277A48
:1066B800F0EE477A002ADBD06346BEF1000F06D021
:1066C800B4EE647AF1EE10FA48BFF0EE667AFDEEA9
:1066D800E77A17EE908AE04504DBA04517EE903A7A
:1066E800A8BF234607EE903AF8EEE77ACEE7069879
:1066F800002800F0F086FDEEE67A0EA901EB820292
:1067080017EE90CAFDEEE47A13462948294E5A46F8
:1067180017EE907A9B4614E0FDEEC77A17EE908A42
:10672800474503DCA0454346A8BF234607EE903AF9
:10673800F8EEE77A8B45E6EC017A00F110003DF4BB
:1067480056AA90ED007AF1EC017AE7EE257A3B46FD
:10675800B0EE647AA7EE837AF0EE477A002ADBD0AF
:10676800BEF1000F06D0F4EE474AF1EE10FAC8BFAA
:10677800F0EE667AFDEEE77A634617EE908AC44536
:10678800D0DDD3E7BCBD02082C2B0020D156002059
:1067980002BC0208E84A0020944100208CBB020891
:1067A800103A00208FC2753CD06D393A00000000C5
:1067B800FC3F002064290020BDEEE67A17EE106A3F
:1067C800B0EE647AA3EE277AF0EE477ABEF1000FB6
:1067D80040F04E82FDEEC77A17EE90EA17EE907AF7
:1067E800A645A8BF27467645C8BF374607EE907A24
:1067F800F8EEE77A012AC3ED007A3DF4F5A991EDA8
:10680800047ADDED0F7AE7EE257AB0EE647AA3EE2E
:10681800277AFDEEC77A17EE90EA17EE907AA6452A
:10682800A8BF2746B645B8BF374607EE907AF8EEB8
:10683800E77A022AC3ED017A3DF4D6A991ED087AE8
:10684800DDED107AE7EE257AB0EE647AA3EE277ACA
:10685800FDEEC77A17EE90EA17EE907AA645A8BF24
:106868002746B645B8BF374607EE907AF8EEE77A7E
:10687800032AC3ED027A3DF4B7A991ED0C7ADDED58
:10688800117AE7EE257AB0EE647AA3EE277AFDEE68
:10689800C77A17EE90EA17EE907AA645A8BF274662
:1068A800B645B8BF374607EE907AF8EEE77A042A7D
:1068B800C3ED037A3DF498A991ED107ADDED127AD3
:1068C800E7EE257AB0EE647AA3EE277AFDEEC77A72
:1068D80017EE90EA17EE907AA645A8BF2746B64568
:1068E800B8BF374607EE907AF8EEE77A052AC3ED87
:1068F800047A3DF479A991ED147ADDED137AE7EE87
:10690800257AB0EE647AA3EE277AFDEEC77A17EE01
:1069180090EA17EE907AA645A8BF2746B645B8BFB5
:10692800374607EE907AF8EEE77A062AC3ED057A3D
:106938003DF45AA991ED187ADDED147AE7EE257A3F
:10694800B0EE647AA3EE277AFDEEC77A17EE90EAE6
:1069580017EE907AA645A8BF2746B645B8BF374672
:1069680007EE907AF8EEE77A072AC3ED067A3DF447
:106978003BA991ED1C7ADDED157AE7EE257AB0EEAC
:10698800647AA3EE277AFDEEC77A17EE90EA17EE3F
:10699800907AA645A8BF2746B645B8BF374607EE42
:1069A800907AF8EEE77A082AC3ED077A3DF41CA935
:1069B80091ED207ADDED167AE7EE257AB0EE647A6D
:1069C800A3EE277AFDEEC77A17EE90EA17EE907AD3
:1069D800A645A8BF2746B645B8BF374607EE907A02
:1069E800F8EEE77A092AC3ED087A3DF4FDA891ED9F
:1069F800247ADDED177AE7EE257AB0EE647AA3EE15
:106A0800277AFDEEC77A17EE90EA17EE907AA64538
:106A1800A8BF2746B645B8BF374607EE907AF8EEC6
:106A2800E77A0A2AC3ED097A3DF4DEA891ED287ABF
:106A3800DDED187AE7EE257AB0EE647AA3EE277AD0
:106A4800FDEEC77A17EE90EA17EE907AA645A8BF32
:106A58002746B645B8BF374607EE907AF8EEE77A8C
:106A68000B2AC3ED0A7A3DF4BFA891ED2C7ADDED2F
:106A7800197AE7EE257AE3EE274AFDEEE47AFDF788
:106A8800A5B807F037FA0890FDF709B96F49096802
:106A980011F080512AD0B6EE007A67EE877AF4EECC
:106AA800E75AF1EE10FA3FF562ABFFF755BB0798CE
:106AB800C0003EF53FABFDF7F1B9654C654D664A40
:106AC800D4ED004AD5ED003A644C1278CAED857AC7
:106AD800CAED833ACAED844AD4ED006A002A3CF430
:106AE80048AA01228AF81822FCF743BA13F4800155
:106AF80001D00021CFE7B6EE007AF4EEC75AF1EEE6
:106B080010FAC8DCFCF72EBDFDEEE67A20460EAB87
:106B18005349544F17EE906A744603EB820C86462D
:106B2800D1ED007AB3EC017AA7EEA57A1031B0EE78
:106B3800646AA3EE076A07EE906AB0EE467A34B14B
:106B4800B4EE646AF1EE10FA48BFB0EE667ABDEEB4
:106B5800C77A17EE100A864204DC7045A8BF704653
:106B680007EE900AF8EEE77A9C45E7EC017AD7D170
:106B7800FCF796BE012A7FF786AA07EE101AB8EE30
:106B8800C77AC7EE876AB1EEE68AFFF77EBA012AAE
:106B980040F33E8507EE101AB8EEC77AC7EE876A4B
:106BA800B1EEE68AB8F1030F14D0BBF1000F09D09B
:106BB80007EE90BAF8EEE77AB4EEE78AF1EE10FA4B
:106BC80000F3BF86636E03EB550393FBF5F3236372
:106BD800FFF740BAB0EE480A22F014FD00B2E4E72D
:106BE800012A40F3198507EE101AB8EEC77AC7EEE6
:106BF800876AB1EEE68AB8F1030F14D0BBF1000F33
:106C080009D007EE90BAF8EEE77AB4EEE78AF1EE2B
:106C180010FA00F39686236E03EB550393FBF5F306
:106C2800E362FFF7FEB9B0EE480A22F0EBFC00B2CF
:106C3800E4E79FED0D7AF4EEC76AF1EE10FA44BF6F
:106C48009FED0A7A77EE666AFFF7D1BA1C2B00200F
:106C5800A4290020C040002054450020D040002036
:106C6800FC3F002064290020DB0FC9BFDB0F49C0AF
:106C7800B4EEE47AF1EE10FAB8BFF0EE667AFDEE03
:106C8800E77A17EE907A17EE90EAA742A8BFA646D1
:106C9800BE42C8BFB64607EE90EAF8EEE77A012A88
:106CA800C3ED007A3CF4A0AF91ED047ADDED0F7AE4
:106CB800E7EE257AB0EE647AA3EE277AB4EEE47AAA
:106CC800F1EE10FAF0EE477AB8BFF0EE667AFDEE14
:106CD800E77A17EE907A17EE90EAA742A8BFA64681
:106CE800B742B8BFB64607EE90EAF8EEE77A022A4E
:106CF800C3ED017A3CF478AF91ED087ADDED107AB6
:106D0800E7EE257AB0EE647AA3EE277AB4EEE47A59
:106D1800F1EE10FAF0EE477AB8BFF0EE667AFDEEC3
:106D2800E77A17EE907A17EE90EAA742A8BFA64630
:106D3800B742B8BFB64607EE90EAF8EEE77A032AFC
:106D4800C3ED027A3CF450AF91ED0C7ADDED117A87
:106D5800E7EE257AB0EE647AA3EE277AB4EEE47A09
:106D6800F1EE10FAF0EE477AB8BFF0EE667AFDEE73
:106D7800E77A17EE907A17EE90EAA742A8BFA646E0
:106D8800B742B8BFB64607EE90EAF8EEE77A042AAB
:106D9800C3ED037A3CF428AF91ED107ADDED127A59
:106DA800E7EE257AB0EE647AA3EE277AB4EEE47AB9
:106DB800F1EE10FAF0EE477AB8BFF0EE667AFDEE23
:106DC800E77A17EE907A17EE90EAA742A8BFA64690
:106DD800B742B8BFB64607EE90EAF8EEE77A052A5A
:106DE800C3ED047A3CF400AF91ED147ADDED137A2B
:106DF800E7EE257AB0EE647AA3EE277AB4EEE47A69
:106E0800F1EE10FAF0EE477AB8BFF0EE667AFDEED2
:106E1800E77A17EE907A17EE90EAA742A8BFA6463F
:106E2800B742B8BFB64607EE90EAF8EEE77A062A08
:106E3800C3ED057A3CF4D8AE91ED187ADDED147AFD
:106E4800E7EE257AB0EE647AA3EE277AB4EEE47A18
:106E5800F1EE10FAF0EE477AB8BFF0EE667AFDEE82
:106E6800E77A17EE907A17EE90EAA742A8BFA646EF
:106E7800B742B8BFB64607EE90EAF8EEE77A072AB7
:106E8800C3ED067A3CF4B0AE91ED1C7ADDED157ACF
:106E9800E7EE257AB0EE647AA3EE277AB4EEE47AC8
:106EA800F1EE10FAF0EE477AB8BFF0EE667AFDEE32
:106EB800E77A17EE907A17EE90EAA742A8BFA6469F
:106EC800B742B8BFB64607EE90EAF8EEE77A082A66
:106ED800C3ED077A3CF488AE91ED207ADDED167AA1
:106EE800E7EE257AB0EE647AA3EE277AB4EEE47A78
:106EF800F1EE10FAF0EE477AB8BFF0EE667AFDEEE2
:106F0800E77A17EE907A17EE90EAA742A8BFA6464E
:106F1800B742B8BFB64607EE90EAF8EEE77A092A14
:106F2800C3ED087A3CF460AE91ED247ADDED177A72
:106F3800E7EE257AB0EE647AA3EE277AB4EEE47A27
:106F4800F1EE10FAF0EE477AB8BFF0EE667AFDEE91
:106F5800E77A17EE907A17EE90EAA742A8BFA646FE
:106F6800B742B8BFB64607EE90EAF8EEE77A0A2AC3
:106F7800C3ED097A3CF438AE91ED287ADDED187A44
:106F8800E7EE257AB0EE647AA3EE277AB4EEE47AD7
:106F9800F1EE10FAF0EE477AB8BFF0EE667AFDEE41
:106FA800E77A17EE907A17EE90EAA742A8BFA646AE
:106FB800B742B8BFB64607EE90EAF8EEE77A0B2A72
:106FC800C3ED0A7A3CF410AE91ED2C7ADDED197A16
:106FD800E7EE257AB0EE647AA7EE837AB4EEE47A27
:106FE800F0EE477AF1EE10FAB8BFF0EE667AFDEEF1
:106FF800E77AFCF7EBBDFDEEE77ABDEEE67A17EE31
:1070080090EA17EE907AA64517EE106AA8BF2746B1
:107018007645C8BF374607EE907AF8EEE77A012A38
:10702800C3ED007A3CF4E0AD91ED047ADDED0F7A22
:10703800E7EE257AB0EE637AA3EE277AFDEEC77AFB
:1070480017EE90EA17EE907AA645A8BF2746B645F0
:10705800B8BF374607EE907AF8EEE77A022AC3ED12
:10706800017A3CF4C1AD91ED087ADDED107AE7EED6
:10707800257AB0EE637AA3EE277AFDEEC77A17EE8B
:1070880090EA17EE907AA645A8BF2746B645B8BF3E
:10709800374607EE907AF8EEE77A032AC3ED027ACC
:1070A8003CF4A2AD91ED0C7ADDED117AE7EE257A8C
:1070B800B0EE637AA3EE277AFDEEC77A17EE90EA70
:1070C80017EE907AA645A8BF2746B645B8BF3746FB
:1070D80007EE907AF8EEE77A042AC3ED037A3CF4D7
:1070E80083AD91ED107ADDED127AE7EE257AB0EEF8
:1070F800637AA3EE277AFDEEC77A17EE90EA17EEC9
:10710800907AA645A8BF2746B645B8BF374607EECA
:10711800907AF8EEE77A052AC3ED047A3CF464AD78
:1071280091ED147ADDED137AE7EE257AB0EE637A05
:10713800A3EE277AFDEEC77A17EE90EA17EE907A5B
:10714800A645A8BF2746B645B8BF374607EE907A8A
:10715800F8EEE77A062AC3ED057A3CF445AD91EDE1
:10716800187ADDED147AE7EE257AB0EE637AA3EEAD
:10717800277AFDEEC77A17EE90EA17EE907AA645C1
:10718800A8BF2746B645B8BF374607EE907AF8EE4F
:10719800E77A072AC3ED067A3CF426AD91ED1C7A0E
:1071A800DDED157AE7EE257AB0EE637AA3EE277A5D
:1071B800FDEEC77A17EE90EA17EE907AA645A8BFBB
:1071C8002746B645B8BF374607EE907AF8EEE77A15
:1071D800082AC3ED077A3CF407AD91ED207ADDED7E
:1071E800167AE7EE257AB0EE637AA3EE277AFDEEFB
:1071F800C77A17EE90EA17EE907AA645A8BF2746F9
:10720800B645B8BF374607EE907AF8EEE77A092A0E
:10721800C3ED087A3CF4E8AC91ED247ADDED177AF9
:10722800E7EE257AB0EE637AA3EE277AFDEEC77A09
:1072380017EE90EA17EE907AA645A8BF2746B645FE
:10724800B8BF374607EE907AF8EEE77A0A2AC3ED18
:10725800097A3CF4C9AC91ED287ADDED187AE7EEAD
:10726800257AB0EE637AA3EE277AFDEEC77A17EE99
:1072780090EA17EE907AA645A8BF2746B645B8BF4C
:10728800374607EE907AF8EEE77A0B2AC3ED0A7ACA
:107298003CF4AAAC91ED2C7ADDED197AE7EE257A6B
:1072A800E3EE273AFDEEE37AFCF790BCDC49C978B7
:1072B800002900F06A81DA48BAF91411877805982C
:1072C800A0EB010E8EEAEE70A0EBEE70B84240F330
:1072D800C58101208AF81C010598CAF8182188423E
:1072E800C8BF7F4207EE907AF8EEE77A38EE278A31
:1072F80085ED038AFCF7AFBD8223FEF7F0BCDFED16
:10730800C97AFEF7B8BC8300CF180AEB030EC64B48
:1073180003EBCC1C5FEA980300F0248301331B01C4
:1073280007930CEB030007F110010CF110030EF1A9
:10733800100213ED024A13ED035A13ED016A13ED1F
:10734800047A51ED024A51ED035A51ED016A51EDAB
:10735800047A64EE244A65EE255A66EE266A67EEDC
:10736800277A1033834242ED024A42ED035A42ED36
:10737800016A42ED047A01F1100102F11002D8D13C
:10738800079B103B0CEB0302F918734418F0030831
:107398003EF41EABB2EC017AF1EC017A67EE277A83
:1073A800B8F10108E3EC017AF4D1FEF711BB9F4A6A
:1073B8009F4BD2681B689A423EF649AF33780C3B24
:1073C800022B7DF68BAC9AF8B8313770002B3DF460
:1073D80085ACFEF7EABFDFED977AFFF72CB907EE29
:1073E800907ADFED956AB8EEE77A66EEA65A9FEDD9
:1073F800935A9FED936ADFED937AA5EE856A26EEA0
:10740800A55AE5EE867AE5EE276A26EE870AFFF7A3
:107418000BB9FDEEE67A0EA8CDED087AFDEEE47A1A
:10742800CDF82CA0884EDFF82CC2DDF820A00A93F6
:1074380017EE907AB1EE433A00EB8202CDF8248041
:107448005B46069496ED007AF0EC017AE7EE257A31
:10745800B0EE637AA3EE277AF0EE477AE3B9FDEE51
:10746800C77ABB4617EE908A474504DC069CA045C0
:10747800A8BFA046C34607EE90BAF8EEE77A0029FF
:1074880000F042829042ECEC017A06F11006D9D164
:10749800DDF82CA0FCF7ABBBBEF1000F06D0F4EE74
:1074A800474AF1EE10FAC8BFF0EE667AFDEEE77AC9
:1074B80017EE90BADA4507EE90AA05DC069CA345BC
:1074C800A8BFA34607EE90BAF8EEE77AD7E7F0EE42
:1074D800627AFBF7D1BFFDEEE47A0EA817EE907A38
:1074E800FDEEE67ACDF82CA0574EDFF868C10A9376
:1074F80017EE90AACDED087A00EB8202CDF8248031
:107508005B46069496ED007AF0EC017AE7EE257A70
:10751800B0EE647AA3EE277AF0EE477ACBB9FDEEA7
:10752800C77ABB4617EE908A474504DC069CA045FF
:10753800A8BFA046C34607EE90BAF8EEE77A00293E
:1075480000F0EE819042ECEC017A06F11006D9D1F8
:107558009EE7BEF1000F06D0F4EE474AF1EE10FAAE
:10756800C8BFF0EE667AFDEEE77AD04617EE90BA1D
:10757800DA4505DC069CA34517EE908AA8BFA0460D
:1075880007EE908AF8EEE77AD9E7254ABAF914E1C6
:107598009078059AA2EB0E0282EAE277A7EBE277EF
:1075A800874276DD02EBD27201215210CAF82821F7
:1075B8008AF82C118AF81C11DAF810217244B2F5F5
:1075C800FA6FA8BF4FF4FA62B2F57A7FB8BF4FF4EA
:1075D8007A7207EE902AB8EEE78A85ED038AFCF7FF
:1075E8003ABC06999FED197A098F07EE901AF8EEC2
:1075F800E77A174967EE877AC1ED007AFCF74EBC47
:10760800F0EE477AFDF720BDB0EE677AFDF706BDCC
:107618009FED088AFFF7C6BA9FED068AFFF7EBBA17
:107628003C2B002000000243904B002088000020E3
:10763800782B00200000000084F9223F92E741B92E
:107648009730083C15A82ABEFC3F00206F12833AE9
:1076580000000020642900200000C8429AF81C019C
:1076680028B1DAF824018AF81C21CAF82001DAF8CE
:1076780010210A44A3E71FED080AD04B0B9325EE0F
:10768800800A21F0BFFFCE4FDAF8D451F880FDF719
:107698006ABC9AF81C21002A8ED0DAF824218AF8CC
:1076A8002C118AF81C11CAF8202185E7C549C64A59
:1076B8008E46FEF77CB995ED000A0793069221F0F5
:1076C800A1FFC249DFF84CE3D1F8EC10BC4F069A91
:1076D80038808EFB013EC917C1EBAE1107EE901A38
:1076E800F8EEE77A079BFDEEE77A17EE901A7980B5
:1076F800FCF72CBC07EE905AF8EEE78ADFEDB47A77
:107708009FEDB40A8AF8B05168EEA78A38EE800A6D
:10771800FDEEC07A17EE903A2033402B40F23181CB
:107728009FEDAD0AAD4BFDEEE87A83ED010A17EE49
:10773800903A2033402B00F22181DFEDA97AF4EE54
:10774800E78AF1EE10FA40F3AC81DFEDA66ADFEDCF
:10775800A67A01E0F0EE478AF4EEE78AF1EE10FA35
:1077680038EEE67AF6DCDFEDA17AB4EEE77AF1EEF0
:1077780010FA40F193819FED9B6ADFED9D6A01E06D
:10778800B0EE677AB4EEE67AF1EE10FA77EE067AA2
:10779800F6D49FED907AF4EEC77AF1EE10FA40F342
:1077A800D5809FED8F7A77EE677A27EEA76ADFEDAF
:1077B800915ADFED916A9FED917AE6EE256A67EEC0
:1077C800865AA6EE267AE5EE877ACAED6D7AFDF737
:1077D8008BBF06F08FFB069B794F98F80020DAF8EC
:1077E800D45199F80060C01AB880FEF7F3B906F0D2
:1077F80081FB069B724F99F80060C01A7880FEF7EB
:1078080092BA06F077FB069B6D4FDAF8D881DAF862
:10781800D451C01A7880FEF765B9B0EE667AFEF7E3
:10782800C4BC774B1B6803F59C530833CAF8BC31BA
:107838003378012B7DF452AA9AF8B831002B7DF4E5
:107848004DAA032F00F0238121F076FB01238AF84B
:10785800B831FDF743BAF0EE476AFEF7BCBCDFED7E
:10786800607AF4EEE76AF1EE10FA40F34681DFED54
:107878005D5A9FED5D6A01E0F0EE676AF4EEC66A54
:10788800F1EE10FA76EEE57AF6DCDFED586AF4EE02
:10789800E67AF1EE10FA40F12D81DFED525A9FEDB4
:1078A800546A01E0F0EE667AF4EEC67AF1EE10FA68
:1078B80077EEA56AF6D4DFED477AF4EEE76AF1EEE3
:1078C80010FA04DDDFED467A77EEE66A8DE5DFED46
:1078D8004D7AF4EEE76AF1EE10FA44BFDFED437A31
:1078E80077EEE66A81E509980CF0FCFBFEF782BDAD
:1078F800454B1B78002B47D1444B1B8B07EE903A26
:10790800F8EEE77AFEF7B2BC0A9C002C7FF4BAAD19
:10791800099CA046079CA045B8BFF0EE667AB1E581
:107928000A9C002C7FF40EAE099CA046079CA0453B
:10793800B8BFF0EE667A05E6234901F1800EFEF73E
:1079480030B9F880A4F8A850FBF7B1B99FED2D7AAB
:10795800F4EEC77AF1EE10FA44BF9FED247A77EE81
:10796800677A22E77346394662460FE503F0DEFC84
:10797800AF7800283EF468ACFEF71FBDDFED167A3D
:1079880023E703F0E1FACDE6DFED137AFEF76EBCEC
:107998009AF80032002B7BF43BA8FBF724B81C4A6A
:1079A800D35C002B7EF4A1AD00233B604FF0FF3287
:1079B80004237A603370AF78FEF746BCAC720020BF
:1079C800D2420020104D00208C1B0020280E0020E1
:1079D80035FA8E3CDB0FC93F000000000000002094
:1079E800DB0F4940DB0FC940E4CB1641DB0F49C030
:1079F800E4CB16C192E741B99730083C15A82ABED6
:107A0800E84A0020DB0FC9BF544500202C45002060
:107A18008CBB0208D34D621021F0C8FB00283EF44D
:107A280064AD374BAF784FF480521A800A23337015
:107A3800FEF70ABC99F80010132920D04BB105F5C0
:107A4800F460B0EE480A2044D4F89C379847B0EE6A
:107A5800408A99F80030132B7DF48BA9B0EE480AC0
:107A680021F0D0FD7880FDF786B980201CF068FEF3
:107A780008B110F0DFFA21F05FFAFEF752BDB0EE60
:107A8800480A079321F0BEFD079B3880D6E780207F
:107A98001CF056FE00287DF421A9D5E6F0EE477AC1
:107AA80077E6B0EE687A5EE60B9BD3ED03DA154B0A
:107AB80093ED020A144B3BEEEDDA28EE000A20EEB5
:107AC8000D0A83ED020AFBF76AB99AF8F031002B28
:107AD800EAD10C4B234493ED000A059BD3ED01DA60
:107AE80028EE000A3BEEEDDA20EE0D0A8BED000AD7
:107AF800FBF755B9F0EE676ADDE6F0EE667AC4E6A4
:107B0800242B0020743A0020082900202DE9F04F8A
:107B18002DED028B8FB0064614F040FF9C4B1F786A
:107B280027B10FB0BDEC028BBDE8F08FDFF8C0B213
:107B3800DBF800305905F4D5964B974D1B78002B90
:107B480040F05C81954B1B78002B6BD0944C954A88
:107B5800D4F86C31F31A934201F2478094F8748197
:107B6800B8F1000F31D1904F386806F013FCC0B25D
:107B780001280ED9022841F0E6838C4B1A78002A96
:107B880041F0ED85D4F87821B21AB2F57A6F81F018
:107B98004C87D4F87C31002B44D094F87431BBB9AD
:107BA800834B1B689B7801211E3B00228B4284F883
:107BB800741184F8882141F237863868022104302C
:107BC80014F0F5FA94F880310FE0D4F87C314BB317
:107BD800D4F8843140F6B732F31A934222D994F894
:107BE8008031002B01F0E0826F4F013BDBB284F85B
:107BF8008031002B01F06B80D4F87C1194F8882137
:107C080011F801EB94F88931C4F87C1172440133FE
:107C1800386884F88821714684F8893106F0BEFBFB
:107C2800C4F88461634B2F681B7853B1DFF8C481B3
:107C3800D8F8000028B1604B1B78013B012B41F2BA
:107C480055805E4B1B7863B15D4F3B684BB1544C1C
:107C5800D5F80090D4F8C032A9EB0303632B00F2E7
:107C68002587584C2378022B01F07F82DFF8888122
:107C780098F80030032B01F01680534B1B7873B132
:107C8800524F3B685BB1464C06F034F9D4F8C83221
:107C9800009044F61F62C31A934200F27F814C4B56
:107CA8001B78002B4BD14B4B1B7843B13C4CD4F881
:107CB800183403F5C333A0339E4280F05787464BF0
:107CC8001B78002B3FF42DAF354E444C444D06F243
:107CD8003947206806F05EFB00283FF422AF206891
:107CE80006F050FB2B7880465A1E33B120682A7064
:107CF80006F050FB0028F2D113E703223946781E1C
:107D080023F07CFD96F8383496F8392486F83B84BD
:107D180083F47F4383F0FF039B1A1FFA88F89BB212
:107D2800B8EB132FD5D196F83A24DBB29A42D0D1CA
:107D3800781E14F04BF92B7818442870C9E7294CA1
:107D48002278002A40F0F286154CD4F8103403F556
:107D5800C333A0339E42A6D3234A94F81434C4F8FC
:107D68001064D55CE90701F1EC83AA0701F1A88347
:107D78006B0701F1B4821D4A94F814341178013369
:107D880093FBF1F201FB123384F814348BE700BF44
:107D9800D1420020E0430020E84A0020EA430020C6
:107DA800BC1D00203F0D0300B04200200800002049
:107DB800B4420020EC430020F4430020FC430020A0
:107DC800D85F00203E2500200444002008440020FD
:107DD800704400207E4400200E44002014440020FB
:107DE80018440020D8430020784400207D44002017
:107DF800504A0020584200207D0000205D4C2A682F
:107E0800D4F85C31D31A7C2B7FF69CAE94F86031A1
:107E1800DFF880919FED588AC4F85C21013384F81B
:107E280060314FF02408404614F074FA534BF9ECD3
:107E3800016A1B8A07EE103AF8EEE66AB8EEC77ACE
:107E480008F10108C6EE877A5FFA88F867EE887A43
:107E5800FDEEE77ACDED007ABDF900A05FFA8AF071
:107E680014F02EFACAF3072014F02AFAB8F1270FF3
:107E7800D9D1302014F04EFAD4F86491DFF8188183
:107E88005FFA89F014F01CFAC9F3072014F018FA05
:107E9800D8F800005E2106F081FA94F860319A075C
:107EA8002DD1D4F85C2141F288339A4201F28E85B3
:107EB800142014F02FFA324B324AB3F9043082FB03
:107EC80003124FEAE379C9EBA2090FFA89F95FFABD
:107ED80089F014F0F5F9C9F3072014F0F1F91C2022
:107EE80014F018FA002014F0EBF9002014F0E8F967
:107EF8005E21D8F8000006F051FA94F8603158076E
:107F080001F09A83282B7FF41DAE00271720D5F89F
:107F1800009084F8607114F0FDF9384614F0D0F937
:107F2800194B1A4CA3FB09239B0BA4FB0312520900
:107F3800C2EB0212A3EB8203D8B214F0C1F91820E5
:107F480014F0E8F9124BA3FB09239B09A4FB0312C5
:107F58005209C2EB0212A3EB8203D8B214F0B0F9B3
:107F6800384614F0ADF9D8F800005E2106F016FA8C
:107F7800E8E500BFBC1D002000007A44344300201F
:107F8800784300206766666673B2E7458988888803
:107F9800D34D621068430020B842002094F8CE32D6
:107FA800002B41F07981E34B1A6802F00803002B9B
:107FB80048F603414AF60B404BF60F4349F607488B
:107FC80004BF0346884612F0040F4FF0190118BF8A
:107FD8009846920684F8CE1203D548F4804848F0B3
:107FE8002008D54B1A79C8F309010191002A41F0FC
:107FF8005A855B79002B41F0D9869A4664204FF068
:10800800FF330A464FF00009CDF81880CDF81C80E0
:108018000892ADF826A0ADF828308DF83600ADF8F6
:108028002490CDF82A90CDF82E90CDF832900DF10D
:10803800180CBCE80F00DFF810E384F85190AEE8A4
:108048000F009CE80F00AEE807002EF8023B7146CF
:108058004FF0010C1B0C4FF0FE0E1F20C82201F838
:108068001E3984F84EE084F8522084F853C084F80E
:108078004F0094F8DE0284F8500080F0F10383EAA0
:108088000313DAB2130983F0E70343EA022383EA0E
:10809800C2031BB283EA0312D2B2C3F3072383EAF3
:1080A800121343EA022383EAC2031BB283F0C80215
:1080B80082EA0212D2B2C3F3072383EA121343EA15
:1080C800022383EAC2031BB283EA0C0E8EEA0E1E59
:1080D8005FFA8EFEC3F3072282EA1E1242EA0E22DC
:1080E800604482EACE0E84F8DE02A4F84CE001F186
:1080F8001F0011F8013B83EA0E0383EA0313DBB286
:108108001A0982EA1E2242EA032282EAC3031BB248
:108118001FFA83FE8142A4F84CE0EAD183F07C0385
:1081280083EA0313DBB21A0982EA1E2E8EEA032EB3
:108138008EEAC30E0FFA8EFE1FFA8EF34FEA132A49
:108148005FFA8EFEA4F84C30DFF8009284F874A031
:1081580004F16E0384F873E004F14E0C0193DCF82B
:108168000C30DCF80000DCF80410DCF80820C84605
:10817800A8E80F00019B0CF1100C9C45C146EED1FC
:10818800DCF80000C8F80000DFF8C4819CF804306F
:1081980089F8043008F1270984F82DE384F82EA320
:1081A80018F8011F386806F0F9F8C145F8D194F8B5
:1081B800CF22002A41F0758060492B6808780A218F
:1081C80084F8CF12002801F07181DFF888C10128F6
:1081D800BCF80010059141F2C185BCF8021002916B
:1081E800022801F07C84BCF804100391032801F0F4
:1081F800F485BCF806100191042801F0E8850528EB
:10820800BCF8081001F0DE850628BCF80AA001F0C9
:10821800D5850728BCF80CE001F0B985BCF80E90AC
:1082280094F8DE220693104680F0300383EA0313A5
:10823800DBB20490424A9DF810C0128884F850C0FE
:10824800180980F07A0040EA032080EAC3033D4819
:10825800C2EB022280FB02C01044D217C2EB60229C
:1082680005988DF82D204FF0000860F30F0803984B
:108278004FF0000C60F30F0C00201BB261F30F00ED
:1082880000216EF30F0183EA031EC3F30723039350
:10829800029B63F31F48019BCDF81C8063F31F4CBE
:1082A800039BCDF820C05FFA8EFE6AF31F4069F386
:1082B8001F4183EA1E134FF0000A09900A918DF8B6
:1082C8002CA043EA0E2C0DF11809B9E80F008CEA2E
:1082D800CE0E0FFA8EFE8EF0C808DFF86CC084F858
:1082E80051A088EA08185FFA88F8CEF3072EACE8A0
:1082F8000F008EEA181E4EEA082399E8030083EA65
:10830800C8080FFA88F383F023024CF8040B82EABA
:108318000210C0B2C3F3072282EA1012049B2CF8A1
:10832800141942EA0022591C82EAC0004FF02308BF
:10833800162211E0684B0020C8440020804300202A
:108348005029002003082080101E0020C42000208F
:10835800C3200020126300204FF0FE0EC82384F8CB
:10836800DE12A4F84C000CEB020184F8538084F868
:108378004EE084F84F2084F852301CF8013B43400B
:1083880083EA0313DBB21A0982EA102242EA0322C3
:1083980082EAC3031BB298B28C45A4F84C00ECD116
:1083A80083F0F40383EA0313DBB24FEA131E8EEA69
:1083B800102E8EEA032E8EEAC30EA0460FFA8EFE0A
:1083C8001FFA8EF958F84E0FDFF818C4A4F84C902D
:1083D8004FEA192A5FFA8EFE84F86AE084F86BA0E7
:1083E800D8F80410D8F80820D8F80C30ACE80F00FA
:1083F800D8F81000D8F81410D8F8182004F2253945
:10840800ACE8070004F2073884F825A384F824E3CD
:1084180018F8011F386805F0C1FFC145F8D194F874
:10842800D6E2BEF1000F40F04687E64B94F8DEC274
:10843800B3F90010B3F90220B3F904309FEDE26AF2
:1084480084F851E007EE103A2B6806938CF06A0323
:1084580083EA031306EE901AD9B20B0983F0D50309
:1084680043EA012383EAC1031BB283EA03115242A0
:10847800C9B207EE902AC3F3072383EA111343EA2C
:108488000123F8EEE77AF8EEE66AB8EEC77A83EAEF
:10849800C1031BB267EE867A66EE866A27EE067A15
:1084A800002083F0C805CDED087ACDED076A8DED83
:1084B800097A0A900B900C9085EA05150DF11809B8
:1084C800EDB2C3F30728B9E80F0088EA151848EA9F
:1084D800052888EAC505DFF810832DB2A8E80F0043
:1084E80085F01E0E99E807008EEA0E13DBB2C5F37D
:1084F800072E8EEA131E4EEA032E88E807008EEA3E
:10850800C30EA8F110051C20C8214FF005091E2331
:108518004FF0FE080CF1010284F8521084F8D6924C
:1085280084F8533084F84E8084F84F00291884F872
:1085380050C0A4F84CE084F8DE2215F8013B83EA29
:108548000E0383EA0313DBB21A0982EA1E2242EA07
:10855800032282EAC3031BB21FFA83FE8D42A4F8EA
:108568004CE0EAD183F0270383EA0313DBB21A094C
:1085780082EA1E2E8EEA032E8EEAC30E0FFA8EFEB4
:108588001FFA8EF34FEA13295FFA8EFEDFF8548242
:10859800A4F84C3084F8719084F870E004F14E0C23
:1085A80004F16E0ADCF80000DCF80410DCF808209E
:1085B800DCF80C3045460FC50CF1100CD445A84624
:1085C800F0D1824DBCF80030A8F8003005F124083D
:1085D80084F82AE384F82B9315F8011F386805F00E
:1085E800DDFE4545F8D194F8D7320293002B40F0D0
:1085F8005D86774B1B68052213F0140F84F8D72289
:1086080040F0B286DFED737A94F8DE826D4B724AE1
:10861800B3F90410B2F90620704D7148CDED087A0F
:1086280088F0220383EA03135FFA83FE4FEA1E13DE
:1086380083F05903B2F5FA6F43EA0E2383EACE03B7
:10864800A8BF4FF4FA621BB2B2F57A7F83EA031E21
:10865800B8BF4FF47A725FFA8EFE4FF0640CA2F541
:108668007A72C3F307230CFB02F283EA1E1385FB1D
:10867800025980FB0150D21743EA0E25C9174FF063
:10868800000AC2EBA912C1EBA00185EACE050DF1E3
:10869800180CADF82A20ADF82810CDF818A0CDF8A0
:1086A8001CA0CDF824A02DB285F0C80ECDF804C0CA
:1086B800BCE80F008EEA0E1E5FFA8EFEC5F3072592
:1086C80085EA1E15DFF82091DCF800C084F8508098
:1086D80045EA0E25A9E80F0085EACE0212B282F01B
:1086E8004A0383EA0313DBB2C2F3072282EA1312B6
:1086F80049F810C942EA03224A2082EAC3034FF02C
:10870800140E002508F101084FF0FE0C84F8530000
:10871800C82084F8515084F8DE82A4F84C304A46C8
:1087280009EB0E0184F84EC084F84FE084F852003B
:108738001D4612F8010B684080EA0010C0B2030918
:1087480083EA152343EA002383EAC00000B285B216
:108758008A42A4F84C50ECD180F0140080EA001052
:10876800C0B24FEA101E8EEA152E8EEA002E8EEA4F
:10877800C00E25460FFA8EFE1FFA8EF855F84E0FDA
:10878800DFF860C0A4F84C804FEA182A5FFA8EFE22
:1087980084F869A084F868E06968EB68AA68ACE8BE
:1087A8000F00286969692B8BACE8030004F20735D0
:1087B800ACF80030A84684F823A384F822E304F236
:1087C800233A13E07843002088C3E43AC32000200A
:1087D800684B00200000000012630020D34D621097
:1087E80067666666C4200020101E002018F8011F66
:1087F800386805F0D3FDC245F8D1D14BD14A1B7872
:108808001278013B12F00100DBB214BFC0224022F3
:10881800172B04D8CC490B4493F824300293CB4B44
:1088280019888B071ABF002342F01002012311F4A4
:10883800027F18BF022311F0100F18BF062311F092
:10884800200F18BF1023002841F07C80032194F8E2
:10885800DEE206938EF0460383EA0313D8B20309D7
:1088680083F0920343EA002383EAC0031BB283EA3E
:108878000310C0B2C3F3072888EA101848EA002892
:1088880088EAC0080FFA88F888F0C80C9DF8080034
:108898008DF81C008CEA0C1C00235FFA8CFC8DF808
:1088A8001E200320019A8DF81D30C8F307288DF883
:1088B8001F108DF8200088EA1C1807CA48EA0C28FF
:1088C80088EACC0C0FFA8CFC8CEA0C18A9E8030097
:1088D8005FFA88F8CCF3072181EA181141EA0821E8
:1088E80081EAC80894F854C089F800200FFA88F281
:1088F8008CEA020C8CEA0C1C5FFA8CFCC2F307228F
:1089080082EA1C1242EA0C2294F8550094F8561098
:1089180094F8579094F8588084F8533082EACC023F
:1089280012B2504080EA0010C0B2C2F3072282EAB5
:10893800101242EA002282EAC00212B2514081EAD1
:108948000111C9B2C2F3072282EA111242EA0122D6
:1089580082EAC10212B289EA020989EA09195FFAB0
:1089680089F9C2F3072282EA191242EA092282EA45
:10897800C90212B288EA020888EA08185FFA88F879
:10898800C2F3072282EA181242EA082294F859C070
:1089980094F85A0094F85B1094F85C9084F851307D
:1089A80082EAC80212B28CEA020C8CEA0C1C5FFA4A
:1089B8008CFCC2F3072282EA1C1242EA0C2282EAE9
:1089C800CC0212B2504080EA0010C0B2C2F30722B3
:1089D80082EA101242EA002282EAC00212B2514030
:1089E80081EA0111C9B2C2F3072282EA111242EAEE
:1089F800012282EAC10213B289EA030282EA021260
:108A0800D2B2C3F3072383EA121343EA022383EAA9
:108A1800C2031BB283F0320282EA0212D2B2C3F35B
:108A2800072383EA121343EA022383EAC2031BB231
:108A38009AB24FF0FE0CDFF8288184F850E0092044
:108A4800C8210EF1010EDBB284F84EC04FEA122C99
:108A580084F84F0084F8521084F8DEE2A4F84C2021
:108A680084F85EC084F85D30D8F80000D8F80410A7
:108A7800D8F80820B8F80CA008F2BA2EAEE807001B
:108A880008F2CA288EF80290AEF800A084F818C33D
:108A980084F8173315F8011F386805F07FFCA845DE
:108AA800F8D1009BC4F8C832FFF7F9B8DFF8B4A0D2
:108AB800DFF8B480412013F02DFBBAF9023088FBAF
:108AC8000320DB17C3EBA00080B213F009FBBAF94F
:108AD800003088FB0320DB17C3EBA00080B213F043
:108AE800FFFABAF9043088FB0320DB17C3EBA000B8
:108AF80080B213F0F5FA164B3868197805F04EFC79
:108B080094F8C43213F0010800F03C84114AC4F808
:108B1800C0920133DBB2A2FB0312D20802EB82023D
:108B2800A3EB420384F8C432FFF79BB80A4B0B4906
:108B3800186805F003FC00232370FFF705B900BF90
:108B4800942B0020D1560020DCBD0208EE2D002019
:108B58003C640020CDCCCCCC74440020B44300202D
:108B68000A1E0020784300206766666694F81C3465
:108B7800C74AC4F8186402EB8302D26B42B30EAD45
:108B880004F22343C34E45F8203D002104F2354347
:108B98003180079380211523A52784F8223428469D
:108BA80084F8211484F8207490472846318802F00C
:108BB800BBF8069DB84804F584616D1A152DA8BF49
:108BC80015252A4622F00FFEB44A94F81C34157075
:108BD800B34A013382FB0312A2EBE37202EB4202B7
:108BE8009B1A84F81C34FFF76AB8AE4BAE4AD4F827
:108BF80070112868128893F80BE0AC4B401A4FF4B8
:108C08007A71D7B201FB0EF1120A9F771F7588425D
:108C18004FF00007DA775A759F701F7180F0518303
:108C2800A34AA449DFF89CC212680F688868DFF875
:108C380098E2C4F86C618CFB0281D217C2EB611216
:108C4800D4F864118CFB018C8EFB07988EFB009E78
:108C5800C017C0EBAE0002F5FA724FEAE17E92B29D
:108C6800CEEB6C1CFF1701F5EA4EC7EBA8070EF117
:108C7800300E9A76120A0CF1780C4FEA2E2E30310B
:108C8800DA764FEA272802121F7783F81D8083F8C7
:108C9800200083F8212083F824C083F823E083F898
:108CA8002210FEF75BBF844F386803685B699847FA
:108CB80000283EF4E2AF3868036801219B699847B1
:108CC8000222002388F800202370FEF7D6BF94F80C
:108CD800881194F8893138684A1C013384F888214E
:108CE80084F8893105F05AFBFEF79ABF734CDFF818
:108CF800DC914FF0000A0BE01B2B00F049820D2B92
:108D080000F012824FF0010389F80130D8F8000012
:108D180005F040FB002837D0D8F8000005F032FBFA
:108D280083B27E2B2A6828D099F80120002AEDD139
:108D380094F88A110029DFD07D2B00F0098294F87D
:108D48008EE1BEF1000F04D080F02003DBB284F87E
:108D58008E214A1CD2B2092A635484F88A2100F071
:108D6800EB81082AD2D8B4F88C21134403EB1323DF
:108D780003F0FF03A4F88C31C8E784F88AA184F8CB
:108D88008BA189F801A0C1E794F88F312BB16378E2
:108D980084F88F01302B00F0658594F88B213C4BCB
:108DA800DFF82C91DFF82CC1DFF82CA14FF0010E71
:108DB800002A3EF446AF2968C91B012900F2AF8199
:108DC80094F8A482B8F1000F40F0F98194F8BC122D
:108DD80033F8110010B984F8BCE2E9E70131B0F5C5
:108DE800826F84F8BC1200F0E0801ED9B0F5E26F03
:108DF80000F0C18034D9B0F5046F00F0CA80B0F536
:108E0800116F00F02581B0F5E46FD1D12C4AD76BF2
:108E1800118A642303FB07F393FBF1F113F0ADF917
:108E2800002384F88B31FEF70CBFB0F5007F00F00B
:108E3800298153D8B0F5807F00F04781B0F5887F4D
:108E4800B6D1D9F800104907B2D5D4F864114FF457
:108E5800887013F092F9002384F88B31FEF7F1BE85
:108E6800B0F5C06F00F02181B0F5E06FA0D1144AD1
:108E7800506B118A642303FB00F34FF4E06093FB0B
:108E8800F1F113F07AF9002384F88B31FEF7D9BE9B
:108E9800DCBD02088C430020F85300200D5400204C
:108EA80056555555904200205C4200201C44002035
:108EB800B01C002060420020D4250020BC1D0020EA
:108EC800344300201F85EB51676666660800002062
:108ED800684B0020C84400209E420020B0F5047F63
:108EE80000F00381B0F5806F7FF462AF94F8BD3273
:108EF8000133DBB2032B00F2328142F2107184F8A5
:108F0800BD3201FB03F1BE4B1B88002B40F02581CD
:108F18000131BC4B1B78D807BB4B1B8848BF0431B9
:108F2800DA0748BF0A31980748BF14311A0648BF04
:108F38002831D80548BF28315A0748BF6431180777
:108F480048BFC8319A0548BF01F5C871980648BF9F
:108F580001F57A71DA0648BF01F5FA61580648BF8B
:108F680001F57A614FF4806013F007F9002384F863
:108F78008B31FEF766BEA54A976B118A642303FB03
:108F880007F393FBF1F113F0F8F884F88B81FEF7FF
:108F980058BE9F4BB3F9041001EB8101490013F04F
:108FA800ECF884F88B81FEF74CBED9F8001011F06C
:108FB80020087FF4FDAEDBF80010090600F13C84C0
:108FC8009449097B00293FF4F3AE94F8BE120329B3
:108FD80000F24486DFE801F0322819028E4B1B6844
:108FE80059799A79DB7901F1407101EB022101EBA2
:108FF8000341002384F8BE324FF4826013F0BDF8B9
:10900800002384F88B31FEF71CBE844B1A68137A50
:10901800507992781B0403EB002313444A1C84F80C
:10902800BE2203EB0161E7E77C4B1A68D37910791C
:1090380052781B0403EB00231344EFE7774B1A68BD
:109048009379D07812781B0403EB00231344E5E7E7
:109058009CF8041000293FF4ABAE9AF800100029E0
:109068003FF4A6AE6E4B1B8803EB83035B004FF403
:10907800116093FBF1F113F080F8002384F88B3131
:10908800FEF7DFBD9CF8051000293FF491AE654B53
:1090980065491B6881FB0321DB17C3EBA10113F0B2
:1090A8006CF884F88B81FEF7CCBD9CF8051000297C
:1090B8003FF47EAE5B4B4FF4C060996813F05DF8E7
:1090C800002384F88B31FEF7BCBDD9F8001048079F
:1090D8007FF56EAE554B4FF48070196813F04DF85C
:1090E800002384F88B31FEF7ACBD9CF804100029EE
:1090F8003FF45EAE9AF8000000283FF459AE454BA5
:109108005B7B002B00F01A84454B198891FBF0F12A
:1091180001EB810149004FF4047013F02EF800238D
:1091280084F88B31FEF78DBD4FF0010284F88A2157
:109138002370A4F88C11E9E5B4F88C21C2F1FF0280
:1091480093427FF4DFAD4FF0010384F88F31D9E506
:109158004FF0010384F88E31D8E50231D9E60123B6
:1091680084F8BD3242F21071CDE604F0C3FE304BF4
:109178001A6840F6B833801A984200F2EB802D4FF7
:109188003B793A2B00F0F18200232370FEF775BD7E
:10919800D8F8000005F0FEF800287FF4B3AD4FF0D2
:1091A800010384F88B31B1E5C4F87C3184F874315B
:1091B800214F13F02FF894F88031FEF716BDD4F83C
:1091C8009432DFF8789094F8BA224B4500F04A843C
:1091D800511C94F8BBE2D4F898C284F8BA1202F091
:1091E8000F028DF818200DF11902ACEB03010029CC
:1091F80040F3458506A901910DF11E0723E000BF44
:1092080012410020D1560020EE2D002034430020CA
:109218007843002090420020006900200C43002081
:109228005C4200206042002067666666B01C002031
:10923800442500202C250020B0420020501F00208B
:10924800002840F39C800133C4F8943213F8011CC1
:1092580002F8011BBA42ACEB030081EA0E0EEFD311
:1092680084F8BBE200F00585501CB84282F800E0A3
:1092780005D20EAB9A1A1B3A002122F0D9FA0199AD
:10928800322012F05FFF4FF00008002384F8A48218
:1092980084F88B31FEF7D5BC013B84F8CE32FEF75B
:1092A80086BF013A84F8CF22FFF7B9B8013B84F8AA
:1092B800D732FFF7F6BB0EF1FF3E84F8D6E2FFF790
:1092C80092B9C64A29681278C4F87011013A012A7D
:1092D8003FF6A6AC1021022299701A71A0E4C04A88
:1092E800C04B12680793A3F1240800202121D50060
:1092F80003F8240C88F8021040F11483BA490327B4
:10930800BA4B1B88580500F10A83DA0700F1E48399
:1093180003F00203B64A002B1CBF03271146B54DC4
:109328003A46284622F05FFA7B190EA80133A91E97
:1093380040F8203D00225B1A7A5588F8013013F076
:10934800EBFAFEF718BD12F055FFAB4B01221A706D
:10935800FEF71FBCA94AB2F8C63200210133A2F8B1
:10936800C6322170FEF789BCA54B9FEDA67AD3EDD6
:10937800007AF8EEE77A67EE877AFFF745B984F85E
:10938800BBE271E7994B1B88DA0515D4D80600F1C2
:10939800AE83990600F15E845A0600F19E84180790
:1093A80000F1BD84D90700F19C8413F0020F0CBFB3
:1093B8004FF004084FF00C08934B944A1B78D2786E
:1093C80003F001030AB143F002035320009312F0A3
:1093D800A1FE8F4A128802EB820202EB8202900001
:1093E80080B212F07DFE002012F07AFE894A8A4986
:1093F80012883868C2EBC212520081FB0231114454
:109408004FEAE27ACAEB612A5FFA8AFA514604F017
:10941800C5FF824B38681A78009B48EA03087F4BDF
:109428008AEA020A002183F800A004F0B7FF414647
:10943800386804F0B3FF794B784A1B78386888EAB3
:109448000303DBB21946137004F0A8FF94F8C43282
:10945800002B7FF45BAB4F2012F05CFE1BF0C0F9D1
:109468001BF0BEF91BF0BCF90121386804F096FF27
:109478006B4A6A4B92F800801B78684A386808F093
:109488000108414683F00103137004F087FF634B22
:1094980038681B7888EA0308604B414683F80080E7
:1094A80004F07CFF94F8C432FFF730BB864682464E
:1094B800014601900390029005908146FEF7B0BEE8
:1094C800484B534907930EAFA3F1210047F8200DED
:1094D8004FF0080E4FF000080A2003F822EC03F8BA
:1094E800230C03F8248C3846098801F0F7FB4D4B10
:1094F8004D491B6881FB0321DB17C3EBA1013846EB
:1095080089B201F0EBFB494BB3F806900EF0D6FA9E
:10951800069B5A1C069283F80080069B4FEA192284
:10952800591C06911A70069B5A1C069283F80090E3
:10953800069B5A1C06921870384613F0EDF9FEF790
:1095480017BCDFF8F0809FED3A8AB8F90230254A57
:10955800079207EE903AF8EEE77A0EAF67EE887A50
:10956800A2F12403FDEEE77AA2F12101002047F8D9
:10957800201D02F8240C0822CDED007A5A701E2214
:109588009A70BDF80010384601F0A8FBB8F9003011
:1095980007EE903AF8EEE77A384667EE887AFDEEFD
:1095A800E77ACDED007ABDF8001001F097FBB8F925
:1095B800043007EE903AF8EEE77A384667EE887A94
:1095C800FDEEE77ACDED007ABDF8001001F086FBDC
:1095D800384613F0A1F9FEF7C8BB00BF30300020B1
:1095E8001C2B0020B4430020F8E00208EE2D0020D8
:1095F80008E102089343002008000020BC1D002059
:10960800B01C00200AD7233CD1560020A0440020DB
:109618005C42002050290020030820803C64002080
:10962800245600206042002067666666C844002011
:1096380058A08B4178430020022012F06BFECD4BDE
:10964800CD4ADB69323382FB0329DB17C3EB691987
:109658005FFA89F012F034FEC9F3072012F030FEE9
:10966800032012F057FEC54B1B78D90740F17281D1
:109678001CF072FCC24B9FEDC37AD3ED037A67EE00
:10968800877AFCEEE77ACDED007ABDF80030002845
:1096980000F0D982DFB24FEA1329384612F010FEE3
:1096A800484612F00DFEDFF8109399F80430002BAD
:1096B80040F020820DF118094946B34812F0C4FD64
:1096C800132012F027FEBDF91870F8B212F0F8FD59
:1096D800C7F3072012F0F4FD1B2012F01BFEBDF9A2
:1096E8001A70F8B212F0ECFDC7F3072012F0E8FD8B
:1096F800232012F00FFE4E2012F0E2FD002012F09F
:10970800DFFD4946A04812F09FFD122012F002FE2C
:10971800BDF91870F8B212F0D3FDC7F3072012F0A4
:10972800CFFD1A2012F0F6FDBDF91A70F8B212F04A
:10973800C7FDC7F3072012F0C3FD222012F0EAFD8F
:10974800452012F0BDFD002012F0BAFD5E21D8F8C8
:10975800000004F023FE94F86031FEF7D3BBC4F890
:10976800786183F80080FEF714BABB78DBB103F1A7
:10977800FF3C5FFA8CFC0CF1010CBC44BE46002295
:109788001EF8013B534083EA0313DBB2120AD900E7
:1097980042EA0322F44581EA131382EA0302EFD175
:1097A800002A7FF4F1AC794BDFF810C2D3F800E05F
:1097B800774B78491B68DEF83080774ACCF8383028
:1097C800764B0988CCF81810CCF868001168B3F803
:1097D800C6029268CCF82810CCF84820CCF858007B
:1097E800B8F1000F00F08F82D8F80430DEF840108E
:1097F8008B423BBFDEF80C205B1A5B1A9B18002BD0
:109808007EF434AADEF80030DFF8B4819B69704634
:10981800022198470423F87888F8003008F05EFFA2
:1098280003232370FEF724BA0221386804F0A6FD4A
:1098380094F88031FEF7D9B910230422184606A9F6
:109848008DF81A808DF81B808DF81C808DF81D808E
:109858008DF818308DF8192012F074FC84F88B817B
:10986800FEF7EFB9A3785A09012A40F0CA8103F03C
:109878000F0C13F0100300F0D681DFF84881E3786D
:1098880094F804E0A4F8B20208EB03018EEA03009E
:1098980084F890214346C4F8A882C4F8AC12A8F111
:1098A800070284F8B802A4F8B0E294F8B802DFF826
:1098B800188186460CE012F8011BC4F8A80242453C
:1098C80081EA0E0E197007D2D4F8AC12D4F8A83277
:1098D800994203F10100EED1424584F8B8E200F064
:1098E8006182127894F8B8329A4200F0CE812C4BFB
:1098F800C4F8943200220133B4F8B012C4F8983294
:1099080084F8902101234FF6F672A4F89C1284F88B
:10991800943184F8A432A4F89E22FFF73EBA0327B4
:109928002049FCE4DBF800301F4A204903F4800397
:10993800834216BF114604270327E1E4154B198813
:10994800FFF7E6BB1A49C97800290CBF0421052195
:10995800FEF77DBFDFF86090164BB9F80670A3FBE1
:109968000737BF08F8B212F0ABFC380A12F0A8FCAF
:109978009BE600BF302900201F85EB51D1560020FF
:10998800A0420020CDCC4C3E80969800D4250020E3
:10999800B01C00205C42002060420020BC1D00205A
:1099A800501F0020FCE00208F8E00208F0E002087E
:1099B800A0440020CDCCCCCCC84400200C00002012
:1099C8007D000020C81D0020C41D0020DFF884A3EE
:1099D800102012F09FFCD54ADAF8003082FB0329E8
:1099E800DB17C3EB69195FFA89F012F069FCC9F358
:1099F800072012F065FC212012F08CFCDAF8002018
:109A0800CA4B83FB023AD3176421C3EB6A1301FBE9
:109A18001323002BD8BF5B421BB2D8B212F050FC04
:109A2800002012F04DFCFEF743BA012238681A7084
:109A380004F0A8FC8046386804F0A4FC18F07F0FF6
:109A48007EF4A7A88E287EF4A4A894F87431002B7D
:109A58007EF4BBA8B64BC4F87C312D2384F8803142
:109A6800FEF79EB8B4F99E12D4F898C294F89CE216
:109A7800501C02F00F0242F010020029B8BF42F059
:109A880020028DF81820ACEB090282EA0E0E5FFA6C
:109A98008EFE8DF8192084F8BA0284F8BBE20DF125
:109AA8001A02FFF7A2BBA3495A790B8803EB830379
:109AB80003EB83034FEA830A1FFA8AFA002A00F0AD
:109AC80032819D4B1B681BB202930DF0F7FF029B7E
:109AD800019A40B2FEF796BA984904271FE49646C1
:109AE80092461146019203929146FEF799BB4FF0B8
:109AF800340861E4DFF860A29AF80020002A3FF4F5
:109B0800D9ADB4F868718B4B00921B883F01642172
:109B1800BFB201FB03235100B3FBF1F347EA03276C
:109B2800BFB2C3F303231F43062012F0F3FBF8B2BE
:109B380012F0C6FB380A12F0C3FBB4F868317D4A4C
:109B48007F491788009A01339BB293FBF2F002FB1E
:109B58001033487AA4F86831012800F00E814B7B55
:109B68006E2202FB07F7152297FBF2F7002B40F055
:109B7800FE803A2012F0CEFBBFB24FF0640AB7FB6A
:109B8800FAF293B2D8B20192009312F099FB009BBB
:109B9800180A12F095FB3B2012F0BCFB019A0AFB55
:109BA800127080B20A23053090FBF3F0C0B212F0B5
:109BB80087FB002012F084FBDFF87CA1282012F03C
:109BC800A9FB0A23DAF8007097FBF3F7F8B212F052
:109BD80077FBC7F3072012F073FB042012F09AFBFF
:109BE800B9F80630002B40F08680DAF8087087F361
:109BF8001007F8B212F064FBC7F3072012F060FBFD
:109C080058E5504B504AC4F89432591C012384F843
:109C1800900184F89401C4F89812C4F89C2284F83E
:109C2800A432FFF7BAB894F89021002A3FF4B5A8F7
:109C380094F8B922013202F00F02624555D084F837
:109C48009031FFF7AAB8DBF80020D2067FF522ADE5
:109C5800814622E54FF02408FFF7AEBB4B1CDBB270
:109C6800042B84F8BE324FEA01617FF4C5A9FFF7DF
:109C7800C0B90199322012F065FAFFF706BB06ABAE
:109C880001930DF11E07FFF7EFBA304BD4F8A82265
:109C9800C4F8AC224FF0000E03F52272114603F50A
:109CA800C479C4F8982203F527707246C4F8A8321C
:109CB800C4F89CE2C4F8949284F890E1F6F760FA4C
:109CC800013067D0D4F89432C4F898320123C4F82C
:109CD800949284F8A432FFF760B84FF01008FFF7A9
:109CE8006BBB4FF00808FFF767BBD4F8AC12D4F889
:109CF800A832174AD9E50DF0E1FE12F0E1FA00208A
:109D080012F0DEFAD6E4DEF81C10DEF820309942B4
:109D18003BBFDEF80C205218CB1AD31A6FE54FF070
:109D28002008FFF749BB4FF0FF33CCE61F85EB5106
:109D38001C4400205C4200206042002000E1020830
:109D480090420020501F00200000F6FFC81D002090
:109D5800BF1D0020B01C00209E420020964692465F
:109D680011460192039202929146FEF759BABFB288
:109D78009AF8003097FBF3F7FBE6392012F0CAFA9D
:109D8800F8B212F09DFA380A12F09AFA14E79146DE
:109D9800FEF746BAD4F894320222591CC4F8941239
:109DA8001A708FE784F8B9C2FEF7F7BF0E4B9246D8
:109DB800B3F9003064200A46FEF724B99646914666
:109DC800FEF72EBA964692469146FEF729BA96466F
:109DD800924611469146FEF723BA96469246114698
:109DE80001929146FEF71CBA60420020002870B527
:109DF8001EDB0928044620DD012303EB83035B00F7
:109E0800B0FBF3F2092AF8D87BB10E4EB4FBF3F09D
:109E18000928CCBF57223022A6FB03E5024403FBE6
:109E28001044EB0801F8012BF0D100230B7070BD32
:109E38002D230B7040420131DBE7303001F8010B74
:109E4800F3E700BFCDCCCCCC884230B44FF001044E
:109E58002ED301FB04F4B0FBF4F58D42F9D284B1A2
:109E6800AAB901E0B0FBF4F5092DCCBF5722302286
:109E78002A4404FB150003F8012BB4FBF1F4002C71
:109E8800F0D100221A7030BC7047B0FBF4F5092DF0
:109E9800CCBF372230222A4404FB150003F8012BDB
:109EA800B4FBF1F4002CF0D100221A7030BC7047DA
:109EB8000546002AEBD1D7E703685A1C02601970DF
:109EC800704700BF2DE9F047089C2578002B804695
:109ED80089460CBF4FF0200A4FF0300A661C35B394
:109EE800002A29DD334601E0024698B113F8011B28
:109EF800501E0029F8D1971E60B13D46013D5146DC
:109F08004046C8476B1C002BF8DC257827EAE77029
:109F1800013055B1041B29464046C847301916F888
:109F2800015B002DF7D1BDE8F087BDE8F087002A76
:109F380004DC2846BDE8F0870020EBE7571EDCE785
:109F48000A44914251D030B441F2210411F8013B46
:109F580080EA0320430010F4004F84EA03059BB213
:109F6800ADB208BF1D466B0015F4004F84EA03002C
:109F78009BB280B208BF1846430010F4004F84EA31
:109F880003059BB2ADB208BF1D466B0015F4004F28
:109F980084EA03009BB280B208BF1846430010F45D
:109FA800004F84EA03059BB2ADB208BF1D466B00A3
:109FB80015F4004F84EA03009BB280B208BF18462C
:109FC800430010F4004F84EA03059BB2ADB208BF0A
:109FD8001D466B0084EA030015F4004F85B298B261
:109FE80018BF28468A42B1D130BC7047836842689E
:109FF800D0ED037A00EB83010133934281ED040A2B
:10A00800836004BF0023836000EB830393ED047A2D
:10A01800036870EE277A9A42C0ED037A77EEC77A22
:10A02800C0ED037A0CDA013307EE103AF8EEC76A8E
:10A03800B7EE007A87EEA60A036030EE070A70478B
:10A0480007EE102AB8EEC77A87EE870A704700BF76
:10A0580090ED097A90ED004AD0ED0A6AD0ED014AF8
:10A06800D0ED047A90ED035AD0ED025AA4EE007AAE
:10A07800B0EE406AB0EE470AB0EE667AA6EE247AF1
:10A0880067EEC07AA0EE457AE6EE257A80ED097A89
:10A09800C0ED0A7A704700BFD0ED057A90ED013A1D
:10A0A800D0ED003AD0ED064A90ED024A90ED077ADD
:10A0B80090ED035A90ED086AD0ED045AC0ED067A87
:10A0C800F0EE406A27EE830AC0ED056AA3EEA60A01
:10A0D80080ED087AA4EE240AA5EE470AA5EEC60A82
:10A0E80080ED070A704700BFD0ED007A90ED017A45
:10A0F80030EE670AE7EE007AB0EE670AC0ED007A44
:10A10800704700BF704700BF2DE9F041364F374D0B
:10A11800B7F80AC02A883B89B7F91240B7F914E0A2
:10A128006E68B7F90250B7F90E80A2EB0C0203FB78
:10A1380002F3DA139644E30293FBFEF31344A3F508
:10A148007A6E0EFB0EF4B7F90CC0FB6122130EFBFE
:10A1580005F5B7F9044002FB08F8ED1202FB0CF212
:10A16800B7F900C00EFB04F405EBE825B7F920E0C9
:10A17800FF88121402EB643205EB8C0505FA0EF524
:10A188000232023592104CF25034A6EBA50502F5C6
:10A19800004244FA0EF404FB05F407FB02F2D20B6A
:10A1A800002CB9BFB4FBF2F252006400B4FBF2F227
:10A1B800141204FB04F50E4E40F6DE3404FB05F4DD
:10A1C80003EB830306FB02F524145B0004EB254430
:10A1D800083304F6CF641B1102EB241200B10260AD
:10A1E80001B10B60BDE8F08128560020F82100205D
:10A1F80043E3FFFF50F8043C012280F8352014386F
:10A2080003B11847704700BF037F33B1012B03D157
:10A218004FF400630382704770474FF480630382F2
:10A22800704700BF90F8493013B1002280F84920E8
:10A238001846704770B5044682B01830256D94F8FA
:10A248005C106B460622A847A8B19DF804009DF84B
:10A2580000609DF801109DF802509DF803209DF8BC
:10A26800053041EA062143EA002342EA0522A18497
:10A27800E2842385012002B070BD00BF70B504469A
:10A2880082B00830256A6B4606223B21A847A8B150
:10A298009DF804009DF800609DF801109DF802509B
:10A2A8009DF803209DF8053041EA062143EA002382
:10A2B80042EA05226182A282E382012002B070BDD7
:10A2C80030B490E81200057B43690222AA404A6034
:10A2D8002268586A996A4FF6FE752A4088422260B9
:10A2E80004D1012283F8442030BC70479C695A6B22
:10A2F8000C44D4600DD818690024411A51609C623E
:10A308001168002041F0010183F8440030BC11605D
:10A318007047411A51609862F2E700BF70B4046850
:10A32800037B2268022101FA03F31A4213D042691F
:10A338000A49582000FB02124FF6FE7650685289EF
:10A34800C5680068296831402960C168D24392B263
:10A358000A40C260636070BC704700BF5845002067
:10A3680030B4094B1C7864B1084B002503EBC404D6
:10A378001A6899885562D06808330143A342D160AE
:10A38800F6D130BC704700BF784900207C490020D6
:10A39800F0B4334C00EB800004EB80046468002CBC
:10A3A8005BD0304E49004FF42040CDB23060A169F7
:10A3B800090444D460682C4F45F08071384041F45A
:10A3C800903101434FF420406160306003E0411E4A
:10A3D800002838D00846A1698F07F8D54FF42040E7
:10A3E800A262306002E0421E68B31046A2691106FC
:10A3F800F9D562681C4945F0007545F480350A4076
:10A4080015434FF420406560306002E0421ED0B131
:10A418001046A2699207F9D5A362A3694FF42040B8
:10A428009B06306005D4431E68B11846A3699B0695
:10A43800F9D520233060E3610120F0BC7047411E4C
:10A4480008B10846B3E7094A138801339BB24FF0B5
:10A45800FF3131601380F0BC70472046F0BC704774
:10A468009C730020C4730020009800FCC87300206F
:10A47800134600200A4668218AE72DE9F341056959
:10A4880006460F467DBBD0F80080C8F30A0323B305
:10A498000023D6F80080019313F064FE042819D134
:10A4A800214C236943F001032361BBB2A8F80030B3
:10A4B80013F058FE04282ED108F102030193019BE2
:10A4C8003F0C1F8013F04EFE2369042823F001037C
:10A4D800236125D06FF0010505E013F043FE042841
:10A4E80005D04FF0FF35284602B0BDE8F0810E4C8C
:10A4F800236943F002032361C4F81480236943F0FD
:10A508004003236113F02EFE2369042823F002037D
:10A518002361BDD0E5E7236923F001032361D9E76F
:10A52800336804333360DEE700200240F8B50446A0
:10A538000D468E180027B54201D12069F8BDE368A1
:10A54800591CE160234415F8012B1A720429F2D131
:10A55800A1682046FFF791FFE7602061EBE700BFA5
:10A56800014B186803F01ABF0073002038B5054680
:10A5780000BF064C206804F02DFD28461CF034F876
:10A58800206804F02DFD00BF38BD00BFD43900207D
:10A5980010B582B001AB0322F62177201DF048FCEC
:10A5A8009DF80530084A9DF804409DF80600B2F968
:10A5B800202006491B0243EA04430343C2F1080270
:10A5C800D3404B6002B010BD28560020F82100206F
:10A5D80000B583B001AB0222F62177201DF028FCDC
:10A5E8009DF804109DF80530034A43EA01231380BF
:10A5F80003B05DF804FB00BFF821002068201DF0BF
:10A6080017BC00BF70B5044690F84D00002833D140
:10A6180004F11805636D80226B2128469847642051
:10A6280003F00EFD636D284603226B219847636D86
:10A6380094F848201921284698470F2003F000FD78
:10A64800636D94F8462028461A219847636D28467A
:10A6580018221B219847636D284618221C21984709
:10A66800636D28460222372198472846636D0122E8
:10A678003821BDE87040184704F05AF8054604F040
:10A68800D9FC01460028C3D1D5B12023E871AB71AC
:10A69800284604F0E3FA21460F4B41F8143F2846B8
:10A6A80014F0AEFAAB88B3FA83F3C3F11F035A1C54
:10A6B800AED001229A4009490B6813430B60A7E703
:10A6C800294604F0CBFA2146034B41F8143F2846AB
:10A6D80014F096FA0122EEE7FDA1000800040140FB
:10A6E800F0B5064683B00D460024012714E003297F
:10A6F8000CBF03220122C3F3011E6946C3F3810381
:10A7080030468DF805208DF806E08DF8073017F0F3
:10A71800C7FD0134102C0FD02B8807FA04F213421E
:10A72800F7D0AB78E9780092022903F003028DF89C
:10A738000420DCD10A46DEE703B0F0BD437A5A1C98
:10A748000344D2B242729972037A934200D802B992
:10A75800704710B504460368406804F10A01984739
:10A768000023637210BD00BF10B40B49002301E041
:10A77800272B0CD011F8132082424FEA430403F12F
:10A788000103F5D121445DF8044B48787047002057
:10A798005DF8044B704700BF24BE020870B54488BA
:10A7A80006460D46C4F30B0422460021284621F034
:10A7B8003FF83369094A934209D3094A934206D2BA
:10A7C800224628461946BDE8704021F00CB823B14E
:10A7D80021462846BDE87040184770BDD4100308CC
:10A7E8007A110308064B07498B4202D30023184607
:10A7F80070471A88C2F30B029042F8D01433F3E77B
:10A80800D80C0308D4100308024A136823EA00008E
:10A81800106070476C2B0020F8B51A4D2B789F2BD1
:10A828002ED16B78BE2B2BD105221749A81C21F0FD
:10A838004AF828BB072229464FF6FF70FFF780FB2E
:10A84800124FEC1D22884AB1A618BE4218D2052A1A
:10A8580016D92146FFF774FB3446F3E72146022256
:10A86800FFF76EFB0222A118FFF76AFB0634084BBC
:10A87800641B1C8041F60F53C31A58425841F8BD57
:10A888000020F8BD00F003080CE1020800000408ED
:10A89800323000202DE9F04FDFF854914F4F8DB042
:10A8A8000326A7EB090718220DEB0200002120F070
:10A8B800BFFF4B4BCDF8189007971A69120604D5BD
:10A8C800484A5A6002F188325A6001228DF82C20D9
:10A8D8003422DA60444B454C18689A8804909B7976
:10A8E800ADF8142004A9072206A88DF81630FFF742
:10A8F8001DFE072204A94FF6FF70FFF721FBDFF8C2
:10A90800F4B080464FF0000A5C4536D30CAC002505
:10A9180024F82C5D0222214606A8FFF707FE022232
:10A9280021464046FFF70CFB40BAC043ADF808008B
:10A93800022202A906A8FFF7F9FD099860B108AB41
:10A94800C0F104022946184420F072FF089906A8AD
:10A95800FFF793FD09950A909DF82C300A9A23B1C8
:10A968001F490B6943F080030B61013E2DD0002A7B
:10A9780099D1FFF751FF50B32CE065888DF80DA0F1
:10A98800C5F30B05AA1DADF808202288C2F30B01F8
:10A99800120BADF80A108DF80C2002A9062206A8A1
:10A9A800FFF7C4FD062202A94046FFF7C9FA61680D
:10A9B80080462A4606A8FFF7B9FD616840462A4640
:10A9C800FFF7BEFA143480469EE7002AD1D005204E
:10A9D80003F03AF80DB0BDE8F08F00BF000004089E
:10A9E800002002402301674572BE0208D80C030804
:10A9F80000F00308D41003080378202B024600F166
:10AA08000100F9D0092BF7D02D2B2CD02B2B03BF0D
:10AA18005378B7EE000A0246B7EE000AA3F13001F8
:10AA2800C8B209289FED467A10D8F2EE046A07EEFC
:10AA3800901AF8EEE77A12F8013FE7EE267AA3F1CA
:10AA48003001C8B20928B0EE677AF0D92E2B4CD065
:10AA580003F0DF03452B0BD0F7EE007A67EE276A89
:10AA680020EE260A70475378BFEE000A0246D5E763
:10AA780010B451782D2959D02B290ABF9178501C30
:10AA8800901C0024A1F13003092B53D8002303EBB9
:10AA9800830301EB430310F8011FA1F13002092AD7
:10AAA800A3F13003F3D9B3F59A7F28BF4FF49A7313
:10AAB800072B42D9DFED236A1A46F7EE007A083AE7
:10AAC800072A67EEA67AFAD803F007032BB1F2EE4D
:10AAD800046A013B67EEA67AFBD124B3C7EE276A66
:10AAE8005DF8044B20EE260A70475378A3F1300135
:10AAF800C8B2092802F10102AAD8F2EE046AF0EEFF
:10AB0800665A07EE901AF8EEE77A12F8013F87EED8
:10AB1800A66AA3F13001C8B2092866EEA56A37EE25
:10AB2800067AEED994E767EE276AD9E7901C917800
:10AB38000124A7E7F7EE007ACFE7F7EE007AC5E73A
:10AB48000000000020BCBE4CB5EEC00ADFED317A33
:10AB5800F1EE10FACCBF30EE270A30EE670ADFEDCF
:10AB68002E7A20EE270A30B5FDEEC07A87B017EEB0
:10AB7800904A054684EAE470002303A9A0EBE47038
:10AB880001930093029319F0C9FB002CACBF20235A
:10AB98002D2303A88DF800301DF0D4FC012803A94B
:10ABA80024D002282DD0032805BF302368466846E4
:10ABB8008DF8013020F062FE68461DF0C3FC0338B2
:10ABC800C4B222466946284620F0B6FE00232B551B
:10ABD80028461DF0B7FC2E22431C2A540DEB040115
:10ABE800E81820F068FE284607B030BD30236846D4
:10ABF8008DF801308DF802308DF8033020F03EFEDC
:10AC0800DAE7302368468DF801308DF8023020F0FD
:10AC180035FED1E76F12033A00007A442DE9F0417E
:10AC2800064615460846B6FBF2F43CB905FB146423
:10AC3800124B1B5D00F8013BBDE8F081B4FBF2F755
:10AC480067B90E4B05FB174705FB1464DA5D00F87E
:10AC5800012B1B5D00F8013BBDE8F081B7FBF2F862
:10AC6800B8F1000F02D04046FFF7D8FF05FB18786F
:10AC7800024B13F8082000F8012BE3E714E102085F
:10AC880030B402681146531C036011F8024B01608E
:10AC9800D31C517803609378151D05601B0443EAA3
:10ACA8000123D078234343EA006030BC704700BFDB
:10ACB8000368591C1A46016012F8021B0260587892
:10ACC80041EA0020704700BF38B5044600681546C1
:10ACD80020F089FD22682A44226038BD036810B438
:10ACE8000A0A5C1C04601A7003685A1C0260197016
:10ACF8005DF8044B704700BF03685A1C026010B42B
:10AD0800197003680A0A5C1C04601A7003680A0C4C
:10AD18005C1C04601A700368090E5A1C02601970E2
:10AD28005DF8044B704700BF03685A1C0260197035
:10AD38000368090A5A1C0260197070472DE9F04728
:10AD4800002488B080460F461E46A14605AD531C18
:10AD58000393117839B3252933D1931CCDF810907A
:10AD68000393507830284ED04FF0000AA0F13003FA
:10AD7800DBB2092B42D96C2819D0642800F09380E3
:10AD880024D825281CD063D9582876D063281BD10D
:10AD980031784046B847039A531C03931178043618
:10ADA80001340029D7D1204608B0BDE8F087039BBD
:10ADB8005A1C03921B78642B7CD02AD8252B54D19B
:10ADC800252140460134B847039AC0E7732833D099
:10ADD80044D975284FD106F1040E30682B4600225D
:10ADE8000A217646FFF730F8049A0095534639460B
:10ADF8004046FFF767F8039A0444A8E704AA03A9A2
:10AE080013F0ACFBB7E7D31C039390784FF0010A1B
:10AE1800ACE7732B10D05BD9752B3AD0782B96D131
:10AE2800A3F15802B2FA82F2306852092B46102177
:10AE38000436FFF709F8D7E73368049A00933946D0
:10AE480000234046FFF73EF804360444039A7EE7A1
:10AE58000028B9D1204608B0BDE8F0876E28B3D1E4
:10AE6800039A336804361C6071E72AD9582BD7D067
:10AE7800632B8DD06BE77828A6D1A0F15802B2FADF
:10AE880082F2306852092B461021FEF7DDFF0436A6
:10AE9800AAE706F1040E30682B4600220A217646FE
:10AEA800FEF7D2FFA0E7331D306829461E46FEF79D
:10AEB8009DFF99E7331D306829461E46FEF796FF29
:10AEC80092E7002B7FF443AF204608B0BDE8F08737
:10AED8006E2BC6D03BE700BF0EB400B584B005ABFF
:10AEE800019053F8042B0649039301A8FFF726FFA6
:10AEF800019B00221A7004B05DF804EB03B07047A0
:10AF0800C19E00080FB430B583B006AB0B490C489E
:10AF180053F8042B096800680193FFF70FFF094CE9
:10AF28000546206803685B6998470028F9D02846D9
:10AF380003B0BDE8304004B0704700BF643900205A
:10AF48006839002000730020DFED2B7AB4EEE70AA1
:10AF5800F1EE10FA4ADDDFED296A9FED297A01E06A
:10AF6800B0EE670AB4EEC70AF1EE10FA70EE667A30
:10AF7800F6DC9FED247AF4EEC77AF1EE10FA38D5B4
:10AF8800DFED1E6A9FED207A01E0F0EE407AF4EEE4
:10AF9800C77AF1EE10FA37EEA60AF6D4DFED1B7A7F
:10AFA800B4EEE70AF1EE10FA14DDDFED137A37EEAE
:10AFB800C00A60EE006A9FED166A9FED167ADFED13
:10AFC800167AA6EE867A20EE266AE6EE877AA6EE4E
:10AFD800270A7047DFED117AB4EEE70AF1EE10FAAE
:10AFE80044BFDFED087A37EEC00AE2E7F0EE407AB8
:10AFF800BFE7B0EE670AD1E7DB0F4940DB0FC94076
:10B00800E4CB1641DB0F49C0E4CB16C1DB0FC93FC7
:10B0180092E741B99730083C15A82ABEDB0FC9BF93
:10B0280041404A0011F0800F82F0D503D2B2DBB262
:10B0380008BF1346590013F0800F81F0D502C9B23A
:10B04800D2B208BF0A46510012F0800F81F0D50332
:10B05800C9B2DBB208BF0B46590013F0800F81F06C
:10B06800D502C9B2D2B208BF0A46510012F0800F09
:10B0780081F0D503C9B2DBB208BF0B46590013F003
:10B08800800F81F0D502C9B2D2B208BF0A4651007A
:10B0980012F0800F81F0D503C9B2DBB208BF0B46AE
:10B0A8005A0082F0D50013F0800FD2B2C0B208BFA8
:10B0B8001046704780EAE073A3EBE0738B4205DB30
:10B0C800002801DD401A704702D170470020704700
:10B0D8000844704709B909E0194690FBF1F301FBF0
:10B0E80013030846002BF7D1084670470146FBE7D3
:10B0F80010B507EE901A2DED028BB8EE678ADFEDDA
:10B10800227A28EE008A044628EE278AB0EE480AFA
:10B118001EF0C4FAF0EE408AB0EE480A1EF020FA9B
:10B12800F7EE007A9FED197AF0EE675AE8EE875A43
:10B138000023A361B0EE676AC7EEA56A6361236264
:10B14800E361A3626362A8EEC76ABDEC028B77EE87
:10B15800C07AB6EE007AF8EE005A27EE877A20EE2B
:10B16800250A27EE267A26EE266A67EEA67A20EECC
:10B17800260A84ED046AC4ED017A84ED007A84ED30
:10B18800027A84ED030A10BD27D4D236F304353F82
:10B1980010B44C09012250F8243001F01F0102FAC2
:10B1A80001F10B4340F824305DF8044B704700BFB1
:10B1B8004B0901F01F0150F82320012303FA01F184
:10B1C800114214BF18460020704700BF074A084BB9
:10B1D80010781B78074A834296BFC31AC3F18003CD
:10B1E8000020126818441044704700BF2042002015
:10B1F8009D410020782B0020064A074B10781B78C9
:10B2080083428ABFC3F18003C01AC018C0F17F000F
:10B21800704700BF204200209D41002010B582B039
:10B2280000249F2332208DF804308DF805408DF8D6
:10B2380006408DF8074002F003FF8DF8014000BF7B
:10B24800334C206803F0C6FE01A968461BF050F98C
:10B25800206803F0C5FE00BF9DF802309DF801008C
:10B268009DF803102B4A1B0243EA00430B43934209
:10B2780046D01ADD284A93423AD02FDD274A934216
:10B288002FD00132934222D1254B4FF480721A807D
:10B298005A809A881988234C120202FB01F1012076
:10B2A8009A60D960207202B010BD1F4A934218D02C
:10B2B80001329342E8D0A2F51A42033A934206D1EA
:10B2C800174B20214FF4807219805A80E1E7144B04
:10B2D8000020188058809860D860E4E7023A9342CA
:10B2E800F5D10F4B80214FF4807219805A80D0E736
:10B2F8000B4B4FF400714FF4807219805A80C8E7E5
:10B30800074B40214FF4807219805A80C1E700BF73
:10B31800D43900201620C2001920C2001740EF00BF
:10B3280088000020F821002017BA200030B5124C00
:10B33800237A83B01BB90120237203B030BD0522E4
:10B3480000238DF800208DF8013000BF0B4D2868D0
:10B3580003F040FE694601A81BF008F9286803F0CD
:10B368003FFE00BF9DF8053003F0010383F00100A4
:10B37800237203B030BD00BFF8210020D43900206B
:10B3880070B5064C0646256803E023685B1BB3428C
:10B3980003D8FFF7CBFF0028F7D070BDE84A00209C
:10B3A8002DE9F04F89B0B2F10008019003910293A2
:10B3B80040F39E800B46002201EB880153F8040BF2
:10B3C8008B420244FAD1029B0592002B00F0888040
:10B3D800059B002B5DD04B4BDDF814B01B685FFA62
:10B3E80083FA0AEB0B02B2F5807F474AD2688CBF1A
:10B3F800CAF5807ADA469A425DD9190C1A0A4FF0D2
:10B40800020406208DF81F308DF81E208DF81D10BF
:10B418008DF81C40FFF7B4FF0620FFF7A7F83B4A5A
:10B428000123137200BF3A4B186803F0D3FD07A934
:10B4380000201BF05DF80024039D019E5746A1469D
:10B448002968A30000200A46013459B1B94224D220
:10B45800316813F031FF2A68336813443360BF1A28
:10B46800C5F80090A04505F1040506F10406E7D1EA
:10B47800274B186803F0B4FD00BF224B214A1B6814
:10B4880053441360029AABEB0A0B0AB3BBF1000FEB
:10B49800A5D1059809B0BDE8F08F019C04933A4600
:10B4A800E15813F009FF049B2A68E1583944D71B77
:10B4B800E1502F60DCE705981649174AA0EB0B000E
:10B4C8000590059800230B70137009B0BDE8F08F44
:10B4D800059BA3EB0B030593059809B0BDE8F08F16
:10B4E800FFF724FF00287FF473AF029B0593D0E792
:10B4F800029C1CB9FFF71AFF0594CAE700230593BD
:10B50800C7E700BF782B002088000020F821002022
:10B51800D4390020204200209D41002070B5104DF4
:10B52800104E2B7831788B4284B016D00E4A039295
:10B538001A4402928CBF0C46CA1A04A98CBFC3F1E4
:10B5480080020024012341F8102D02A80222019450
:10B55800FFF726FF002333702B7004B070BD00BFC7
:10B568009D41002020420020A041002070B5194CC8
:10B57800194D23782978994284B027D0174A039225
:10B588001A44029234BF0E46CA1A04A934BFC3F142
:10B5980080020026002341F8102D02A802220196FD
:10B5A800FFF7FEFE23781844C0B203062B7848BF85
:10B5B80080F080008342207002D0002004B070BD6B
:10B5C800002301202B70237004B070BD012004B04B
:10B5D80070BD00BF9D41002020420020A0410020F6
:10B5E80008B545F20820FFF7CBFE0620FEF7BEFFA0
:10B5F800064B0122C7201A72FEF7B8FF0448054916
:10B60800054A002303700B70136008BDF821002061
:10B61800204200209D410020782B00202DE9F04198
:10B6280082B00346060C050A032406208DF807306D
:10B63800884617468DF805608DF806508DF8044049
:10B64800FFF79EFE90B100BF0A4C206803F0C2FCD1
:10B6580001A900201AF04CFF3A460021404613F099
:10B668002BFE206803F0BCFC00BF384602B0BDE8E2
:10B67800F08100BFD4390020F0B5124BDD6885B0E9
:10B688000DB905B0F0BDED0A14D0002704AE7C1941
:10B698006410E00210226946FFF7C0FF0F2809DD99
:10B6A8006B4653F8042B01320AD1B342F9D125462F
:10B6B800AF42ECDBFFF732FF034BED021D60E0E722
:10B6C800671CF5E788000020782B0020B0F1FF3FC9
:10B6D8000AD0022810B403DC5DF8044BFEF758BE0C
:10B6E80000205DF8044B704700207047054B93F825
:10B6F80020309B01343303F0FC03F422772100202F
:10B70800E4E700BF285600202E23F42277210020EA
:10B71800DCE700BFF0B5574B574A97B0196891421C
:10B7280000AF00F09C805549554A00234FF4700043
:10B73800C1F888003B607B60136843F48033136072
:10B7480003E03B68B3F5A04F09D0136803F4003356
:10B758007B603B6801333B607B68002BF1D0484B32
:10B768001B6813F4003318BF01237B607B68012B2F
:10B778004BD0424D424B434AEA60434A596A1160F2
:10B788005A6A424E42F080725A625A6907F1580466
:10B7980042F4FC0241F6FF715A6124F8501D03235C
:10B7A80021464FF09040BB72FEF79AFF4FF6FF73A9
:10B7B800214637483B81FEF793FF21463548FEF77F
:10B7C8008FFF21463448FEF78BFF21463348FEF7AA
:10B7D80087FF21463248FEF783FF204616F06CFBB0
:10B7E800BB683049304AA1FB031330499B0CF02455
:10B7F80000204FF0070E5C370B60566085F8234039
:10B808009060C2F800E0BD46F0BD294A1C4B1221E9
:10B8180011605A685A605A685A605A6842F48062DD
:10B828005A605A6822F47C125A605A6842F4E81244
:10B838005A601A6842F080721A601A689201FCD540
:10B8480059680F4A21F003015960596841F0020113
:10B858005960536803F00C03082BFAD189E70022DA
:10B868001A6062B6134B1B6883F30888124B1B6877
:10B878009847FEE7FC9F0020EFBEADDE00ED00E03C
:10B88800001002400005FA054C4A00203F1901004B
:10B898000004004800080048000C00480010004858
:10B8A8000014004883DE1B4310E000E0EC4A00204F
:10B8B8000020024000D8FF1F04D8FF1F2DE9F04FD9
:10B8C800714C54F8205083B0002D00F09A80D5F8C0
:10B8D80054901F46D9F804302B65A9604FF4807343
:10B8E80005F15A019046064605F5AD72674828608D
:10B8F8006961AA61EB602B6199F818001CF094F853
:10B90800D9F80C40F4B16248002103465A689442C1
:10B9180003F11C0303D001310C29F7D10021C1EB3D
:10B92800C10100EB81015B480B6942694FF00C0EC5
:10B938001A43731C426181F818E04B762B6D2C6317
:10B948002433EB64D9F80810002936D05048002475
:10B9580003465A68914203F11C0303D001340C2CAE
:10B96800F7D10024C4EBC40400EB8401494B0A69F5
:10B978005869494C104358610B200876701C48766A
:10B988005869024399F81B005A618309002291F80B
:10B998000DE08DF805304D6101238C6001A88DF80C
:10B9A80006208DF807308DF804E012F071FE2B6D3B
:10B9B800D9F808206A632833AB6495F8590002F077
:10B9C800B7FE044695F8580002F0B2FE3A078246E0
:10B9D80099F819B019D5C4B117F0110F4FF00B032E
:10B9E80006F1010614BF4E213E21A371E6715A46A5
:10B9F800204602F061FFFB0741D52B6B4BB36B6B05
:10BA08003BB3284603B0BDE8F08F17F0010F0CBF19
:10BA18002E274E2718F0020F09D044B10B22731CB1
:10BA2800A271E37120465A46394602F045FF18F0E4
:10BA3800010FE2D0BAF1000FDFD001360C238AF8EB
:10BA480007605A4639468AF80630504602F034FFF5
:10BA5800D3E799F81A308DF8043099F81C30002192
:10BA68009B09012201A88DF805308DF806108DF884
:10BA7800072012F00DFE284603B0BDE8F08F2046DF
:10BA880003F0A8FAB9E700BF703900207CBE0208AD
:10BA98005818002000100240C9A200080348D0F836
:10BAA8003C3113B100F59A701847704758180020B8
:10BAB8000348D0F8203113B100F58C70184770474F
:10BAC800581800200348D0F804310BB1FC3018474F
:10BAD800704700BF581800200348D0F8E8300BB171
:10BAE800E0301847704700BF581800200348D0F8C6
:10BAF800CC300BB1C4301847704700BF581800202D
:10BB08000348D0F8B0300BB1A8301847704700BFD1
:10BB1800581800200348D0F894300BB18C301847DF
:10BB2800704700BF581800200248836F0BB170306F
:10BB380018477047581800200248C36D0BB154309D
:10BB480018477047581800200248036C0BB138306A
:10BB580018477047581800200248436A0BB11C3038
:10BB680018477047581800200248836803B11847DF
:10BB7800704700BF581800201749184B184A194831
:10BB880010B4D1F8884044F47004C1F888401C68A7
:10BB980044F001041C605C6822405A601A6822F074
:10BBA800847222F480321A601A6822F480221A60A1
:10BBB8005A6822F4FE025A60DA6A22F00F02DA6248
:10BBC8001A6B002410404FF0006218639C608A6072
:10BBD8005DF8044B704700BF00ED00E00010024024
:10BBE8000CC07FF8CCFC00FF2DE9F04FB74AB849EC
:10BBF800137895B00446089000F59C4020300A90D0
:10BC08000860002B00F08883B24909688C4240F232
:10BC1800D681B1490391D1F80080B04CB049DFF822
:10BC280000B30291013B137008F480530793002B73
:10BC380040F0D481AB4B05931D7805F00105029BBC
:10BC48005B7D002B40F0DB8118F4004F40F09585B8
:10BC580018F4807F0BD0089AA34BDFF8C8A29A4249
:10BC68009AF8022000F29C87002A40F09D87BBF9D1
:10BC780006909E4E18F4805740F03783029B5B8BEA
:10BC88009945B4BF4FF000094FF00109984B1B6864
:10BC980013F0805300F0D381002D00F0D481029975
:10BCA800944A898C92ED037A07EE901AF8EEE77AB7
:10BCB800B4EEE77AF1EE10FA80F25686B9F1000F89
:10BCC80040F0C88194F8A420002A40F0C3818A4A31
:10BCD8008A49106890F8300000220A604A608A6039
:10BCE800002840F0B781864A1070002D40F0B881D6
:10BCF80096F800E0029ABBF900C0508B918BBBF913
:10BD080002208445CCBF8025002545F040038C45A2
:10BD1800A8BF2B469B0843F080058242C8BF2B462C
:10BD280043F040058A42B4BF2A461A469208BBF936
:10BD380004C0BBF9065042F080038445C8BF1A46C8
:10BD480042F040038C45A8BF13469B0843F080028D
:10BD58008542D4BF1846104640F0400294F8A630F9
:10BD68008D42ACBF05461546AB4200F0588400230F
:10BD780084F8A65084F8A730BEF1000F00F084853F
:10BD8800039B604A1B68049203F00403002B40F0F5
:10BD9800688312AF5C4D00237B6005F15009129354
:10BDA80040F6330A4FF0190840F2833602E00435B2
:10BDB8004D4520D0AA78EB789A4218FB0261F6D25A
:10BDC8006A78043218FB03633BF912205245A8BF76
:10BDD8005246B2F5617FB8BF4FF461728A42E6DD20
:10BDE8009A42E4DC29782329E1D838460435FFF75C
:10BDF800CFF94D45DED1454B97E803001E783C4B03
:10BE080083E80300002E00F0978301213848FFF7EC
:10BE1800CFF9002840F07081039B1B68D80500F11A
:10BE280066813B4F32483C8824F00104A4B20221C9
:10BE38003C80FFF7BDF9002800F06781A20740F1B8
:10BE4800AA85DFF8E4A0334B9AF8001002935868EB
:10BE5800A30708BF81F00201C1F3400103F0C6F84F
:10BE6800049B1B6813F00A0F40F054813C8820485B
:10BE78000C21FFF79DF9002800F07181264B1B78F3
:10BE880044F48074082B3C8000F072810E2B00F083
:10BE98006F81039B1B685D0577D5204B1B79002BB1
:10BEA80000F00A8114211248FFF782F9002840F0B7
:10BEB800088110F073FD012019F096FA002864D06B
:10BEC800DFF8688000244FF0CC0934E07456002075
:10BED8003855002070560020504A00204C2200207F
:10BEE800204A0020D1560020404B4C005618002014
:10BEF8001C2B0020A04200200C4300201429002005
:10BF08008C1D0020684B0020982B0020D142002077
:10BF1800EE2D0020D84A0020942B002090420020CB
:10BF280012630020A0440020D44A0020DC5F0020D7
:10BF3800DCB2022C29D809FB04F6631C58F8065019
:10BF4800002DF5D1C3788C4A90F9020052F82330BD
:10BF580001950322009201212A4618F0B7FE0346F4
:10BF680004EB440000EB0010039353B1294608EB9F
:10BF78008000CC221FF05CFC039B48F8063001349B
:10BF8800E4B21AF00FFD0028D3D1059B1B78DC071B
:10BF980040F11E8179497A4A01230B701370029B84
:10BFA8009AF80010186801F0010103F01FF8049BCB
:10BFB8001B685A0700F17C8115B0BDE8F08F714B02
:10BFC8000393D3F80080704B029308F480536F4CAE
:10BFD800DFF8F8B10793002B3FF42CAE00216C4832
:10BFE800FFF7E6F86B4B002800F0F9861D780593FB
:10BFF800029B5B7D05F00105002B3FF425AE029AFC
:10C00800013BD27D3BF91330002A40F05984A3F557
:10C018007A73B3F57A7FA8BF4FF47A7323EAE37390
:10C0280007EE903A9FED5C7AF8EEE77A67EE877A4A
:10C038005A4AFCEEE77A17EE903A138008E618F4AD
:10C04800800F7FF429AE002284F8A420B9F1000FF4
:10C058003FF43DAE524A01211170002D3FF448AE25
:10C0680018F0100F3FF444AE4E4A1278D2063FF54E
:10C078003FAE002F7FF43CAE002B7FF439AE18F4AE
:10C08800800F7FF435AE96F800E0BEF1000F01F0A6
:10C09800C182454B9B78B9F1000F41F0DC823BB17E
:10C0A800424A434B12681B689B1A002BC1F2BC82A0
:10C0B800012384F8A5301DE6059B1B78D8077FF57A
:10C0C800F8AE3C2018F03CFB00283FF45EAF0BF0C4
:10C0D800B1FF3C2018F0E0FA00283FF456AF0BF00F
:10C0E800A9FF3C2018F0D8FA0028F0D14DE7314BD1
:10C0F800DB78002B3FF495AE049B1B6899077FF50E
:10C1080090AE2D4F3C8844F0010424F00204A4B200
:10C118003C8096E606211E48FFF74AF83C8800282E
:10C1280000F08A83660640F11D8607211848FFF74C
:10C138003FF800283FF49BAE204B214AB3F9043066
:10C1480020493C8882FB0302DB17C3EBA2030B8068
:10C158000F480C21FFF72CF800287FF48FAE1A4BFC
:10C168001B7824F48074A4B2082B3C807FF48EAE34
:10C1780024F040043C808CE6DCD50208D25600202E
:10C18800D01C0020504A0020204A00204C220020C9
:10C198001C2B0020D1560020AAF1823F50290020F4
:10C1A8008C1D002024560020682B0020E84A00201F
:10C1B80008570020A0440020EE2D002078430020DE
:10C1C80067666666941C0020942B0020126300208A
:10C1D800B54B93F80090B9F1000F5FD1DFF84483B5
:10C1E800B24E18F8030C35784146A8F1030419F04B
:10C1F8005DFE002800F06982002D40F0BB8204F14A
:10C208000801607919F052FE002841F00B81A84915
:10C21800A07A19F04BFE002800F06A82022D41F046
:10C228000581A449E07B19F041FE002841F0028114
:10C23800A149207D19F03AFE002800F06A82042DF9
:10C2480041F0FC809D49607E19F030FE002841F0E5
:10C25800F9809B49A07F19F029FE002800F06A8226
:10C26800062D41F0F380974994F8230019F01EFE3B
:10C27800002840F0A486944994F8280019F016FE86
:10C28800002800F06A82082D40F083868F4994F8D0
:10C298002D0019F00BFE002840F06A828C4B012219
:10C2A8001A701AF086F8049B1B685A077FF584AE4B
:10C2B800032019F025FE002800F0BC853B8813F008
:10C2C80008047FF479AE082019F050F98148824DAE
:10C2D8008249834A834BBBF8066000682E80086059
:10C2E80014601C6015B0BDE8F08F1D217E48FEF774
:10C2F8005FFF00287FF4C2AC7C4A029BD2881B8B6C
:10C30800991A894540F31C8613449945B4BF4FF0E8
:10C3180000094FF00109B9E4754C764B2678029371
:10C32800754F002E00F00A83B6B1DFF8FC91DFF8F4
:10C33800FCB1DFF8C481CA460025072D4046E9B2A2
:10C348007B6841F33981984700B20135AE422BF83A
:10C35800020F0AF1040AF0D1684B03931A46684B9E
:10C36800D2F80080089AA3FB023E42F2010318EAC1
:10C3780003034FEA9E1E059300F0EB826148624A70
:10C38800624B00786249049012781A70049B087016
:10C398002BB15E4B93F800B08BF0010304935D4A18
:10C3A800029912785C4B0E9210463A7891F822C0A6
:10C3B8000692A3FB00A30A46C98C09915B081146A3
:10C3C80003EB4303128D0C92C31A0A8B2578119242
:10C3D800DBB294F829200F920CF1040C0F220B9376
:10C3E8004E4EDFF84CB1DFF84C910998CDF84080FB
:10C3F80008F480535FFA8CFCDDF83C8084F8282030
:10C40800AA460D92079300210F97099435B9069B08
:10C418009C458DBF1D46E2466546AA46A94280F264
:10C428002F83049B002B00F00C833D4B33F9112024
:10C4380097B287424FEA410303D30C9CA74240F2CC
:10C44800D88259F82120964580F004833BF90320CF
:10C45800059F002F40F0D5822BF8032001310636C6
:10C46800D4E794F8AB3053B1059B1B78D80706D5B1
:10C47800029BBBF906205B8B9A4200F3728511215F
:10C488001948FEF795FE002800F0208294F8AE3097
:10C498002BB994F8A93013B93223A4F8AC3001238E
:10C4A80084F8AE3075E400BFD25600200A000020A0
:10C4B800373100203C310020413100204631002036
:10C4C8004B31002050310020553100205A310020D6
:10C4D800D01C0020B01C0020A01C0020AC1C002098
:10C4E800A41C00209C1C00201C2B0020C440002001
:10C4F8004C220020204A002080430020504A00207F
:10C50800D34D621014550020A4110020A51100205D
:10C51800C444002085250020ABAAAAAA78220020BE
:10C52800502200202D310020F02500204E2200202E
:10C538001263002088250020DFF84893C14F09F1D5
:10C548005A054FF00108494619F8010C19F0AEFCDC
:10C55800F8B199F8040099F8023099F803E000EB73
:10C56800400104EB8101013BD1F8B42003EB430304
:10C578003B4493420DD094F8E02081F8B0E008FAEB
:10C5880000F022EA0000C1F8B430C1F8B86084F8BD
:10C59800E00009F10609A945D5D1AB4AAB4BAC4936
:10C5A800D2F800901B780968AA4D0691C846002663
:10C5B800A1464FF0010A1C466B684BB31F783FB386
:10C5C800A968A8EB010100290ADB99F8E0100AFA2A
:10C5D80006F021EA000108F5FA7089F8E010A86071
:10C5E800B4B1297858780431C9B2002840F0C18123
:10C5F800029A3BF91110108B00F1C80E714540F3F7
:10C60800778499F8E0109B783141C90740F17B8421
:10C618000136042E05F10C05CED1FFF7F6BB94F8D0
:10C62800A780B8F1F90F00F2988108F101085FFAC4
:10C6380088F884F8A78084F8A650BEF1000F00F0AF
:10C648002481B8F1140F7FF49BAB5F2D40F030814B
:10C6580005990B7813F0010200F0B8867E4A9278AB
:10C6680003F0FE030B70002A40F05187039B1B6800
:10C678005B0700F1A1813378002B40F0A2810021F3
:10C68800BB2D129100F03B87B72D00F01B87BE2D04
:10C6980000F03887BD2D00F08C87792D00F07A875F
:10C6A8007A2D00F070879E2D00F066879D2D00F092
:10C6B8005B87AE2D00F07587AD2D7FF461ABFF2150
:10C6C800002015F046FEFFF75BBB08F10501607915
:10C6D80019F0ECFB00283FF49AAD012D40F0A2863A
:10C6E80004F10D01A07A19F0E1FB002840F09E86C4
:10C6F8005A49E07B19F0DAFB00283FF499AD032D85
:10C7080040F098865649207D19F0D0FB002840F06B
:10C7180095865449607E19F0C9FB00283FF499AD0D
:10C72800052D40F08F865049A07F19F0BFFB0028E7
:10C7380040F08C864D4994F8230019F0B7FB002887
:10C748003FF499AD072D40F03A84494994F8280000
:10C7580019F0ACFB002840F01C84464994F82D00E1
:10C7680019F0A4FB00283FF499AD092D3FF496ADCC
:10C778004FF009094B4600F00FBCD4F88C30089AEA
:10C78800D31A002BFFF664AA3B4A94F89030517CE8
:10C798003A4A029E32F811200A98B17DC4F88C00FA
:10C7A800013303F00F0384F89030234492B292FBD4
:10C7B800F1F283F8942094F8940094F8951094F882
:10C7C800962094F8973001440A4494F8980094F815
:10C7D80099101344184494F89A2094F89B30014413
:10C7E8000A4494F89C0094F89D101344184494F853
:10C7F8009E2094F89F3001440A4494F8A00094F8CD
:10C80800A1101344184494F8A23094F8A3200144CA
:10C818000B441A4442F30B12642AF17DA8BF642228
:10C8280013B209B1C2F1640307EE903A9FED147A8E
:10C83800F8EEE77AFFF7FABB24F04004A4B23C8094
:10C8480073E400BFA4BE0208E84A0020C4440020E4
:10C8580000690020FC220020CF2700203C31002066
:10C8680041310020463100204B310020503100205A
:10C87800553100205A31002078730020947300202D
:10C8880014AE234145300020F0460021B548FEF79C
:10C898008FFC68B3002384F8A83016F0CFFD94F815
:10C8A800A730142B7FF46CAA3378002B40F0C7868E
:10C8B800059B1B7803F00103002B7FF461AA22E09B
:10C8C800C3F53B6308331BB2FFF7A1BB94F8A9304B
:10C8D800002B3FF45EAA059B1B7813F001037FF43D
:10C8E80058AA012284F8A93084F8AA20FFF751BA7F
:10C8F800059B9D4A1B781060DF0700F1DB84B8F1C7
:10C90800140F7FF43DAA94F8A650572D00F0F08438
:10C91800039B1B6813F0040342D05A2D40D194F8AE
:10C92800A920002A40F06C8694F8AB208F49049126
:10C9380082F0010284F8AB20FFF728BA93F822307E
:10C948003E780433DBB2B3428EBF267023701E4696
:10C95800EAE4874B1B7804931AE584F8A630BEF105
:10C96800000F92D0FFF70CBA012284F8A420FFF739
:10C9780071BB012800F0D68499F8E0100AFA06F392
:10C9880001360B43042E89F8E03005F10C057FF4DD
:10C9980013AEFFF73ABA44F002043C80FFF751BAED
:10C9A8005D2D00F0FE845B2D00F0E9825E2D00F025
:10C9B8001185562D00F05E8533782BB16F2D00F070
:10C9C8005585694B00221A60972D00F04385A72DE5
:10C9D8007FF455AE6749039B0A781B6842F004024E
:10C9E8000A70624A049203F00403FFF7CFB90246C3
:10C9F8004B000EF5967749F82170059F002F3FF4FC
:10CA08002BAD0B9C5F182744099C04EB4707BA859C
:10CA1800B8F1000F03D10E9C022C7FF61DADB6F8BD
:10CA280002803288B78842441744534A3FB282FB97
:10CA38000742524CA2EBE772E75212B24FF00108DC
:10CA48000AE50028D3D059F8212096454FEA41033A
:10CA5800FFF4FCAC4A4A4A4CD25CE718002A00F0C2
:10CA68008681022A40F071817A7802EB820202EB19
:10CA7800820202F2EE2292B2032969DD12B2E7E4E1
:10CA88000D99099C3F4B0F9F84F800A042460F293F
:10CA980084F829200CBF01220022DDF8408084F8A8
:10CAA80028101A7006D11B212E48FEF781FB00289A
:10CAB80000F069843448354A354B11688268C16092
:10CAC8008A1A012119704368324E9A42029A3170CB
:10CAD80088BF002392F8226088BF80F82130079B26
:10CAE8003878B2F826C0B2F818E00436F6B2002B4F
:10CAF80000F049818642224A40F2D881264E1746E4
:10CB080000210DB982460546A94218DA12F81130FB
:10CB180083B1022B0CD17B7803EB830303EB8303F4
:10CB280003F2EE239BB226F8023B01310237E8E715
:10CB38003388F8E7CBB2032BFAD87346F3E784F8C7
:10CB480000A00E9B154A01331370079BFFF76FB8BF
:10CB5800012404FA01F70D9C24EA070412B20D948B
:10CB680076E400BF1C2B00200C570020684B0020E7
:10CB7800C44400202456002056555555C022002094
:10CB880024260020C5440020A0440020E84A0020B4
:10CB9800A4110020A5110020126300208525002083
:10CBA80012B901228AF802201B2019F0A9F99AF873
:10CBB80021309AF82020B44EB44FDFF8E882049070
:10CBC8009946052A00F2AC80DFE802F092865118F7
:10CBD800283C19F0C1F9012800F0FF83049B002BC1
:10CBE8006ED0AB4B1B79002B6AD00DF00FFC0322E3
:10CBF8004FF47A738AF82020CAF81C303B8843F037
:10CC080002033B8016F0BAF8D8F80020DAF81C3096
:10CC180013440422CAF818308AF82020B9F1010F09
:10CC280040F0C283D8F80030DAF818209A4277D258
:10CC3800307818B919F064F9002871D13B8823F0CD
:10CC480002033B80924BD8F80020DB88642101FB6B
:10CC580003234FF4806000228AF820208AF80320FA
:10CC6800CAF8103018F07AFC9AF82020A9E7B9F130
:10CC7800010F04BF05238AF82030002D5BD0029BEA
:10CC8800D8F800E0B3F91810814B002261F30F02C5
:10CC980061F31F42B3F90200CBF800200023DAF851
:10CCA800142061F30F0360F31F439645CBF804305B
:10CCB80043D8B9F1010F40F0E2849AF8202080E7C8
:10CCC800B9F1010F2CD0D8F80030DAF810209A42C8
:10CCD8003ED301238AF82030B9F1010FB2D06C4B52
:10CCE8001B7A012B34D00DF091FB9AF8202068E7CD
:10CCF800002D7FF46EAF049B4FF48060002B6BD047
:10CD080018F034FC059BBBF906901D78039B0022A4
:10CD1800D3F80080CAF8102005F00105FEF7AABF75
:10CD2800059BBBF906901D78039B05F00105D3F818
:10CD38000080FEF79FBFD8F8003047F23052032337
:10CD4800CAF81C208AF8203058E73BF8032093E6FD
:10CD58000DF05CFB032240F6B8338AF82020CAF8AD
:10CD68001C304BE744F040043C80FFF7DEB9CAB200
:10CD7800022A40F29C82032AE7D1119A079C002CD0
:10CD880008BF024678E686421946424A57D84248C2
:10CD980017460DB9B24635468D427FF7D0AE12F828
:10CDA800113083B1022B0CD17B7803EB830303EBA7
:10CDB800830303F2EE239BB220F8023B01310237D2
:10CDC800E7E70388F8E7CBB2022B03D9032BF8D1A6
:10CDD8006346F1E77346EFE718F0C0FB92E71946A0
:10CDE80005931B7813F001053EF429AF2B4A95787B
:10CDF80003F0FE030B70002D3EF421AF284F3A7864
:10CE08000B2A0DD80121914040F603050D4040F052
:10CE18007B8311F4C06F03D0093A012A40F2518490
:10CE2800204A214912684A600B2203F001053A7032
:10CE3800FEF705BF082018F091FBFFF7BDB8164EA6
:10CE480017460DB982460546A942BFF678AE12F8D4
:10CE5800113083B1022B0CD17B7803EB830303EBF6
:10CE6800830303F2EE239BB226F8023B013102371B
:10CE7800E7E73388F8E7CBB2022B03D9032BF8D1C5
:10CE88006346F1E77346EFE7561800201241002089
:10CE9800DC4000202426002012630020CF27002039
:10CEA800CE270020E84A00202C2B0020B348174644
:10CEB80000210DB9B24635468D427FF740AE12F8D3
:10CEC800113083B1022B0CD17B7803EB830303EB86
:10CED800830303F2EE239BB220F8023B01310237B1
:10CEE800E7E70388F8E7CBB2032BFAD87346F3E7F2
:10CEF800C838814228DA99F8E0109B783141CA078E
:10CF08003FF586AB5B42791E162900F29680DFE872
:10CF180011F0820196016B01D300AA01BB015801EF
:10CF2800450120010B01F6009400D300E300BB018A
:10CF380058014501BF00AB00970084006E005A00FD
:10CF48004FF00109FEF7A2BE99F8E0300AFA06F19F
:10CF580023EA010308F5FA7189F8E030A960FFF7C0
:10CF680057BB00218648FEF723F900287FF487AADB
:10CF7800322384F8AB00A4F8AC30FFF780BA814ABA
:10CF880001218148814D0260814A29700492FEF78F
:10CF9800FDBE4FF008094B4603EB83031C4486F89B
:10CFA8000090A178607806F095FC059B794A1B787B
:10CFB80001211170D9077FF574A9FEF7F0BF4FF072
:10CFC80007094B46E8E7D9F8E400734A90F83A10A5
:10CFD800977819446429A8BF642121EAE17180F88F
:10CFE8003A10002F40F05B830CF014F8C4E4D9F831
:10CFF800E400694A90F83B1097781944FE29A8BFC5
:10D00800FE2121EAE17180F83B10002FECD01620B8
:10D0180018F0D4FFD9F8E400E6E7069841781944F7
:10D02800B1F5967FA8BF4FF4967121EAE1715A4B8A
:10D0380041709B78002B40F02C83D9F8E400D3E7AB
:10D04800D9F8E40081781944C829A8BFC82121EA81
:10D05800E171514B81709B78002BC5D0142018F0DA
:10D06800ADFFD9F8E400BFE7D9F8E40041781944E6
:10D07800C829A8BFC82121EAE171474B41709B78B4
:10D08800002BB1D0132018F099FFD9F8E400ABE7D2
:10D09800D9F8E40001781944C829A8BFC82121EAB1
:10D0A800E1713D4B01709B78002B9DD0122018F048
:10D0B80085FFD9F8E40097E7069A37489179807890
:10D0C80019446429A8BF642121EAE17191710028FB
:10D0D80040F0F1820D2FB0D0069F2F4A79799078D1
:10D0E80019446429A8BF642121EAE17179710028F3
:10D0F800A3D00E2018F062FFD9F8E40074E7D9F83D
:10D10800E400254A017A97781944C829A8BFC8219C
:10D1180021EAE1710172002F3FF466AF0B2018F08D
:10D128004DFFD9F8E4005FE7D9F8E4001A4AC1795D
:10D1380097781944C829A8BFC82121EAE171C171AB
:10D14800002F3FF451AF0A2018F038FFD9F8E40057
:10D158004AE7D9F8E400104A817997781944C82930
:10D16800A8BFC82121EAE1718171002F3FF43CAFCB
:10D17800092018F023FFD9F8E40035E712630020EE
:10D188001C2B0020A42600200C430020F442002081
:10D19800684B0020D01C0020CF270020D9F8E400DD
:10D1A800BA4A417992781944C829A8BFC82121EA06
:10D1B800E1714171002A40F07682112F7FF442AF6D
:10D1C80012E7D9F8E400B14A017992781944C829DC
:10D1D800A8BFC82121EAE1710171002A40F0338219
:10D1E800102F7FF443AFFFE606990F791F44642F91
:10D1F800A8BF642727EAE7770F7118F0F9FEA34B59
:10D208009B78002B3FF419AF0320394618F0D6FE5F
:10D21800D9F8E400E8E6069801781944FA29A8BF85
:10D22800FA2121EAE171994B01709B78002B3FF4B8
:10D2380004AF012018F0C2FED9F8E400D4E606983D
:10D24800817819446429A8BF642121EAE1718F4BD0
:10D2580081709B78002B3FF4F0AE022018F0AEFEF0
:10D26800D9F8E400C0E6069F884AF979907819440D
:10D2780081F30801F97100283FF4DFAE052018F0AA
:10D288009DFED9F8E400AFE6D9F8E4007F4AC178FA
:10D2980092781944C829A8BFC82121EAE171C17050
:10D2A800002A40F021820F2F7FF4F4AE9CE6119AF9
:10D2B800FFF7E2BB764B1B78002B3EF461AD754B54
:10D2C800DB78002B7EF45CAD94F8A8300133DBB238
:10D2D800032B84F8A8307EF653AD6F4B5B781BB9EF
:10D2E800B9F1000F7EF44CAD15F048FDFFF7D7BA41
:10D2F8006A4A6B4B049210461A686A494FF47A736B
:10D30800B3FBF2F3C3EB431203EB82030268DB00C7
:10D318005507A1F8A8307CD4039B1B6803F00403CD
:10D32800FEF734BD3BF91110987840F63303994263
:10D33800A8BF1946B1F5617FB8BF4FF461710C2FD2
:10D34800A1F561714FF4966393FBF0F391FBF3F150
:10D358004ED0182F7FF410ABD9F8E430C9B2C829E1
:10D3680093F817E00846A8BFC82086453FF404ABE9
:10D37800464AD8759278002A3FF4FEAA384618F033
:10D388001DFEFFF7F9BA484A42491368CA688B601C
:10D398009B1AC82B7FF6D5AB012381F82130FFF704
:10D3A800D0BB424A0021ECE5059BD8F80010DAF81A
:10D3B8001C201D78039BBBF90690D3F800800A4413
:10D3C800CAF8182005F00105FEF754BC84F8A72018
:10D3D800FFF79EBA364A0221D3E5364BD8F800202B
:10D3E800DB88642101FB0323CAF81030FFF7F6BB82
:10D3F800314B5B78C9B28B423FF4BEAA084607910D
:10D4080016F030F9214B07999B78002B3FF4B4AA0A
:10D41800B4E7039B294A1B680A21118003F004031F
:10D42800FEF7B4BC4FF001094B46B5E54FF00209D1
:10D438004B46B1E54FF003094B46ADE54FF0040903
:10D448004B46A9E54FF005094B46A5E54FF00609FF
:10D458004B46A1E5039B1A4A1B684FF4C87111801B
:10D468000E4A049203F00403FEF790BC15F0E6FFA1
:10D47800FEF786BC14F030FAFDF70CFA14F014FA33
:10D4880002F0AEF994F8A650FFF796BACF2700201D
:10D49800C4440020A0440020682B0020684B0020D2
:10D4A800AC720020886A0020E84A00205A26002032
:10D4B800EE260020DC400020F44200201C690020F9
:10D4C8001E6900200B464FF6FE718B4A8B48558922
:10D4D800049090892B4401445381918114F0FCF904
:10D4E800FDF7D8F914F0E0F902F07AF9039B1B680C
:10D4F800002203F0040384F8A720FEF747BC0B467C
:10D508000221E2E70223E0E70546FEF798BB7C4FDD
:10D518003A780B2A1BD80121914040F6030911EAF9
:10D5280009097FF4A3A811F4C06F10D0093A012AA1
:10D538000DD845200DF0A2FDFF200DF09FFD71488C
:10D548000DF00EFD48460DF099FD059B1B786E49C0
:10D558006E4A0968516003F001030B223A70002BF0
:10D568007EF40EACFFF7CFB90021FF2014F0F1FED6
:10D5780094F8A650FFF79DB8012014F0EAFE94F83D
:10D58800A650FFF793B8624A137A43F00103137267
:10D59800FEF7F6BB5E4A137A23F001031372FEF717
:10D5A800EFBB0121002014F0D4FE94F8A650FFF739
:10D5B80083B84FF6FE7388E7029A515D9847032DAA
:10D5C8001BDC40F2EE2240F6CA0C00283EF4BDAE49
:10D5D80039F825E0BAF802104FF47A73A0EB0E0080
:10D5E80003FB00F0A1EB0E0190FBF1F01844904210
:10D5F800B8BF10466045A8BF604600B2FEF7A5BE9A
:10D608000122002184F8AA203C4A84F8A910049237
:10D61800FEF7BCBBB9F1000F3EF44AAD94F8A52063
:10D628004AB99E46FEF766BB15F0A8FB002384F8AE
:10D63800A530FEF75DBB84F8A570FEF75BBB94F8D8
:10D64800A650FFF702B81020079318F0B7FCD9F8D6
:10D65800E400079BC4E53BB12B492E4A09684FF407
:10D668007A7000FB0313136094F8A530002B3EF486
:10D6780041AB00229E4684F8A520FEF73BBB059BE4
:10D688001D78039B8146D3F8008005F00105FEF75D
:10D69800F1BA152018F092FCD9F8E400A4E4172098
:10D6A80018F08CFCC9E41120079318F087FCD9F80E
:10D6B800E400079B81E50D20079318F07FFC079B8A
:10D6C80008E545200DF0DAFCFF200DF0D7FC0D48E9
:10D6D8000DF046FC28460DF0D1FC039BD3F80080E2
:10D6E800059B1B78FFF79CBB0F20079318F066FC7F
:10D6F800D9F8E400079BD6E5442B0020684B0020AE
:10D70800CE27002008E00208E84A00202C2B002041
:10D718008444002008570020436A826970B4D154B9
:10D72800436A0469426B0133A34228BF0023436262
:10D73800DAB1116811F0010101D070BC7047856A37
:10D7480086699D422E44D6600BD3641B5460816267
:10D758001368002143F0010380F8441070BC136083
:10D7680070475D1B55608362F2E7026D136843F0F2
:10D7780080031360E1E700BF026B10B462B1036C71
:10D78800C2684469D11A013B615C5DF8044B08BF6B
:10D7980013460364C8B27047016A4369C4685B5C96
:10D7A8000131A14228BF114601625DF8044BD8B28D
:10D7B800704700BF436B13B190F844007047836A09
:10D7C800406A181AB0FA80F040097047416A836AC3
:10D7D80099420AD3CB1A416B026961B14968501E5C
:10D7E8000B4483420AD2C01A704702691144CB1A0B
:10D7F800416B0029F2D1501EC01A704700207047B3
:10D80800036B43B1026C5B6893422FBF981AC068E0
:10D818009B1AC0187047C269036A9A422FBFD01A70
:10D82800C0688018C01A70470A4B30B503F1140459
:10D8380093F900205D78072AC8BF143A8118043389
:10D848000D7313F8025C855413F8012C0A76A34271
:10D85800EED130BDECBE020803682DE9F041DF6966
:10D868001FB13B46BDE8F0411847002A164611DDB6
:10D8780004460D460E4400E023689B6820469847FE
:10D888000028F9D0236815F8011B1B682046984723
:10D89800AE42F1D1BDE8F08100232322027043702B
:10D8A8008370C37070472D2343702E2303712F2379
:10D8B800C371704730B50446006D61710368A26892
:10D8C80023F00103036087B0A379009213F00402E8
:10D8D8003DD04FF4805213F00203019244D10293D9
:10D8E8004FF480630022039311F00103059237D1AE
:10D8F800049308238D07694648BF049316F0CEF8B1
:10D908006079236DA17900F00202002A15BF4FF457
:10D9180040324FF480324FF40034002410F0010FED
:10D92800586808BF2246CC074CBF024320EA0202CF
:10D938005A609A6809074CBF42F0080222F00802B0
:10D948009A601A6842F001021A6007B030BD13F0FD
:10D95800020301920BD04FF4005513460295C1E71C
:10D96800042304930C23C5E74FF40053B7E702934D
:10D97800B8E700BF10B50446006DA160036823F046
:10D9880001030360A37986B013F00402009141D02B
:10D998004FF4805213F00203019244D102934FF4E2
:10D9A800806362790393D1074FF0000304930593D2
:10D9B80045BF0423049308230C236946920748BFF4
:10D9C800049316F06BF86079236DA17900F00202D8
:10D9D800002A15BF4FF440324FF480324FF4003420
:10D9E800002410F0010F586808BF2246CC074CBF2E
:10D9F800024320EA02025A609A6809074CBF42F0C3
:10DA0800080222F008029A601A6842F001021A60BD
:10DA180006B010BD13F00203019207D04FF4005175
:10DA280013460291BDE74FF40053B7E70293B8E7F6
:10DA3800002326220360027027228270012243609D
:10DA480002718371704700BF2DE9F04F013085B036
:10DA5800C3B203938C4D8D4F8D4C8E4E0A23029387
:10DA6800DFF8349210F08AFF4FF4FA7A4FF0100C76
:10DA78004FF47A70D9F80430C3F30803002B40F050
:10DA8800C580EFF31183002B40F0C0802968A2689D
:10DA980000BF2B689942F9D1D7F800E000FB0EF3DC
:10DAA8009B1AB3FBFEF300FB01314FF0010E01910D
:10DAB800D9F80430C3F30803002B40F08B80EFF350
:10DAC8001183002B40F086802B68A16800BF2A686C
:10DAD8009342F9D1D7F800B000FB0BF2521AB2FB0F
:10DAE800FBF200FB0323019A9B1AB3F57A7FDFD37D
:10DAF800BAF1010ABED1039B002B40F0C1804FF45C
:10DB08007A7ADFF8949150464FF0100CD9F8043027
:10DB1800C3F30803002B40F09680EFF31183002B2A
:10DB280040F091802968A26800BF2B689942F9D11A
:10DB3800D7F800E000FB0EF39B1AB3FBFEF300FBE3
:10DB480001314FF0010E0191D9F80430C3F30803F5
:10DB580023BBEFF311830BBB2B68A16800BF2A68B6
:10DB68009342F9D1D7F800B000FB0BF2521AB2FB7E
:10DB7800FBF200FB0323019A9B1AB3F57A7FE3D3E8
:10DB8800BAF1010AC2D1029B013B02937FF468AF4C
:10DB9800414B424ADA6005B0BDE8F08FEFF31188D7
:10DBA8008CF31288A1682368DB0344BFC6F800E041
:10DBB800A1682B6832685FFA88F888F31188D7F86B
:10DBC80000801A4400FB08F35B1AB3FBF8F300FB70
:10DBD8000233D0E7EFF311888CF31288A168236829
:10DBE800DB0344BFC6F800E0A1682B6832685FFA1F
:10DBF80088F888F31188D7F800801A4400FB08F3E6
:10DC08005B1AB3FBF8F300FB02336CE7EFF3118206
:10DC18008CF31288D4F808E02368D90303D50123CC
:10DC28003360D4F808E02B683168D2B282F31188E7
:10DC38003A68194400FB02F3A3EB0E03B3FBF2F3BB
:10DC480000FB013131E7EFF311828CF31288D4F82D
:10DC580008E02368D90303D501233360D4F808E02A
:10DC68002B683168D2B282F311883A68194400FBF4
:10DC780002F3A3EB0E03B3FBF2F300FB013160E701
:10DC8800184610F023FD3AE7E84A0020EC4A002045
:10DC980010E000E0E44A002000ED00E00400FA058E
:10DCA8002DE9F04F013085B0C3B203930B460291C2
:10DCB8008B4C8C4E002B00F099808B4D8B4FDFF8EE
:10DCC800309210F05BFE4FF4FA7A4FF0100C4FF4DC
:10DCD8007A70D9F80430C3F30803002B40F0DE80D3
:10DCE800EFF31183002B40F0D9802968A26800BFA8
:10DCF8002B689942F9D1D7F800E000FB0EF39B1A84
:10DD0800B3FBFEF300FB01314FF0010E0191D9F88E
:10DD18000430C3F30803002B40F08780EFF311832E
:10DD2800002B40F082802B68A16800BF2A689342CC
:10DD3800F9D1D7F800B000FB0BF2521AB2FBFBF294
:10DD480000FB0323019A9B1AB3F57A7FDFD3BAF15C
:10DD5800010ABED1039B002B40F0BD804FF47A7AB4
:10DD6800DFF88C9150464FF0100CD9F80430C3F30B
:10DD78000803002B75D1EFF31183002B71D12968AB
:10DD8800A26800BF2B689942F9D1D7F800E000FBE0
:10DD98000EF39B1AB3FBFEF300FB01314FF0010EAB
:10DDA8000191D9F80430C3F3080313BBEFF31183CF
:10DDB800FBB92B68A16800BF2A689342F9D1D7F84C
:10DDC80000B000FB0BF2521AB2FBFBF200FB03237C
:10DDD800019A9B1AB3F57A7FE3D3BAF1010AC4D149
:10DDE800029B013B0293002B7FF467AF05B0BDE8AF
:10DDF800F08FEFF311888CF31288A1682368DB0396
:10DE080044BFC6F800E0A1682B6832685FFA88F85A
:10DE180088F31188D7F800801A4400FB08F35B1ACE
:10DE2800B3FBF8F300FB0233D2E7EFF311888CF36E
:10DE38001288A1682368DB0344BFC6F800E0A16824
:10DE48002B6832685FFA88F888F31188D7F8008061
:10DE58001A4400FB08F35B1AB3FBF8F300FB023328
:10DE680070E7EFF311828CF31288D4F808E0236886
:10DE7800D90303D501233360D4F808E02B6831684F
:10DE8800D2B282F311883A68194400FB02F3A3EB7B
:10DE98000E03B3FBF2F300FB01317FE7EFF31182CE
:10DEA8008CF31288D4F808E02368D90303D501233A
:10DEB8003360D4F808E02B683168D2B282F3118855
:10DEC8003A68194400FB02F3A3EB0E03B3FBF2F329
:10DED80000FB013118E7184610F0F8FB3EE700BFD9
:10DEE80010E000E0E44A0020E84A0020EC4A002064
:10DEF80000ED00E0204B5B68C3F3080330B4BBB906
:10DF0800EFF31183A3B91D4B1D4C1868A16800BF1E
:10DF18001A689042F9D11B4B1C684FF47A7202FBC5
:10DF280004F3591AB1FBF4F130BC02FB001070473E
:10DF3800EFF31182102383F3128811498C680B6860
:10DF480013F4803F104B02D0012018608C680B49F5
:10DF5800D2B20D68186882F311880A4B19684FF419
:10DF68007A72284402FB01F31B1B30BCB3FBF1F3AC
:10DF780002FB0030704700BF00ED00E0E84A0020D7
:10DF880010E000E0EC4A0020E44A00202DE9F84FB8
:10DF98008046FFF7AFFF254E2549DFF8A0E0254A68
:10DFA800254D844610274FF47A740120DEF804309A
:10DFB800C3F30803D3B9EFF31183BBB90B68D2F8E5
:10DFC80008A000BFD1F800904B45F7D1D6F800B0B3
:10DFD80004FB0BF9A9EB0A09B9FBFBF904FB039352
:10DFE800A3EB0C034345E1D3BDE8F88FEFF3118AA7
:10DFF80087F31288D2F808B01368DB0344BF28609F
:10E00800D2F808B00B68D5F800905FFA8AFA8AF35C
:10E018001188D6F800A0994404FB0AF3A3EB0B037C
:10E02800B3FBFAF304FB0933DAE700BFEC4A00203C
:10E03800E84A002010E000E0E44A002000ED00E09B
:10E048002DE9F04FDFF830C1474A4849484E494D5D
:10E058008046102718F1FF38C0F08480DCF80430BF
:10E06800C3F30803002B5CD1EFF31183002B58D1C5
:10E078000B68946800BF08688342F9D1D6F800900D
:10E088004FF47A7000FB09FEAEEB040EBEFBF9FEFE
:10E0980000FB03EEDCF80430C3F308034FF47A7492
:10E0A8000120FBB9EFF31183E3B90B68D2F808A09C
:10E0B80000BFD1F800904B45F7D1D6F800B004FB6B
:10E0C8000BF9A9EB0A09B9FBFBF904FB0393A3EBD2
:10E0D8000E03B3F57A7FBDD2DCF80430C3F308032E
:10E0E800002BDFD0EFF3118A87F31288D2F808B03B
:10E0F8001368DB0344BF2860D2F808B00B68D5F872
:10E1080000905FFA8AFA8AF31188D6F800A0994439
:10E1180004FB0AF3A3EB0B03B3FBFAF304FB093389
:10E12800D5E7EFF3118487F31288D2F808901368C3
:10E13800D80303D501232B60D2F808900B68286810
:10E14800E4B284F31188D6F800A04FF47A7400EB97
:10E15800030E04FB0AF3A3EB0903B3FBFAF304FB76
:10E168000E3E97E7BDE8F08F10E000E0E84A002097
:10E17800EC4A0020E44A002000ED00E030B4EFF360
:10E188001183102282F312880649074C0A6807484F
:10E19800013200250A602560DBB2026883F311882A
:10E1A80030BC7047E84A0020E44A002010E000E054
:10E1B8001D4B70B59C68236D226BDD69C2B1636B22
:10E1C8002BB12B0702D5236D08221A6270BD2A06CF
:10E1D800F7D5A26A616A8A421FD0511CA069A16260
:10E1E800825C2069266D81423285EAD3A362E8E722
:10E1F800A906E4D5E26A1AB1988C80B29047DEE7A6
:10E20800E1699B8C6069DBB24E1CE6614354E169AD
:10E21800E368994228BFE261D1E7226D136823F0D1
:10E2280080031360CDE700BF703900201D4B70B527
:10E238005C68236D226BDD69C2B1636B2BB12B0760
:10E2480002D5236D08221A6270BD2A06F7D5A26A84
:10E25800616A8A421FD0511CA069A162825C206950
:10E26800266D81423285EAD3A362E8E7A906E4D5A0
:10E27800E26A1AB1988C80B29047DEE7E1699B8C1C
:10E288006069DBB24E1CE6614354E169E368994278
:10E2980028BFE261D1E7226D136823F08003136081
:10E2A800CDE700BF703900201D4B70B51C68236D89
:10E2B800226BDD69C2B1636B2BB12B0702D5236DCD
:10E2C80008221A6270BD2A06F7D5A26A616A8A42D4
:10E2D8001FD0511CA069A162825C2069266D814211
:10E2E8003285EAD3A362E8E7A906E4D5E26A1AB15F
:10E2F800988C80B29047DEE7E1699B8C6069DBB25D
:10E308004E1CE6614354E169E368994228BFE26123
:10E31800D1E7226D136823F080031360CDE700BFB7
:10E328007039002003685B6A03B11847704700BF63
:10E3380003681B6A03B11847704700BF03682DE9DB
:10E34800F041DF691FB13B46BDE8F0411847002A9C
:10E35800164611DD04460D460E4400E023689B680E
:10E36800204698470028F9D0236815F8011B1B6838
:10E3780020469847AE42F1D1BDE8F08103689B6919
:10E38800184700BF0368DB68184700BF03689B682D
:10E39800184700BF03685B68184700BF03681B681D
:10E3A800184700BF054B53F8203033B11A689B88D3
:10E3B800918A0B4218BF1B0493617047D84A00200A
:10E3C800036803F138422DE9F04F920A584DAA5CD0
:10E3D80002F01F0552090124022A04FA05F400F08C
:10E3E8008C80032A00F08E80012A3CD001F00307BC
:10E3F8007A1E012AC1F3810CC1F300188088C1F389
:10E40800411135D9C60700F19780850700F1A3802F
:10E41800440700F1B180020700F1BF80C60600F191
:10E42800CD80850600F1DB80440600F1E980020614
:10E4380000F1F780C60500F10581850500F113811B
:10E44800440500F12181020500F12F81C60400F185
:10E458003D81850400F14B81440400F15981020497
:10E4680055D4BDE8F08F334A55692C435461BDE754
:10E47800002422464FF0010E4FF0030904E0013258
:10E48800102A04F10204ECD00EFA02F636EA00056E
:10E49800F5D1D3F808A009FA04F5ED430AEA050A0C
:10E4A800C3F808A0D3F808B00CFA04FA4AEA0B0A31
:10E4B800C3F808A0B3F804A01FFA8AFA2AEA0606E5
:10E4C8009E80B3F804A008FA02F646EA0A06B6B235
:10E4D8009E801E682E401E60D3F800A007FA04F63E
:10E4E80046EA0A061E60D3F80CA001FA04F605EA0B
:10E4F8000A0A46EA0A05DD60C1E70E4A95692C4317
:10E50800946173E70B4AD5692C43D4616EE71A68A6
:10E5180022F040421A601A6842EA87771F60DA6878
:10E5280022F0404242EA8171D960BDE8F08F00BF15
:10E5380034DE0208001002401A6822F003021A6052
:10E548001A683A431A60DA6822F003020A43850718
:10E55800DA607FF55DAF1A6822F00C021A601A685B
:10E5680042EA87021A60DA6822F00C0242EA810263
:10E578004407DA607FF54FAF1A6822F030021A605C
:10E588001A6842EA07121A60DA6822F0300242EA90
:10E598000112DA6002077FF541AF1A6822F0C00263
:10E5A8001A601A6842EA87121A60DA6822F0C00212
:10E5B80042EA8112C606DA607FF533AF1A6822F4A0
:10E5C80040721A601A6842EA07221A60DA6822F46E
:10E5D800407242EA01228506DA607FF525AF1A68A3
:10E5E80022F440621A601A6842EA87221A60DA68DE
:10E5F80022F4406242EA81224406DA607FF517AFCE
:10E608001A6822F440521A601A6842EA07321A60FD
:10E61800DA6822F4405242EA0132DA6002067FF5F3
:10E6280009AF1A6822F440421A601A6842EA87322F
:10E638001A60DA6822F4404242EA8132C605DA609A
:10E648007FF5FBAE1A6822F440321A601A6842EA73
:10E6580007421A60DA6822F4403242EA014285052C
:10E66800DA607FF5EDAE1A6822F440221A601A6863
:10E6780042EA87421A60DA6822F4402242EA81427A
:10E688004405DA607FF5DFAE1A6822F440121A609A
:10E698001A6842EA07521A60DA6822F4401242EA1B
:10E6A8000152DA6002057FF5D1AE1A6822F4400201
:10E6B8001A601A6842EA87521A60DA6822F440023D
:10E6C80042EA8152C604DA607FF5C3AE1A6822F0C6
:10E6D80040721A601A6842EA07621A60DA6822F021
:10E6E800407242EA01628504DA607FF5B5AE1A68C5
:10E6F80022F040621A601A6842EA87621A60DA6891
:10E7080022F0406242EA81624404DA607FF5A7AEF3
:10E718001A6822F040521A601A6842EA07721A60B0
:10E72800DA6822F0405242EA0172DA6097E600BFE6
:10E7380010B50409013C052C17D80D4B33F81420EB
:10E7480000F00F0042FA00F313F001030DD001238B
:10E7580003FA00F0013810401AF09EFB054A064BF8
:10E76800125D104403EBC00010BD002010BD00BFB7
:10E7780020D802082CD80208E05100202DE9F04FDB
:10E788004A484B4B4B4C4FF090414FF0010A4FF029
:10E7980002094FF004084FF0080C4FF0100E202724
:10E7A8004026802530F8022B12F0010F03D01960A3
:10E7B800A3F804A0083312F0020F03D01960A3F8DD
:10E7C8000490083312F0040F03D01960A3F80480F2
:10E7D800083312F0080F03D01960A3F804C00833F7
:10E7E80012F0100F03D01960A3F804E0083312F0F8
:10E7F800200F02D019609F80083312F0400F02D01A
:10E8080019609E80083312F0800F02D019609D8035
:10E81800083312F4807F05D04FF4807B1960A3F889
:10E8280004B0083312F4007F05D04FF4007B196060
:10E83800A3F804B0083312F4806F05D04FF4806B4E
:10E848001960A3F804B0083312F4006F05D04FF430
:10E85800006B1960A3F804B0083312F4805F05D088
:10E868004FF4805B1960A3F804B0083312F4005F1A
:10E8780005D04FF4005B1960A3F804B0083312F414
:10E88800804F05D04FF4804B1960A3F804B00833CB
:10E89800D20B04D04FF4004219609A80083301F576
:10E8A8008061A1427FF47EAFBDE8F08F20D80208D6
:10E8B800E051002000180048002867D003682DE9BF
:10E8C800F04F03F138445C4EA40A0125345D04F08E
:10E8D8001F066409022C05FA06F558D0032C00F02F
:10E8E800A580012C58D08088B0FA80F4C4F11F04A8
:10E8F800A4B2E50803EB850504F007042E6AA4001A
:10E908000F27A74026EA07062E622E6A01F00307A2
:10E91800A2407C1E3243012CC1F3810CC1F30018C4
:10E928002A62C1F341113CD9C60700F189808507E5
:10E9380000F19580440700F1A380020700F1B1803F
:10E94800C60600F1BF80850600F1CD80440600F1BF
:10E95800DB80020600F1E980C60500F1F780850535
:10E9680000F10581440500F11381020500F12181C0
:10E97800C60400F12F81850400F13D81440400F1B3
:10E988004B81020400F15981BDE8F08F70472B4C90
:10E99800A6693543A561A6E7284C666935436561D4
:10E9A800A1E7002422464FF0010E4FF0030904E0CE
:10E9B8000132102A04F10204E6D00EFA02F636EA11
:10E9C8000005F5D1D3F808A009FA04F5ED430AEAE1
:10E9D800050AC3F808A0D3F808B00CFA04FA4AEA02
:10E9E8000B0AC3F808A0B3F804A01FFA8AFA2AEAA7
:10E9F80006069E80B3F804A008FA02F646EA0A065C
:10EA0800B6B29E801E682E401E60D3F800A007FA9A
:10EA180004F646EA0A061E60D3F80CA001FA04F6CA
:10EA280005EA0A0A46EA0A05DD60C1E7034CE66919
:10EA38003543E56157E700BF34DE020800100240A5
:10EA48001A6822F003021A601A683A431A60DA68F0
:10EA580022F003020A438507DA607FF56BAF1A6874
:10EA680022F00C021A601A6842EA87021A60DA6811
:10EA780022F00C0242EA81024407DA607FF55DAFBA
:10EA88001A6822F030021A601A6842EA07121A60FD
:10EA9800DA6822F0300242EA0112DA6002077FF5F2
:10EAA8004FAF1A6822F0C0021A601A6842EA871249
:10EAB8001A60DA6822F0C00242EA8112C606DA60F9
:10EAC8007FF541AF1A6822F440721A601A6842EA68
:10EAD80007221A60DA6822F4407242EA01228506A7
:10EAE800DA607FF533AF1A6822F440621A601A6858
:10EAF80042EA87221A60DA6822F4406242EA8122F6
:10EB08004406DA607FF525AF1A6822F440521A608D
:10EB18001A6842EA07321A60DA6822F4405242EA76
:10EB28000132DA6002067FF517AF1A6822F4404214
:10EB38001A601A6842EA87321A60DA6822F4404298
:10EB480042EA8132C605DA607FF509AF1A6822F415
:10EB580040321A601A6842EA07421A60DA6822F4F8
:10EB6800403242EA01428505DA607FF5FBAE1A6859
:10EB780022F440221A601A6842EA87421A60DA6868
:10EB880022F4402242EA81424405DA607FF5EDAE84
:10EB98001A6822F440121A601A6842EA07521A6088
:10EBA800DA6822F4401242EA0152DA6002057FF57F
:10EBB800DFAE1A6822F440021A601A6842EA8752E5
:10EBC8001A60DA6822F4400242EA8152C604DA6026
:10EBD8007FF5D1AE1A6822F040721A601A6842EACC
:10EBE80007621A60DA6822F0407242EA016285041C
:10EBF800DA607FF5C3AE1A6822F040621A601A68BC
:10EC080042EA87621A60DA6822F0406242EA816268
:10EC18004404DA607FF5B5AE1A6822F040521A60F3
:10EC28001A6842EA07721A60DA6822F0405242EA29
:10EC38000172DA6002047FF5A7AE1A6822F040423A
:10EC48001A601A6842EA87771F60DA6822F0404241
:10EC580042EA8171D960BDE8F08F00BF002852D028
:10EC6800036803F138422DE9F04F920A504DAA5C2F
:10EC780002F01F0552090124022A04FA05F443D0C0
:10EC8800032A00F09080012A43D001F003077A1E7E
:10EC9800012AC1F3810CC1F300188088C1F3411126
:10ECA8003CD9C60700F18880850700F194804407A5
:10ECB80000F1A280020700F1B080C60600F1BE8014
:10ECC800850600F1CC80440600F1DA80020600F1E6
:10ECD800E880C60500F1F680850500F10481440549
:10ECE80000F11281020500F12081C60400F12E8195
:10ECF800850400F13C81440400F14A81020400F1DA
:10ED08005881BDE8F08F70472A4A95692C43946171
:10ED1800BBE7284A55692C435461B6E700242246CC
:10ED28004FF0010E4FF0030904E00132102A04F1FC
:10ED38000204E6D00EFA02F636EA0005F5D1D3F859
:10ED480008A009FA04F5ED430AEA050AC3F808A081
:10ED5800D3F808B00CFA04FA4AEA0B0AC3F808A078
:10ED6800B3F804A01FFA8AFA2AEA06069E80B3F8C6
:10ED780004A008FA02F646EA0A06B6B29E801E68A1
:10ED88002E401E60D3F800A007FA04F646EA0A06E9
:10ED98001E60D3F80CA001FA04F605EA0A0A46EA4E
:10EDA8000A05DD60C1E7034AD5692C43D4616CE7E5
:10EDB80034DE0208001002401A6822F003021A60CA
:10EDC8001A683A431A60DA6822F003020A43850790
:10EDD800DA607FF56CAF1A6822F00C021A601A68C4
:10EDE80042EA87021A60DA6822F00C0242EA8102DB
:10EDF8004407DA607FF55EAF1A6822F030021A60C5
:10EE08001A6842EA07121A60DA6822F0300242EA07
:10EE18000112DA6002077FF550AF1A6822F0C002CB
:10EE28001A601A6842EA87121A60DA6822F0C00289
:10EE380042EA8112C606DA607FF542AF1A6822F408
:10EE480040721A601A6842EA07221A60DA6822F4E5
:10EE5800407242EA01228506DA607FF534AF1A680B
:10EE680022F440621A601A6842EA87221A60DA6855
:10EE780022F4406242EA81224406DA607FF526AF36
:10EE88001A6822F440521A601A6842EA07321A6075
:10EE9800DA6822F4405242EA0132DA6002067FF56B
:10EEA80018AF1A6822F440421A601A6842EA873298
:10EEB8001A60DA6822F4404242EA8132C605DA6012
:10EEC8007FF50AAF1A6822F440321A601A6842EADB
:10EED80007421A60DA6822F4403242EA01428505A4
:10EEE800DA607FF5FCAE1A6822F440221A601A68CC
:10EEF80042EA87421A60DA6822F4402242EA8142F2
:10EF08004405DA607FF5EEAE1A6822F440121A6002
:10EF18001A6842EA07521A60DA6822F4401242EA92
:10EF28000152DA6002057FF5E0AE1A6822F4400269
:10EF38001A601A6842EA87521A60DA6822F44002B4
:10EF480042EA8152C604DA607FF5D2AE1A6822F02E
:10EF580040721A601A6842EA07621A60DA6822F098
:10EF6800407242EA01628504DA607FF5C4AE1A682D
:10EF780022F040621A601A6842EA87621A60DA6808
:10EF880022F0406242EA81624404DA607FF5B6AE5C
:10EF98001A6822F040521A601A6842EA07721A6028
:10EFA800DA6822F0405242EA0172DA6002047FF520
:10EFB800A8AE1A6822F040421A601A6842EA8777B7
:10EFC8001F60DA6822F0404242EA8171D960BDE8E8
:10EFD800F08F00BF10B1036882881A85704700BFA0
:10EFE80010B1036882889A61704700BF38B1002960
:10EFF8008388026814BF002110218B4093617047F9
:10F0080010B40A4B0A4A1C7801238340234052F863
:10F01800200029B9B3FA83F149095DF8044BE5E703
:10F02800191C18BF01215DF8044BDFE7D44A002002
:10F03800D84A002030B1036882881B8A1A4214BF5C
:10F0480001200020704700BF2DE9F0410B4E3468C5
:10F0580073691C400FD0DFF828800127B4FA84F3C5
:10F06800C3F11F0307FA03F558F82300036898470C
:10F07800AC437561F2D1BDE8F08100BF00040140E6
:10F08800F04A00202DE9F0410B4E346873691C40AA
:10F098000FD0DFF828800127B4FA84F3C3F11F03E7
:10F0A80007FA03F558F8230003689847AC437561DD
:10F0B800F2D1BDE8F08100BF00040140F04A002011
:10F0C8002DE9F0410B4E346873691C400FD0DFF80E
:10F0D80028800127B4FA84F3C3F11F0307FA03F564
:10F0E80058F8230003689847AC437561F2D1BDE82E
:10F0F800F08100BF00040140F04A00202DE9F041F2
:10F108000B4E346873691C400FD0DFF82880012744
:10F11800B4FA84F3C3F11F0307FA03F558F8230080
:10F1280003689847AC437561F2D1BDE8F08100BF30
:10F1380000040140F04A00202DE9F0410B4E3468EC
:10F1480073691C400FD0DFF828800127B4FA84F3D4
:10F15800C3F11F0307FA03F558F82300036898471B
:10F16800AC437561F2D1BDE8F08100BF00040140F5
:10F17800F04A00202DE9F0410B4E346873691C40B9
:10F188000FD0DFF828800127B4FA84F3C3F11F03F6
:10F1980007FA03F558F8230003689847AC437561EC
:10F1A800F2D1BDE8F08100BF00040140F04A002020
:10F1B8002DE9F0410B4E346873691C400FD0DFF81D
:10F1C80028800127B4FA84F3C3F11F0307FA03F573
:10F1D80058F8230003689847AC437561F2D1BDE83D
:10F1E800F08100BF00040140F04A0020084A0948A5
:10F1F80008B5936943F001039361002140221CF094
:10F2080017FB054B4FF0FF321A60C3F8032008BD07
:10F2180000100240F04A0020304B002003685B6A6F
:10F22800184700BF2DE9F041044618460D4616461A
:10F23800984619F087F92768E6722844A07229468B
:10F248007D69434632462046AC46BDE8F0416047FA
:10F25800036810B504461B689847236820469B68D6
:10F268009847A37B0133A37310BD00BF10B5036893
:10F2780004469B689847FF2301226373227310BDDD
:10F28800427A02B9704710B504460368406804F131
:10F298000A0198470023637210BD00BF03680A7A09
:10F2A800591C01601A70704738B50B4C23688BB134
:10F2B8005A68821A002A054604DA0CE05A68AA1A23
:10F2C800002A07DB9A68226018461A689047236864
:10F2D800002BF3D138BD38BDDC5500200B4B002284
:10F2E80010B4027203F5A074032102E0072A09DCB6
:10F2F8009979890702D51979815401329C4203F121
:10F308001403F3D15DF8044B704700BFD0DC02084A
:10F3180010230370704700BF012310B41521142473
:10F32800222244704171C2700370037183705DF8CA
:10F33800044B704770B54E680546304619F002F91F
:10F3480031460446024628681CF04DFA2A6813190B
:10F3580001333B212B60115570BD00BF08B50AF081
:10F36800B3FA024B024ADA60FEE700BF00ED00E0A4
:10F378000400FA05024A034B1278197804F0CABA55
:10F38800881B0020891B00202DE9F0470569C36808
:10F398001D4028D00F4606464FF000484FF00009A0
:10F3A800B5FA85F328FA03F2D2431B3B32611540C4
:10F3B800042B16D8DFE803F03129211903007B6AF2
:10F3C800002B32D003F1FF3A1FFA8AFAC7F82490CB
:10F3D8003C6A34B123682046514698476468002C3B
:10F3E800F8D1002DDCD1BDE8F0873868716B03686F
:10F3F80089B29847002DD3D1F5E77868B16B0368D7
:10F4080089B29847002DCBD1EDE7B868F16B036856
:10F4180089B29847002DC3D1E5E7F868316C0368D5
:10F4280089B29847002DBBD1DDE7F36A1FFA83FA4A
:10F43800CEE700BFF0B5434B43491A68096883B06B
:10F448000123570200935CBF03F180530093D60059
:10F458005CBF43F0100300938C0744BF43F0C6031E
:10F468000093480744BF43F008030093D105374988
:10F47800097848BF43F0006301F0EF0048BF0093EC
:10F4880008286D4651D00E294FD03148009B00788E
:10F49800D70454BF43F0444343F06443002843F483
:10F4A80000530CBF07200F20960648BF43F4807313
:10F4B800540748BF43F4003343F400245205009432
:10F4C80002D5244A1279A2BB182936D00190002708
:10F4D800012639462846FCB2FBF76AFE60B11E4B8E
:10F4E800002203F5D87103E08B420FD013F80C2CDF
:10F4F800944203F10C03F7D10137242FE9D195E8A1
:10F508000300164B83E8030003B0F0BD7A0904F04A
:10F518001F0455F8223006FA04F4013723EA0404DC
:10F52800242F45F82240D4D1E9E743F480530093CF
:10F53800ABE743F4C0130093C6E7009B43F0607346
:10F548000093C3E7504A0020684B0020942B00200A
:10F558005445002090420020E8B90208801B002092
:10F568002DE9F84F4E014FF0000B174D814690469C
:10F5780006F120075C46594628465FFA8BFAFBF7E6
:10F5880017FEC0B1A64215D8A74213D900200F4ACA
:10F59800014604E00131242914D012F80C0C50451E
:10F5A80002F10C02F6D10A4B01EB410103EB810198
:10F5B8004846C04701340BF1010BBBF1240FDAD1E7
:10F5C800BDE8F88F0021F3E7801B0020E8B90208A6
:10F5D800DCB9020800210A4A0B4604E00133242B57
:10F5E8000BD012F80C1C884202F10C02F6D1054827
:10F5F80003EB430300EB830070470020704700BF14
:10F60800F0B90208DCB9020800210A4A0B4604E0F6
:10F618000133242B0BD012F80C1C884202F10C0287
:10F62800F6D1054803EB430300EB83007047002045
:10F63800704700BFE8B90208DCB9020808B5012123
:10F648000220FFF7DDFC094B1B7803F00503052BAF
:10F6580008D000210120FFF7D3FC00210846FFF75E
:10F66800CFFCFEE70AF0E0F9F3E700BF6C390020B1
:10F67800022810B428BF0220064C074B207000EB6C
:10F68800C001064A5DF8044B00EB810003EB400023
:10F6980010607047F44200205A2600200C430020D6
:10F6A80008B512F019F9FBF7F5F8BDE8084012F0B3
:10F6B800FBB800BF38B5434B5A899989914224BF9A
:10F6C80000225A81198ADA89914224BF0022DA81FC
:10F6D800DA7892B1072A10D03B4C3C48A278012135
:10F6E8000025062A01709970DD719D7152D9237920
:10F6F800DFED376A002B3CD138BDDA79002A4ED0CD
:10F708009A783248DFED326A0178042A38BF042239
:10F7180007EE902AB8EEE77A07EE901A27EE267AD7
:10F72800F8EEE77A9A7067EE877A274CA278002578
:10F73800062A9D712BD8274B03EB8203D3ED006A71
:10F74800F4EEE76AF1EE10FA10DDC6EE877AFDEE08
:10F75800E77A17EE903A102BA8BF1023012BB8BFF9
:10F768000123DBB28B4228BF0B4603702379002BA1
:10F77800C2D0013A032ABFD8B7EE000A80EE260AA3
:10F7880019F040FF2388984238BF208038BDDFED4C
:10F79800106AD5E7DFED107AB0EE677ACBE79A7892
:10F7A8000A48DFED0E6A017807EE102A07EE901A74
:10F7B800B8EEC77AF8EEE77A27EE267A67EE877A08
:10F7C800B3E700BF746A00202C450020382B0020C6
:10F7D8006F12033800BF02086F12833A6F120339A1
:10F7E8002DE9F047A84FA94E12F076F8BE421ED276
:10F7F800DFF82083DFF820934446258862197DB11D
:10F808004A450DD2052D0BD933886188C3F30B0304
:10F81800994200F0D880144625886219002DEFD14E
:10F82800716830461436FAF7B9FFBE42E4D3984AF5
:10F838005378022B40F2EC800023964953701378DA
:10F848009548022B016000F2DF8003EBC301934A65
:10F8580003EB810302EB4303914C1846236009F044
:10F86800B5FE904A1378A3F1170102290FD98E49E2
:10F8780011F83300002840F0D180D80001444978BD
:10F8880029B18A4911F83330002B00F0F580884BF4
:10F898009A78042A00F0E78032B91A88B2F5F07F26
:10F8A80084BF4FF4F0721A80824D834A2B681A4045
:10F8B800002A00F0E480DE0700F1D080580400F14F
:10F8C800C880190700F1C0809A0100F1B7809B0435
:10F8D80000F1AD8023689A8CD98C914224BF002214
:10F8E8009A84FFF7E7FE0EF017FA10B9734815F07F
:10F8F80003F916F07DFB0021302271481BF098FFB8
:10F90800704B266803F1500102E00433994279D024
:10F918001A78002AF9D19C78D8788442F5D26A49B5
:10F928006A4B91F800E06A486A4D1C6B6A4B286084
:10F93800C827642111FB0E71DFF8E0E15960674FB9
:10F9480030F8041C664DAEF8001000219960D960AB
:10F95800196159619961D96183F8201083F82110E0
:10F968003A702E600CB111F0F3FE5E4B9FED5E5ABB
:10F978001B885E4A9FED5E6A55795E4C5E495F481A
:10F98800086006EE903AF8EEE66A1388C5EE265A45
:10F9980007EE103A53881279C4ED005A07EE903AF0
:10F9A800B8EEC77A564BF8EEE77A1D725A7227EE10
:10F9B800067A67EE867ABDE8F04783ED017AC3EDF3
:10F9C800007A11F071BF63799B077FF424AF7168E7
:10F9D80094F804A03046FAF7E1FE3388BAEB133FF7
:10F9E8000BD173887068AA1FC3F30B039A4204F102
:10F9F8000601A8BF1A461BF0F6FE1436BE42FFF4F5
:10FA0800FBAE14E701228AE700231370234B23E798
:10FA1800204903EB430301EB830110E7D8000D18DD
:10FA28006D68002D7FF42AAF1725157026E7354835
:10FA3800FAF7EAFE4020FAF7E7FE4BE746F209003C
:10FA4800FAF7E2FE2B6842E72F48FAF7DDFE2B684B
:10FA58003AE72E48FAF7D8FE2B6832E72C48FAF72F
:10FA6800D3FE2B682AE71A8BB2F57A7FBFF41CAF56
:10FA78004FF47A721A8317E71823137007E743F4D1
:10FA880000532B6017E700BFD4100308D80C0308F5
:10FA9800F442002010430020006900205A2600206C
:10FAA8000C430020942B00205CD90208A4C2020851
:10FAB8002C4500206C2B002009600002486A0020B9
:10FAC800FC220020982B0020DC400020344300203A
:10FAD800482B002050730020A04400205618002016
:10FAE80030230020C81C0020C0C9FB483423002054
:10FAF80017B7D138CC1C00205C3A00203661023D93
:10FB0800383A002009400002016000020920000282
:10FB18000860000207F00308000004083C550020B4
:10FB280008B511F0D9FEFAF7B5FE11F0BDFEBDE833
:10FB3800084055E638B50C4C0C4DAC4206D261680D
:10FB480020461434FAF72AFEAC42F8D3084B094C85
:10FB5800094818600025257009F038FD074B084A48
:10FB680065701A6038BD00BFD80C0308D4100308AC
:10FB78000C430020F44200205A260020006900208F
:10FB88001043002008B5FFF7D5FF11F0A5FEFAF7DE
:10FB980081FEBDE8084011F087BE00BFF0B50C2912
:10FBA8002BD8DFE801F06F2A2A2A4C2A2A2A2B2A86
:10FBB8002A2A0700046AB2F80CE097881668674D8D
:10FBC80024F480540462036A4468C16923F400532E
:10FBD80043EA0E3321F4E641A84243EA073341EAF7
:10FBE800062100F0B58005F50065A84200F0B08058
:10FBF80092684460C16102640362F0BD046A968938
:10FC08009588D2F800E0554F24F480740462036AA2
:10FC18004468C16923F4007343EA062321F07301A1
:10FC2800B84243EA052341EA0E017ED04C4DA84272
:10FC38007BD092684460C161C2630362F0BD046A0C
:10FC480096899588D2F800E0444F24F010040462A5
:10FC5800036A4468816923F0200321F0807143EA34
:10FC6800061321F4E641B84243EA051341EA0E219E
:10FC780048D03B4DA84245D0926844608161826378
:10FC88000362F0BD046A9389B2F804E01768334E42
:10FC980024F001040462056A4468816943EA0E039A
:10FCA80021F4803125F002059BB221F07301B042A6
:10FCB80043EA050341EA070114D0294DA84211D0AF
:10FCC80005F54065A8420DD005F58065A84209D024
:10FCD80005F58065A84205D0926844608161426359
:10FCE8000362F0BDD689158A578A23F00803334387
:10FCF8003D43D68824F4407423F00403ADB2334363
:10FD08002C43E9E7D589178AD68823F0800343EA8C
:10FD1800051324F44064558A23F0400344EA870419
:10FD280043EA061344EA8504A6E7D589178AD688E4
:10FD380023F4006343EA052324F44054558A23F44A
:10FD4800806344EA071443EA062344EA051470E78B
:10FD5800158A24F4804444EA851449E7002C0140BC
:10FD6800003401402DE9F84F4FF48C72002185488A
:10FD7800854C864D864E874FDFF83482DFF8349203
:10FD88001BF056FD84488549DFF82CE2DFF82CC2C9
:10FD9800002213588B4200F0D580B3F1804F00F059
:10FDA800D880AB4200F0DC80B34200F0DC80BB427C
:10FDB80000F0DC80734500F0DC80634500F0AD8026
:10FDC800434500F0D9804B4500F0D980DFF8F0A119
:10FDD800534508BF4FF4802A00F0A1801432B2F5D1
:10FDE800AA7FD6D1DFF8B0816D4F6E4D08F5AA769F
:10FDF8004FF0030A4FF0020998F804301C09013C3F
:10FE0800052C03F00F0300F2818037F8140040FA44
:10FE180003F2D2077AD54FF0010B0BFA03F3013B3B
:10FE2800184019F039F8604B1B5D184415EBC004F5
:10FE38006CD055F830305D4898F8081003F1384216
:10FE4800920A825C02F01F005209022A0BFA00FB98
:10FE580071D0032A68D0012A05D14B4A4A48526911
:10FE68004BEA02024261B4F804E0BEFA8EF2C2F133
:10FE78001F0292B2D00803EB800002F00702046A66
:10FE880092004FF00F0C0CFA02FC24EA0C040462F6
:10FE9800046A01FA02F22243002402624FF0010CC4
:10FEA800224603E0102A04F102042FD00CFA02F0D3
:10FEB80030EA0E0102F10102F4D1D3F808B00AFACF
:10FEC80004F1C9430BEA010BC3F808B0D3F808B032
:10FED800C3F808B0B3F804B01FFA8BFB2BEA000094
:10FEE8009880988880B29880186808401860D3F87D
:10FEF80000B009FA04F040EA0B001860D868102A2C
:10FF080001EA0001D96004F10204CFD108F1140814
:10FF1800B0457FF471AFBDE8F88F4FF4005AA3697C
:10FF280043EA0A03A36159E7174A1748D2694BEA1B
:10FF38000202C26197E7144A134892694BEA020227
:10FF4800826190E7A3694FF4006A43EA0A03A36158
:10FF580044E74FF0010AE36943EA0A03E3613DE736
:10FF68004FF0020AF7E74FF0040AF4E74FF0100ADF
:10FF7800F1E74FF0200AEEE74FF4803ACFE74FF46D
:10FF8800003ACCE72C690020001002400004004031
:10FF98000008004000100040D0DC0208002C01409E
:10FFA80020D80208E05100202CD8020834DE0208CC
:10FFB800004001400044014000140040003401406A
:10FFC8000048014001490248FFF7DEB91C6A0020D9
:10FFD8000048014001490248FFF7D6B9CC69002022
:10FFE8000040014001490248FFF7CEB9A46900204A
:08FFF800000800400149024825
:020000040801F1
:10000000FFF7C6B97C6900200004004002494FF0A8
:100010008040FFF7BDB900BF5469002010B5064C01
:1000200006482146FFF7B4F904F1C8010448BDE8C9
:100030001040FFF7ADB900BF2C690020002C014033
:100040000044014001490248FFF7A2B92C69002091
:10005000002C01402DE9F0410468514DA30AAB4248
:1000600000F084800AD94F4DAB4277D00135AB42C6
:100070005FD0023DAB426DD0BDE8F0814A3DAB425E
:1000800070D00135AB4258D0B3F5801FF4D14FF09A
:10009000480E012647794FEA970C00296AD0B00034
:1000A000634685190227D4F80C809F400CEB45036A
:1000B000BFB23D4D03F1040C47EA080745F8231091
:1000C00045F82C20E760EFF31181502282F312886B
:1000D000821905EBC2021369002B32D0136204337C
:1000E000821905EBC202576917B11F6053690433C7
:1000F000821905EBC202976917B11F609369043337
:10010000821905EBC202D76917B11F60D3690433A6
:100110000027CAB21F6082F31188304405EBC0008B
:10012000036A8BB9E3684FF6FE721340E360BDE8E3
:10013000F0814FF4887E0626ACE74FF0980E032638
:10014000A8E705EB0E03CBE7E36843F00103E360A8
:10015000BDE8F0814FF0C00E04269BE74FF0E80E9B
:10016000052697E74FF0700E022693E74FF0200E1A
:1001700000268FE7BF08022306FA03F0BB40DB43EB
:10018000E768094D9BB23B4087190CEB470CE360D5
:100190000CF1040345F82C1045F8232093E700BF29
:1001A0004B001000510010002C69002030B503688E
:1001B0005C4D18885C4CB4FBF2F20139013AAB4259
:1001C00094B283B089B282B266D05848834263D079
:1001D000B3F1804F60D0A0F5983083425CD000F539
:1001E0008060834258D0524883425BD000F58060E3
:1001F00083427DD022F4407200F58C3092B283426B
:100200001A80D9621C850ED0484A93420BD002F561
:100210004062934207D002F58062934203D002F518
:100220008062934201D100221A8601225A611A8803
:100230003C4992B242F001028B421A8062D0B3F183
:10024000804F61D03B4A934260D002F58062934276
:100250005ED002F5006293425CD002F58062934268
:100260005AD002F59032934258D002F54062934240
:1002700056D002F5806293421ED002F5806293420E
:1002800008BF092219D002A84FF0012340F8043D0D
:100290000EF002FA03B030BD254822F0700283420E
:1002A00092B2A3D101201A80D9621C8558611A88A4
:1002B00092B202431A80C5E708221F4B03EBC20328
:1002C00001A893F821408DF80440012300228DF805
:1002D00005308DF807308DF806200EF0DDF91B2C67
:1002E000D8D1164B019301A80EF0D6F903B030BD5A
:1002F00001201A80D9621C8558611A8892B2024383
:100300001A809CE70022D8E70122D6E70222D4E730
:100310000322D2E70422D0E70522CEE70622CCE76B
:100320000722CAE7002C014000A24A040034014021
:10033000001000400004004000BF02081901000145
:10034000204B98422DD0B0F1804F2CD0A3F59433A0
:1003500098422AD003F58063984228D003F50063C1
:10036000984226D003F58063984224D003F5903359
:10037000984222D003F54063984220D003F5806371
:10038000984207D003F58063984208BF092202D043
:100390000020704708220C4B03EBC20393F82000A7
:1003A00070470022F7E70122F5E70222F3E7032274
:1003B000F1E70422EFE70522EDE70622EBE707224B
:1003C000E9E700BF002C014000BF02082DE9FF4112
:1003D000074618F0BBF808284AD1002501AE7C5D1D
:1003E00018F08CFF2044437803F00303022B08BF6E
:1003F000203CAC550135082DF1D10025DFF87C807B
:100400008DF80C507C5D18F079FF2044437803F0A0
:100410000303022B08BF203C7455E4B2214640463A
:100420001BF03FFA28B10135214670191BF039FA4B
:1004300020B115F0B1FC04B0BDE8F081082DE1D188
:100440000D49304611F016FA0B4C0C4800231A5D8A
:1004500004A90A44195C02F80C1C0133082BF6D1DC
:10046000002301A906488DF80C3015F07BFAE2E76D
:100470000028E9D0DDE700BF204A002034DA020876
:1004800039E102082DE9F84F054618F05FF8384FBA
:100490000446D7F80090B0B93648374D374F15F0BD
:1004A000DDF9012655F8241049B106FA04F313EAE0
:1004B000090F02D0384615F0B2F90134F2E7BDE871
:1004C000F84F15F038BA02462D4928461BF0FFF9BF
:1004D00078B92C482C4C2D4D15F0C0F954F8041F58
:1004E0000029ECD00B78002BF8D0284615F097F9AE
:1004F000F4E72B78DFF880B02D2B03BF013504F132
:10050000FF344FF0010A4FF0000A00265BF8268006
:10051000B8F1000F04D11E48BDE8F84F15F036BC05
:100520002246414628461BF0D2F9F8B90120B040D6
:10053000020604D51748BDE8F84F15F027BC83051F
:10054000F8D4BAF1000F0AD0FAF762F9124815F0A0
:1005500085F941460D48BDE8F84F15F003BA40EA69
:10056000090038600D4815F079F9F2E70136CDE75A
:100570006C2B002040E1020800D102084AE1020889
:100580004EE1020853E10208FCD0020871EB0208B8
:100590005EE102086BE1020877E1020880E10208EF
:1005A00070B5054617F0D2FF044690B11122002124
:1005B0000F481BF041F922460E4928461BF0AEF9C0
:1005C00038B1102C2246294628BF102208481BF0BB
:1005D000B7F9094B13F8042F002A064A06BF012178
:1005E00013460021054A0120BDE8704015F092BA7B
:1005F000F84200201F050308F442002088E10208A9
:100600002DE9F04188B0804615F0AEF8054608B3F4
:100610003B4CDFF8F880002519274FF461762379E9
:1006200017FB03630493E37817FB03630393A37837
:1006300002936378019314F8053B009342462B46DE
:1006400000210120013515F065FA0A2DE7D108B027
:10065000BDE8F081404618F049FE0928064648DC0E
:100660008400271808F101008DF81F5015F084F858
:10067000234D804648B118F039FE0D2805D89DF865
:100680001F30E85501338DF81F30404615F074F8DF
:10069000804660B118F02AFE431E042B07D8A31928
:1006A0002B4458709DF81F3001338DF81F304046A1
:1006B00015F062F8804660B118F018FE431E072B53
:1006C00007D89DF81F3034442C440133A0708DF8B6
:1006D0001F30F91C0DF11F022944404615F059F84E
:1006E0009DF81F30052BB2D0EA190023EB5113718E
:1006F000ADE709232A460349034815F033F9A6E775
:100700002A310020A6E10208ACE1020890E10208CB
:1007100008B50B4815F03AFB0A4B1868FEF7B4FD14
:10072000FAF762FFFAF706FE30B115F004F9064851
:10073000BDE8084015F02ABB6420FDF785FCF1E711
:10074000C5E1020844230020CEE102087FB5084C31
:10075000FAF740FDA568A288E668029000926388D7
:10076000218801962A46034815F0FCF804B070BDB4
:1007700088000020D4E102082DE9F04F85B004463E
:1007800014F0F2FF064620B115F006FB05B0BDE8F7
:10079000F08F204603AA4549DFF83C91DFF83CA1E1
:1007A000DFF83CB118F0F3FD34460546B0464FF093
:1007B000FF37B5B939463E48FAF7A8FB3D4B78B24A
:1007C0000C2606FB05F2D118D256824256D00135CE
:1007D000052DF6D1B8F1000F33D13748FAF796FB63
:1007E000D4E7012E0ED0022E11D01EB9284618F0E3
:1007F0007DFD074603AA2D49002018F0C8FD0136EB
:100800000546D6E7284618F071FD8046F2E74946CE
:1008100028461BF0AAF820B9284928461BF0A5F85D
:1008200008B144F00104514628461BF09EF828B94F
:10083000594628461BF099F80028DBD044F0020402
:10084000D8E7002C08BF03240022E4B201920094F0
:100850004346114614F03EFA054618B91848FAF70F
:1008600055FB93E741461748FAF750FB1648FAF74D
:100870004DFB164B2946186813F0D0FF4D68002D2C
:10088000A8D01348FAF742FB54B169798C4207D0DB
:1008900022461048FAF73AFBE1B22846FDF772FD0E
:1008A000EB6A002BE2D00023EB62DFE7B3E3020840
:1008B0003BE20208C049002044E2020832E202089A
:1008C0005CE2020873E20208B6E202085C31002032
:1008D00088E2020898E202082FE2020835E20208E4
:1008E00038E202082DE9F743054614F03DFF0446BF
:1008F00038B135490022012003B0BDE8F04315F0BE
:100900001BB900900190284618F0F0FC2E4B6E1C8D
:1009100040B203EBC40595F90220824250D0013465
:10092000052CF6D100252C46304614F025FF07464D
:1009300028B118F0DBFC0134ADF80000E4B2DFF8B8
:100940008C800026384614F017FF0746C8B118F00F
:10095000CDFC814614F0AAFD58F82030994510D1FD
:10096000022E1AD0032E1DD0431E012EDBB20FD053
:100970000B2B03D88DF803000134E4B20136042EAA
:10098000E0D1052C15D803B0BDE8F04315F004BA4A
:10099000042BF3D88DF80400EEE70528EED88DF887
:1009A0000600E9E7831EDBB20D2BE7D88DF80500C2
:1009B000E2E76B4603CB2860696003B0BDE8F083D3
:1009C0008DF802000124AFE7486A0020DCD5020858
:1009D00038B50D4618F08AFC041E09DB0C4B1B7859
:1009E0009C4205DA21460B48FAF790FA204638BDBA
:1009F0002DB1FF2C03D10848FAF788FAF6E7044B2B
:100A0000064819780139FAF781FA4FF0FF34EDE71B
:100A10002C290020D9E20208ECE2020801E30208D6
:100A20002DE9F74F054614F09FFE044618B9314BE7
:100A30009B78042B04D815F0AFF903B0BDE8F08F14
:100A4000284601AA2C49DFF8C490DFF8C48018F0CA
:100A50009EFC2746054645B9284B294A1B689B1A28
:100A6000284A18BF01231370E7E777B90121284608
:100A7000FFF7AEFF431C0446DFD001AA1E49002049
:100A800018F085FC01370546E5E712F0AFFD284672
:100A900018F02CFC2F28054626D8FF2C1BD1DFF898
:100AA00074A000265FFA80FB9AF800309E4209D3BA
:100AB000052D02DC0A20FDF7C7FA29461248FAF78D
:100AC00025FADAE798F800301BB15946F0B212F077
:100AD00073FB0136E8E798F80030002BE8D0C1B28C
:100AE000E0B212F069FBE3E72F214846FAF70EFA6D
:100AF000C3E700BF2C450020B3E3020848450020AF
:100B0000FD2B0208BC4900202AE3020840E302084A
:100B1000544500202C29002010B504460B4814F041
:100B20009DFE0B4B1868FEF7AFFB0A4B186814F0DC
:100B30000DF808F0CDFE084B084A24B108490948D1
:100B40000860DA6010BDDA6010BD00BF62E3020821
:100B5000442300205C31002000ED00E00400FA0591
:100B6000FC9F0020EFBEADDE38B5084D2868FEF7CB
:100B70008BFB074B00241C702C71C5F8044109F055
:100B80005BF82046FFF7C8FF2C6038BD44230020E7
:100B9000D14200200120BFE770B5044608460E464A
:100BA00017F0D4FC3146024620461AF090FE08B1F8
:100BB000002070BD18F0A2FB0546304617F0C6FCB9
:100BC000235C1D446A78120701D4002BF0D1013058
:100BD000204470BD2DE9F04F82468FB091460E46FD
:100BE000154600273378089373780993F3780A93AE
:100BF00096F904300B9396F9028096F905300C9320
:100C0000B3790D93B8F1000F04D10FB0BDE8F04FE8
:100C100014F091BEB9F1000F4ED02B78089C6A7881
:100C200095F90210E87895F904E095F905C095F872
:100C300006B09C423ED1099C94423BD1884539D1B3
:100C40000A9C844236D10B9C744533D10C9C64457C
:100C500030D10D9C5C4514BF002401240390029107
:100C600001920093CDF818B0CDF814C0CDF810E083
:100C70003B46124A2146504614F036FF0D9B069320
:100C80000C9B05930B9B04930A9B0393099B019375
:100C9000089B0093CDF808803B46084A2146504601
:100CA000013714F037FF102F06F1070605F107058D
:100CB00098D1AAE70024D1E74C46DFE76EE30208AB
:100CC0002DE9F0478AB0054617F040FC024630B9DE
:100CD00087490120FFF77EFF0AB0BDE8F0870522B3
:100CE000844928461AF0F3FD044660B97022014693
:100CF0007F481AF0A1FD804B20462246C2500C309E
:100D00006028FBD1E8E704227C4928461AF0DFFD81
:100D1000044620BB284614F02FFD06460028DBD0F1
:100D200017F014FCDFF8F881074658F824501DB975
:100D3000734815F02BF8CFE73A46294630461AF0AB
:100D4000C6FD50B9204605F099FA29466D4814F0C1
:100D500009FE6D48FFF7B4FFBEE70134E5E707225F
:100D60006A4928461AF0B3FD0446002875D12021AF
:100D700028461AF096FD064617F0E8FB054680BBAC
:100D8000634814F04CFD2C46624D21462846013440
:100D900014F045FD0E2CF8D114F0CDFDDFF8849150
:100DA000554FDFF8848100242146484614F037FD72
:100DB0000C26DFF878A1002506FB04763268564839
:100DC0000123AB40134214BF41465146013514F094
:100DD00026FD0E2DF2D1013414F0ADFD082CE3D127
:100DE0007AE7304601AA4D494C4E18F0D0FA02ADD0
:100DF00000283DD0022C15D1029A072A2AD803993F
:100E00000D2927D80378722B17D06E2B22D10C23F3
:100E100053433948012202FA01F1C25822EA010281
:100E2000C25013E018F062FA01AA45F824003146D6
:100E3000002018F0ACFA0134DAE70C232E4C5343AF
:100E4000012000FA01F1E0580843E0502F48FFF775
:100E500037FF41E714F0A0FFF8E7284601AA2F4921
:100E60002E4E18F094FA002402AD78B1082C02D16D
:100E700014F092FF30E718F039FA01AA45F824007F
:100E80003146002018F083FA0134EEE7082CEFD148
:100E9000029B0F2BECD8DDF80CC0BCF1070FE7D894
:100EA000049F0D2FE4D8059E06F16402C82ADFD8FE
:100EB000069DFF2DDCD807986428D9D808996429A5
:100EC000D6D88842D4DA099C032CD1D8DFF820E0A8
:100ED000C3EBC3020EEB02030EF802C018715F7081
:100EE0009E70DD7059719C710748FFF7E9FEF3E6CB
:100EF000E82E00208DE30208F42D002093E3020881
:100F00005EE1020898E3020887E20208A2E3020811
:100F100073EB0208AAE30208AFE30208B3E3020896
:100F20008CC60208F2060308E0E302088BE302081D
:100F30002DE9F04FDFF820B189B08046894616468A
:100F40000D4614464FF0000A002E71D06A6863689F
:100F50009A426BD1AF68A368FB1A5F425F4194F974
:100F60000B30049394F90A300393B4F908300293D8
:100F7000B4F906300193B4F9043000935A4653464D
:100F80003946404614F0B0FD95F90B30049395F9BD
:100F90000A300393B5F908300293B5F9063001938E
:100FA000B5F9043000935A465346394640460AF193
:100FB000010A14F0AFFDBAF1080F05F10C0504F1B8
:100FC0000C04C1D10024DFF894A0254696B3002775
:100FD000012303FA07FB325959F8043053403BEA26
:100FE000030314BF0123002312EA0B0F079306D05B
:100FF00000972B4652460799404614F075FD59F864
:1010000004301BEA030F06D000972B46524607997F
:10101000404614F07FFD01370E2FD9D10135082D40
:1010200004F10C04D2D109B0BDE8F08F002796E797
:101030003746A9E73746012359F80420BB4013423D
:1010400006D000972B4652460121404614F062FD1F
:1010500001370E2FEFD1E1E7B5E30208CDE3020837
:10106000F0B585B0054614F07FFB002838D1044662
:101070002B78002B3BD1062C41D1BDF904309AB21C
:10108000072A3CD8BDF90610A1F2EE2292B240F236
:10109000DC54A24233D8BDF90820A2F2EE2080B27F
:1010A000A0422CD8BDF90A00814228DC824226DB0E
:1010B000914224DCBDF90C5005F16404A4B2C82CA3
:1010C0001DD8BDF90E40112C19DC1A4E0C2707FB58
:1010D00003639980DA8018819D72DC7205B0F0BDDF
:1010E00014490022012005B0BDE8F04020E72D2B77
:1010F00003D0A3F13002092A16D8052C04DD05B06F
:10110000BDE8F04014F048BE284618F0EFF804ABF4
:10111000661C03EB440424F80C0C15F8013F303B2B
:10112000092BFAD93446A3E7202BE8D1013526460E
:10113000F8E700BFF42D00202DE9F347DFF868A0A1
:1011400081460F46904602260024B8F1000F28D0B1
:1011500037F8242038F824309A4238F806201ED177
:10116000BD5BA91A4D424D41019200935246234660
:101170002946484614F0B8FCBB5B019337F824308D
:1011800000935246234629464846013414F0C2FCD7
:10119000042C06F10406D8D102B0BDE8F087002582
:1011A000E2E74546E8E700BFE2E302082DE9F04147
:1011B000054614F0D9FA064628B100222849012034
:1011C000BDE8F041B8E7274928461AF03DFB70B961
:1011D000234B4FF47A714FF4FA6219805A80998048
:1011E000DA8019815A819981DA81BDE8F081284637
:1011F00018F07CF80328044629D8284614F0BCFAD5
:10120000064658B118F072F801270546304614F02A
:10121000B3FA30B9BDE8F04114F0BEBD054607464B
:10122000F4E718F063F8002FF4D0A5F2EE2240F2B4
:10123000DC539A42EED8A0F2EE229A42EAD8084B4A
:1012400023F8245003EB84035880BDE8F081324634
:10125000032305490548BDE8F04114F083BB00BFF6
:10126000F02500208DE30208F3E30208ACE1020858
:101270002DE9F04F2DED088BDFF80C9193B08046EF
:1012800092460D461446002695ED008AB5EE408A3A
:10129000F1EE10FA71D0D5ED019A95ED029AD5EDE7
:1012A000038ABAF1000F3FD094ED000A94ED01BA21
:1012B000D4ED02AA94ED03AAB4EE408AF1EE10FA3E
:1012C00060D1F4EE4B9AF1EE10FA5BD1B4EE6A9A6B
:1012D000F1EE10FA56D1F4EE4A8AF1EE10FA0CBF94
:1012E000012700270FA8F9F733FCB0EE4B0A83461D
:1012F0000CA8F9F72DFCB0EE6A0A059009A8F9F7D9
:1013000027FCB0EE4A0A049006A8F9F721FC049ADB
:10131000059B039002920193CDF800B033464A46F4
:101320003946404614F0E0FBB0EE480A0FA8F9F742
:101330000FFCB0EE690A07460CA8F9F709FCB0EEFD
:10134000490A834609A8F9F703FCB0EE680A04903D
:1013500006A8F9F7FDFB049B039002938DE8800833
:1013600033464A4600214046013614F0D3FB0C2E8A
:1013700005F1100504F1100486D113B0BDEC088B03
:10138000BDE8F08F0027ADE7FBE302082DE9F04749
:10139000494E4A4FDFF840810446204614F0E4F9F4
:1013A000814628B1002246490120BDE8F0475FE7A9
:1013B0000522314620461AF08AFA40B940490022F7
:1013C00043181030C0281A60FAD1BDE8F087042213
:1013D000394620461AF07BFA0546204615BB14F024
:1013E000CBF98146002865D017F0B0F82C465FFA9B
:1013F00080FA58F8245025B93248BDE8F04714F077
:10140000C5BC5246294648461AF061FA40B9204602
:1014100013F08CFA29462C482C4C14F0A3FABCE7A4
:101420000134E6E717F062FF0B2805463AD820465C
:1014300014F0A2F9064648B3F9F7E2FA204B03EBA1
:10144000051383ED000A0124304614F095F9064691
:1014500038B1F9F7D5FA1A4B03EB051383ED010AFE
:101460000134304614F088F9064638B1F9F7C8FA65
:10147000134B03EB051383ED020A0134304614F0DD
:101480007BF928B9BDE8F04714F086BC0446DBE7D9
:10149000F9F7B6FA0A4B032C03EB051585ED030AA1
:1014A000F0D17FE74A460B2309490A48BDE8F047D7
:1014B00014F058BABDE8F0878DE3020893E3020800
:1014C000406200205EE1020898E3020887E2020819
:1014D000A6E10208ACE102088CC602082DE9F04F33
:1014E000834687B092460C46154600274FF01909EF
:1014F0004FF46178BAF1000F4ED023782A789342E6
:101500002B7947D160786978884243D1A078A9784F
:1015100088423FD1E078E97888423BD121799942ED
:1015200038D166796979711A4E424E410593EB784C
:101530000493AB7819FB038303936B78019219FB37
:10154000038302936B790093144A3B463146584615
:1015500014F0CAFA23790593E3780493A3780F4A29
:1015600019FB03830393637819FB038302932378A6
:1015700001936379009331463B465846013714F096
:10158000C9FA0F2F04F1060405F10605B2D107B020
:10159000BDE8F08F0026C9E75646DBE70FE40208F6
:1015A000F7B5074614F0E0F8044630B1002236499A
:1015B0000120FFF793FF03B0F0BD384617F096FE09
:1015C0000E28054659DC06264643781C8DF8074050
:1015D00014F0D2F82C4C074650B117F087FE0328C0
:1015E00006D8A31958719DF8073001338DF80730DC
:1015F000384614F0C1F8074658B117F077FE0D28A9
:1016000007D806236B43E0549DF8073001338DF86B
:101610000730711C0DF107022144384614F0B9F867
:1016200014F0AAF8074660B117F060FE182808D831
:10163000062303FB0543D8709DF8073001338DF86E
:101640000730384614F098F860B117F04FFE0D28B7
:1016500008D8062303FB05459DF8073028710133A0
:101660008DF807309DF80730062BA4D0A21900236F
:10167000A351938014F090FB9DE70E23224603496B
:10168000034814F06FF996E744300020A6E1020801
:10169000ACE102080020704700207047014B33F88E
:1016A000110070474C240020044B93F8240018B11B
:1016B000002283F824200120704700BF4C24002022
:1016C000024B03EB8101088D704700BF4C240020C2
:1016D00003788B4283BF034B03EB4101B1F86000F9
:1016E000002070474C24002070B4024601210023E2
:1016F00005261E2502E0013302320131032BCCBF47
:101700000124002400F8134004D012295570F2D1AE
:1017100070BC70475670EEE7024B03604360836015
:10172000C3607047E803D007014B33F811007047DE
:101730001C550020014B33F8110070471C55002048
:101740002DE9F0416D4D95F88030022B02D000203C
:10175000BDE8F08195F88640E4B1013CE4B2013483
:1017600005F184000444002210F8013B534083EA51
:101770000313DBB2120AD90042EA0322A04281EA33
:10178000131382EA0302EFD122B1002085F8800012
:10179000BDE8F081B5F884305BBA9BB243F60162D4
:1017A000934209D043F60362934205D0002385F8A3
:1017B00080300120BDE8F08195F88B7095F88AC0E3
:1017C00095F88D6095F88F1095F8914095F89300F5
:1017D00095F88C2095F88E3095F890E095F89B80E0
:1017E0000CEB072C95F8927002EB062203EB012319
:1017F00095F8946095F895100EEB042E07EB0027F2
:1018000095F8964095F89700CCF3CC0CC2F3CC0237
:1018100006EB012604EB002495F8991095F8980042
:10182000A5F860C0A5F8622095F89DC095F89C20A9
:10183000C3F3CC0300EB0120A5F8643095F89A10AF
:1018400095F89E3002EB0C2295F89FC001EB082121
:1018500003EB0C23CEF3CC0EC7F3CC07C6F3CC06B8
:10186000C4F3CC04C0F3CC00C1F3CC01C2F3CC026E
:10187000C3F3CC03A5F866E0A5F86870A5F86A6024
:10188000A5F86C40A5F86E00A5F87010A5F87220B8
:10189000A5F8743095F8A53095F8A41095F8A1C076
:1018A00095F8A04095F8A3E095F8A20095F8A770E8
:1018B00095F8A62095F8A96001EB032195F8A830CA
:1018C00004EB0C2400EB0E2002EB072203EB0623B3
:1018D000C4F3CC04C0F3CC00C1F3CC01C2F3CC02FE
:1018E000C3F3CC03A5F87640A5F87800A5F87A10E4
:1018F000A5F87C20A5F87E3058E700BF4C240020D6
:1019000010B50446FCF7FAFA2E4BD3F8AC20821A35
:10191000B2F5FA7F11D90022C3F8AC0083F8B020E9
:1019200083F8B120E1B204291DD020291BD093F8FF
:10193000B420A2B3944243D010BD93F8B12052BB5F
:1019400093F8B020C3F8AC00002AEBD0E1B293F8D2
:10195000B2009C180138824284F8BC1017D00132C2
:1019600083F8B02010BD002202244FF6FF7083F8E8
:10197000B840A3F8B6009C18481E824283F8B41001
:1019800083F8B21083F8B32084F8BC10E7D10122A9
:1019900083F8DC2010BD013A83F8B12010BD552C2E
:1019A000C8D101211F2083F8B440A3F8B62083F8E2
:1019B000BC4083F8B31083F8B81083F8B200CEE7C8
:1019C0000022C4E74C24002038B5394C0546FCF70A
:1019D00095FAD4F8EC30C4F8EC00C01AB0F57A7F70
:1019E0001CDD0023282284F8F03084F8803084F84D
:1019F000F23084F8F1203D2D42D03E2D0DD12D4AFC
:101A0000C4F8F420012384F880300123157084F891
:101A1000F03094F8F1209A4220D038BD94F8F020AC
:101A2000002AE8D0531CDBB2D4F8F41084F8F0306C
:101A3000062B8D54EDD194F88030012B2BD094F8E7
:101A4000F230012B23D00023282284F8F03084F8D0
:101A5000803084F8F23084F8F12038BD94F880307A
:101A6000012B04BF022384F8803094F8F230012B5C
:101A700015D00022282384F8F02084F8F13038BDF6
:101A80000D4AC4F8F420012384F8F230BDE78B78C6
:101A9000092BF2D9D7E78B78282BD0D8EDE7022392
:101AA00084F8F230FCF72AFAC4F8F800E1E700BF46
:101AB0004C240020D02400202C2500202DE9F843C0
:101AC0002C220646002119F0B7FE1E23194FB375CC
:101AD00040F2DC5440F24C4040F26C71022213237D
:101AE000348370830E2440F24650B183B27740F2C3
:101AF000753140F6430286F820300F4D86F82240BB
:101B00000123F184B084328573723375B84607F1CE
:101B1000080900244121404619F0C3FEC31B10B13F
:101B2000484538BFF45415F8011F01340029F2D19B
:101B3000BDE8F88334DA020830E402082DE9F04FFA
:101B4000D94C94F8DC3089B023B90023184609B089
:101B5000BDE8F08F94F8B3300022012B84F8DC202C
:101B600000F0E38094F8B250AE1E00F0988104F1CA
:101B7000BC0188194FF6FF7311F8012B9B1A8142A3
:101B80009BB2F9D1190A254495F8BB208A42DCD1D1
:101B90002644DBB296F8BC209A42D6D194F8B430F1
:101BA000202B40F0758194F8B8108B1C009301F144
:101BB0000803019301F10A03039301F10C03049359
:101BC00001F10E03059301F11003069301F11603D1
:101BD00001F1040C01F1060901F1120801F11407E9
:101BE000029301F1180A01F11A0B9DF8003054FA22
:101BF00083F29DF8043054FA83F307939DF80C3078
